:100000000C9405060C942D060C942D060C942D06CC
:100010000C942D060C942D060C942D060C942D0694
:100020000C94AF070C942D060C942D060C942D0601
:100030000C942D060C942D060C942D060C942D0674
:100040000C942D060C942D060C9491660C942D06A0
:100050000C9492670C94D9670C942D060C942D0681
:100060000C942D060C942D060C947A630C942D069A
:1000700050726F6772616D20006C6F630077746BF4
:10008000657900747474006376006A6300647000BC
:100090006370006372007570006A7000636F006ABD
:1000A0006F007370006A7300636D006373006A6EA3
:1000B000006A6C00646C007375006375007765619D
:1000C000746865722E6F70656E737072696E6B6C9A
:1000D00065722E636F6D002F7765617468657200BD
:1000E00024442E70793F6C6F633D2445266B6579FF
:1000F0003D2445266677763D244400747A00736378
:10010000616C650073756E7365740073756E7269EA
:10011000736500485454502F312E30203230302037
:100120004F4B0D0A0043616368652D436F6E747217
:100130006F6C3A206D61782D6167653D36303438DB
:1001400030302C207075626C69630D0A00436F6E4D
:1001500074656E742D547970653A20746578742FC7
:100160006373733B636861727365743D7574662D68
:10017000380D0A436F6E74656E742D456E636F643F
:10018000696E673A20677A69700D0A00436F6E7472
:10019000656E742D547970653A20746578742F6A91
:1001A0006176617363726970743B636861727365D1
:1001B000743D7574662D380D0A436F6E74656E74E8
:1001C0002D456E636F64696E673A20677A69700DBA
:1001D0000A000D0A00244600244600244624460056
:1001E0003C7363726970743E77696E646F772E6CCE
:1001F0006F636174696F6E3D222F223B3C2F7363E6
:10020000726970743E0A007B22726573756C742289
:100210003A24447D007B22726573756C74223A2403
:10022000447D00244600222446223A24447D006472
:100230006179005D002C2453002453005B00747925
:10024000706500656E640073746172740068697330
:1002500074007400656E00736964005D2C226E7317
:10026000746174696F6E73223A24447D002C0024FB
:10027000440022736E223A5B00637077006E7077E1
:10028000007474740077746B6579006C6F63006A36
:10029000737000726400656E007262740072736E37
:1002A000002C2264657870223A24442C226D6578F3
:1002B00070223A24447D002C00222446223A244411
:1002C000003C6D657461206E616D653D22766965E7
:1002D00077706F72742220636F6E74656E743D2246
:1002E00077696474683D6465766963652D776964D0
:1002F00074682C696E697469616C2D7363616C65D7
:100300003D312E302C6D696E696D756D2D73636195
:100310006C653D312E302C757365722D7363616C85
:1003200061626C653D6E6F223E0D0A003C73637224
:10033000697074207372633D2224452F686F6D6568
:100340002E6A73223E3C2F7363726970743E0A3CBE
:100350002F626F64793E0A3C2F68746D6C3E0076A4
:100360006172207665723D24442C697061733D246E
:10037000443B3C2F7363726970743E0A003C214415
:100380004F43545950452068746D6C3E0A3C687464
:100390006D6C3E0A3C686561643E0A24463C2F68E9
:1003A0006561643E0A3C626F64793E0A3C73637225
:1003B0006970743E005B302C305D5D2C226C727570
:1003C0006E223A5B24442C24442C24442C244C5D7F
:1003D0007D005B24442C244C2C244C5D2C00305D8F
:1003E0002C227073223A5B0024442C002264657630
:1003F00074223A244C2C226E627264223A24442CD9
:1004000022656E223A24442C227264223A24442C1F
:10041000227273223A24442C2272647374223A2486
:100420004C2C226C6F63223A222445222C227774B2
:100430006B6579223A222445222C2273756E7269EB
:100440007365223A24442C2273756E736574223AC4
:1004500024442C227362697473223A5B006E616DCE
:1004600065007069640070696400706964005D7D96
:1004700000225D00225D2C00245300244C5D2C22C0
:1004800000244C2C0024445D2C5B0024442C005B95
:1004900024442C24442C24442C5B00226E70726F64
:1004A0006773223A24442C226E626F617264732255
:1004B0003A24442C226D6E70223A24442C226D6E14
:1004C0007374223A24442C22706E73697A65223A3E
:1004D00024442C227064223A5B003C6872202F3E38
:1004E0003C666F726D206E616D653D6F6620616365
:1004F00074696F6E3D6375206D6574686F643D67E8
:1005000065743E3C703E3C623E5363726970742079
:1005100055524C3A3C2F623E3C696E7075742074A3
:100520007970653D746578742073697A653D3332FE
:10053000206D61786C656E6774683D313237207666
:10054000616C75653D22244522206E616D653D6AB2
:1005500073703E3C2F703E3C703E44656661756C26
:10056000742069732024533C6272202F3E49662018
:100570006C6F63616C206F6E2075534420636172F1
:10058000642C20757365202E2F3C2F703E3C703EEE
:100590003C623E50617373776F72643A3C2F623EE7
:1005A0003C696E70757420747970653D7061737309
:1005B000776F72642073697A653D3332206E616DA6
:1005C000653D70773E3C696E707574207479706516
:1005D0003D7375626D69743E3C2F703E3C687220BD
:1005E0002F3E3C2F666F726D3E005D2C226D617850
:1005F0006C656E223A24447D0073746E5F7365717E
:1006000000726673746E0073746E5F646973006168
:1006100063745F72656C61790069676E6F72655FA4
:100620007261696E006D61736F70002C002224533B
:10063000220022736E616D6573223A5B002C0024E8
:1006400044005D2C222446223A5B00707700436F01
:100650006E74656E742D547970653A206170706C9B
:1006600069636174696F6E2F6A736F6E0D0A436FF1
:100670006E6E6E656374696F6E3A20636C6F73653E
:100680000D0A004163636573732D436F6E74726F5F
:100690006C2D416C6C6F772D4F726967696E3A20D3
:1006A0002A0D0A00507261676D613A206E6F2D63EA
:1006B000616368650D0A0024462446244624460DDD
:1006C0000A7B0024462446244624460D0A00436F34
:1006D0006E74656E742D547970653A207465787403
:1006E0002F68746D6C0D0A00244624462446244667
:1006F0000D0A005D0D0A002C00222C00302C220077
:100700002C002C005B002E747874004E5450205343
:10071000796E63696E672E2E2E004465746563746E
:10072000696E67207553442E2E2E00302E2054659E
:100730007374202831206D696E29002E200020005E
:10074000486F6C6420423320746F2073746172743C
:1007500000436C69636B20423320746F206C6973B3
:10076000740052756E20612050726F6772616D3A2D
:10077000003A000001080006040001450000820064
:100780000040002000504F53542024462048545429
:10079000502F312E300D0A486F73743A2024460DC5
:1007A0000A244624534163636570743A202A2F2A31
:1007B0000D0A436F6E74656E742D4C656E677468B8
:1007C0003A2024440D0A436F6E74656E742D54797B
:1007D00070653A206170706C69636174696F6E2F27
:1007E000782D7777772D666F726D2D75726C656ECB
:1007F000636F6465640D0A0D0A2453004745542055
:100800002446245320485454502F312E300D0A488A
:100810006F73743A2024460D0A24460D0A0D0A000F
:100820004163636570743A20746578742F68746DE1
:100830006C00E30004FA0001000000016677760016
:10084000747A006E747000646863700069703100BF
:100850006970320069703300697034006777310065
:10086000677732006777330067773400687030004D
:100870006870310068777600657874005F00736493
:1008800074006D6173006D746F6E006D746F66003F
:100890007572730072736F00776C0064656E006927
:1008A00070617300646576696400636F6E006C69E3
:1008B000740064696D00726C7000757774006E74FA
:1008C0007031006E747032006E747033006E74702C
:1008D00034006C67007265736574004669726D77E9
:1008E0006172653A2000545A6F6E653A004E54505A
:1008F0003F0055736520444843503F005374617472
:1009000069632E6970313A005374617469632E69AA
:1009100070323A005374617469632E6970333A001F
:100920005374617469632E6970343A004761746569
:100930007761792E6970313A004761746577617922
:100940002E6970323A00476174657761792E69705B
:10095000333A00476174657761792E6970343A00E3
:100960004854545020706F72743A000048617264A9
:10097000776172653A20004578702E20626F61724F
:10098000643A000053746E2064656C61793A004DDE
:1009900061732E2073746174696F6E3A004D6173D8
:1009A0002E20206F6E2061646A2E3A004D61732EF6
:1009B000206F66662061646A2E3A005261696E207B
:1009C00073656E736F723A004E6F726D616C6C7905
:1009D000206F70656E3F002520576174657220742A
:1009E000696D653A0044657669636520656E61628C
:1009F0006C653F0049676E2070617373776F726436
:100A00003F004465762E2049443A004C434420631D
:100A10006F6E74726173743A004C43442062616378
:100A20006B6C696768743A004C43442064696D6D6F
:100A3000696E673A0052656C61792070756C7365F8
:100A40003A0055736520776561746865723F004EA2
:100A500054502E6970313A004E54502E6970323A1B
:100A6000004E54502E6970333A004E54502E697027
:100A7000343A00456E61626C65206C6F6767696E21
:100A8000673F00526573657420616C6C3F004D6F69
:100A90006E005475650057656400546875004672B1
:100AA00069005361740053756E008E0A920A960AAB
:100AB0009A0A9E0AA20AA60A206D73002073656333
:100AC00000207365630025004E6F00596573002B8D
:100AD000002B0020474D54003030003A002D002BF1
:100AE000000020202020002D44697361626C656441
:100AF000212D003A0045004D433A002D002D004DB8
:100B000041433A002E002D0020002020003A002012
:100B100000486F6C6420423320746F2073617665E7
:100B20000042312F42323A2B2F2D2C2042333A2DC6
:100B30003E003D3D536574204F7074696F6E733D88
:100B40003D00506C6561736520576169742E2E2ECF
:100B500000526573657474696E67204465766963D5
:100B60006500436F6E6E656374696E672E2E2E008E
:100B70007C3C3E5E2B3D3F2F5B5D3B2C2A225C0084
:100B800000002100240027002A0000002200250088
:100B900028002B000000200023002600290002026C
:100BA0000202020202020404040404040404030313
:100BB0000303030303030101010101010101010218
:100BC0000408102040800102040810204080010227
:100BD000040810204080804020100804020100001A
:100BE00000010200000000000000040307060000EE
:100BF000000000000000000000000000000051089C
:100C0000BD2D673B2A511662B96811241FBECFEF74
:100C1000D0E1DEBFCDBF13E0A0E0B1E0ECE0F6ED47
:100C200002C005900D92AC35B107D9F71DE0ACE5D7
:100C3000B3E001C01D92AA3FB107E1F71BE0CAE093
:100C4000DCE004C02297FE010E94C96ACE3FD107B2
:100C5000C9F70E94296A0C94046B0C940000FC01F3
:100C600088279927E89421912032E9F3293010F060
:100C70002E30C8F32B3241F02D3239F4689404C081
:100C80000E945407820F911D219120532A30C0F3F6
:100C90001EF4909581959F4F08951F93FC0199270D
:100CA0008827BC01E89411911032E9F3193010F053
:100CB0001E30C8F31B3251F01D3249F4689406C04F
:100CC0000E943F07610F711D811D911D11911053ED
:100CD0001A30B0F33EF490958095709561957F4FF2
:100CE0008F4F9F4F1F910895FB01DC0102C00590BB
:100CF0000D9241505040D8F70895FB01DC010D9052
:100D00000020E9F7119705900D920020E1F7089572
:100D1000FB01DC0105900D920020E1F70895FB0135
:100D2000DC0104C08D910190801921F441505040A4
:100D3000C8F7881B990B0895FB01DC0102C00190E4
:100D40000D9241505040D8F70895DC0101C06D93D9
:100D500041505040E0F70895FB01DC010D90002068
:100D6000E9F7119701900D920020E1F70895FC0139
:100D70008191861721F08823D9F799270895319713
:100D8000CF010895FB01DC0101900D920020E1F7F5
:100D90000895FB01DC014150504030F08D910190ED
:100DA000801919F40020B9F7881B990B0895FB01ED
:100DB000DC014150504048F001900D920020C9F7ED
:100DC00001C01D9241505040E0F70895A0E0B0E00E
:100DD000ECEEF6E00C94D76A7C01EB018A01690124
:100DE00009C0CE012196F6010995F70181937F0193
:100DF0000150104001151105A1F7CDB7DEB7E8E0AD
:100E00000C94F36AA0E0B0E0E8E0F7E00C94D76A55
:100E1000EC017B018A01690109C0CE012196F7012D
:100E200061917F01F60109950150104001151105EE
:100E3000A1F7CDB7DEB7E8E00C94F36AFB019F01A0
:100E4000E8944230C4F04532B4F44A3029F497FBB8
:100E50001EF4909581959F4F642F77270E94636AB7
:100E6000805D8A330CF0895D8193CB010097A1F7F7
:100E700016F45DE251931082C9010C948107592F39
:100E8000482F372F262F660F771F881F991F660F51
:100E9000771F881F991F620F731F841F951F660F8E
:100EA000771F881F991F08957AE0979F902D879F3D
:100EB000802D910D11240895FA01CF93FF93EF93A4
:100EC0002230CCF02532BCF4C22F2C2F33274427FC
:100ED0005527FF93EF930E948A6AEF91FF91605D1F
:100EE0006A330CF0695D6193B901CA0160507040CA
:100EF0008040904051F710828F919F91CF910C9438
:100F00008107DC01FC01672F71917723E1F73297AC
:100F100004C07C916D9370836291AE17BF07C8F3D4
:100F200008959C01F999FECF32BD21BDF89A80B594
:100F300008959C01F999FECF1FBA32BD21BD60BD55
:100F40000FB6F894FA9AF99A0FBE0895FC01A6819B
:100F5000B7816D93B783A68381E090E008951F92D7
:100F60000F920FB60F9211242F933F934F935F93DD
:100F70006F937F938F939F93AF93BF93EF93FF9361
:100F8000809169078F5F809369078091690780313D
:100F900028F0E0916707F09168070995FF91EF91BC
:100FA000BF91AF919F918F917F916F915F914F9181
:100FB0003F912F910F900FBE0F901F901895ABEEA1
:100FC000B8E080E090E0FC01E559F84F1082118212
:100FD00012821382FC01E55DF74F108211821282AA
:100FE00013821D920496803C910569F710922309A3
:100FF000109224091092250910922609F999FECF22
:1010000089E090E092BD81BDF89A80B580936A072F
:101010000895982F80916A07981708F041C0992386
:1010200009F43EC0892F90E0019727E430E0AC013D
:10103000429FC001439F900D529F900D11249C012F
:10104000265F3F4F8F5A9F4F24C0F999FECF32BD84
:1010500021BDF89A50B5F999FECF72BD61BDF89ADD
:1010600040B5F999FECF1FBA32BD21BD40BD0FB6C4
:10107000F894FA9AF99A0FBEF999FECF1FBA72BD89
:1010800061BD50BD0FB6F894FA9AF99A0FBE2F5F62
:101090003F4FB901695B7F4F2817390709F0D5CF5A
:1010A000089510922A071092290785ED92E09093F7
:1010B00028078093270789E1809330071092330730
:1010C0001092460710924D0710924F070895AF9265
:1010D000BF92DF92EF92FF920F931F93CF93DF9314
:1010E00000D000D007E217E0ADB7BEB712961C9350
:1010F0000E93119782E792E014969C938E93139728
:101100000E94DD36FF240F900F900F900F90D02E8D
:10111000E12E9FE6A92E92E0B92ECDE6D2E04FC097
:101120000F2D10E000D000D000D0ADB7BEB71196A3
:10113000EDB7FEB7D182E2821396BC92AE921297BF
:10114000F80183E0F595E7958A95E1F7E25FF54FC1
:10115000808190E098012770307002C09595879546
:101160002A95E2F78170907015969C938E93149750
:101170000E94DD3680910D0A90E001972DB73EB7B1
:101180002A5F3F4F0FB6F8943EBF0FBE2DBF081722
:101190001907A1F000D000D0ADB7BEB71196DC9210
:1011A00011971296EC9212971496DC93CE931397A4
:1011B0000E94DD360F900F900F900F90F3942091C6
:1011C0000D0AF21608F4ACCF00D000D000D0EDB775
:1011D000FEB7319687E297E0ADB7BEB712969C9303
:1011E0008E9311978BE592E09383828324831582FB
:1011F0000E94DD36EDB7FEB736960FB6F894FEBF07
:101200000FBEEDBFDF91CF911F910F91FF90EF9037
:10121000DF90BF90AF9008958F929F92AF92BF9250
:10122000DF92EF92FF920F931F93CF93DF93EB0127
:1012300000D000D000D0EDB7FEB7319607E217E03E
:10124000ADB7BEB712961C930E93119722E436E009
:1012500033832283958384830E94DD36FF24EDB798
:10126000FEB736960FB6F894FEBF0FBEEDBFD02E78
:10127000E12E3FE3832E36E0932E2DE3A22E26E0CF
:10128000B22E40C000D000D000D0ADB7BEB711968E
:10129000EDB7FEB7D182E28213969C928E9212979E
:1012A0000F2D10E0FE01E00FF11F808114968C934A
:1012B000149715961C920E94DD3680910C0A90E0DE
:1012C00001972DB73EB72A5F3F4F0FB6F8943EBF48
:1012D0000FBE2DBF08171907A1F000D000D0ADB781
:1012E000BEB71196DC9211971296EC921297149653
:1012F000BC92AE9213970E94DD360F900F900F9024
:101300000F90F39480910C0AF81608F4BBCFDF918C
:10131000CF911F910F91FF90EF90DF90BF90AF9012
:101320009F908F9008958DB79EB70C970FB6F89445
:101330009EBF0FBE8DBFEDB7FEB7319687E297E037
:10134000ADB7BEB712969C938E93119787EB96E03C
:101350009383828383E191E0958384838EE496E096
:101360009783868383E896E09187808784EA96E076
:10137000938782870E94DD368DB79EB70C960FB695
:10138000F8949EBF0FBE8DBF08950E9493090E94DE
:10139000670880E008958DB79EB70C970FB6F89454
:1013A0009EBF0FBE8DBFEDB7FEB7319687E297E0C7
:1013B000ADB7BEB712969C938E93119783EC96E0CF
:1013C0009383828383E191E0958384838EE496E026
:1013D0009783868383E896E09187808784EA96E006
:1013E000938782870E94DD368DB79EB70C960FB625
:1013F000F8949EBF0FBE8DBF08958DB79EB70C9712
:101400000FB6F8949EBF0FBE8DBFEDB7FEB73196F5
:1014100087E297E0ADB7BEB712969C938E93119773
:1014200088EE96E09383828383E191E095838483C1
:101430008EEC96E09783868384EA96E09187808796
:1014400083E896E0938782870E94DD368DB79EB74A
:101450000C960FB6F8949EBF0FBE8DBF08950E94E4
:10146000FD098DB79EB708970FB6F8949EBF0FBEC3
:101470008DBFEDB7FEB7319687E297E0ADB7BEB747
:1014800012969C938E9311978AED94E093838283B6
:1014900084E494E09583848380E091E0978386835D
:1014A0000E94DD368DB79EB708960FB6F8949EBFA2
:1014B0000FBE8DBF80E008950F931F93DF93CF93EE
:1014C000CDB7DEB728970FB6F894DEBF0FBECDBFFD
:1014D0008091E009882329F48DEB90E060E00E9480
:1014E000B9370EEA16E01C821B8285ED92E09A83E2
:1014F00089831E830D8318870F838DB79EB70C9742
:101500000FB6F8949EBF0FBE8DBFEDB7FEB73196F4
:10151000CE010196ADB7BEB712969C938E931197EC
:1015200080EE90E09383828380919A028483158277
:1015300084E194E09783868384E894E091878087B0
:101540008091E001828713860E94DD36D8010D90DC
:101550000020E9F71197A01BB10BA00FB11F25E2E6
:1015600037E0EDB7FEB73C960FB6F894FEBF0FBE5E
:10157000EDBF50E342E395E213C08C91B901615095
:101580007040803249F4F9015083FB01408392930B
:101590009F012150304003C0F90180839B011197C6
:1015A000F6E0AE3ABF0749F78C91D9018C93809150
:1015B000060A8F7B8093060A0091DE011091DF01FD
:1015C00080E590E09093DF018093DE0187ED90E06D
:1015D000B9014DEB50E02EE63BE00E948D2E1093BA
:1015E000DF010093DE0128960FB6F894DEBF0FBE30
:1015F000CDBFCF91DF911F910F910895AF92BF9210
:10160000CF92DF92EF92FF920F931F937B018C0199
:101610008091070A82958F7079F58091060A83FD83
:101620002BC086FF03C084E893E002C08EE190E007
:101630002091480A3091490A40914A0A50914B0A38
:10164000211531054105510569F057016801A21ABC
:10165000B30AC40AD50AA0E0B0E08A159B05AC0520
:10166000BD0550F4E092480AF092490A00934A0AF4
:1016700010934B0A0E945C0A1F910F91FF90EF900C
:10168000DF90CF90BF90AF900895EF92FF920F93AD
:101690006EEA76E048E726E634E001E0EE24FF2437
:1016A0000E944035882311F480E114C08EEA96E050
:1016B0000E942F069C01181619065CF480916A0797
:1016C00090E0281739072CF4822F0E94090881E046
:1016D00001C081E10F91FF90EF900895EF92FF928A
:1016E0000F93CF93DF93EB01C45ADC4F01C02196D7
:1016F0008881882309F480C08632C9F76EC08EEADB
:1017000096E00E942F069C0185E0213A380720F4DC
:101710003093FF092093FE09CE016EEA76E048E798
:1017200024E031E001E0EE24FF240E9440358823CC
:1017300069F08EEA96E00E942F069C0185E0213A2E
:10174000380720F43093010A2093000A0E94F23FE8
:10175000CE016EEA76E048E72EEF30E001E0EE24BD
:10176000FF240E944035882359F08EEA96E00E94BB
:101770002F068B3F910520F480936A020E94B33AB2
:10178000CE016EEA76E048E72BEF30E001E0EE2490
:10179000FF240E9440358823D1F08EEA96E00E9413
:1017A0002F069C018136910590F48091E60190E02E
:1017B0002817390761F02093E6011092440A10922D
:1017C000450A1092460A1092470A0E94B33A809145
:1017D000060A80648093060A0FC0CE016EEA76E0A6
:1017E00048E72BE031E001E0EE24FF240E94403581
:1017F000882309F491CF83CFDF91CF910F91FF9090
:10180000EF9008956F927F928F929F92BF92CF92A6
:10181000DF92EF92FF920F931F93DF93CF93CDB799
:10182000DEB728970FB6F894DEBF0FBECDBF80910C
:10183000A00289838091A6028A838091AC028B8367
:101840008091B2028C83BB243E010894611C711C00
:1018500045E0842E912C8C0E9D1E6091D7016F5F08
:101860006093D701C3010E940E310E94E5666B01AF
:101870007C0188EE93E0A0E0B0E0C80ED91EEA1E1D
:10188000FB1E0E948F4A8C010E94AC31012B09F48F
:1018900041C0C4016091D7010E94412E8823D1F13B
:1018A000ED80FE800F81188580EC98EDA4E5BCE703
:1018B000E80EF91E0A1F1B1F6091E60170E080E030
:1018C00090E024E833E040E050E00E94386AE60E01
:1018D000F71E081F191F08C0B39494E1B91609F048
:1018E000BCCFEE24FF248701B701C80128960FB6AC
:1018F000F894DEBF0FBECDBFCF91DF911F910F9146
:10190000FF90EF90DF90CF90BF909F908F907F904F
:101910006F9008950E94E5666C157D058E059F0504
:1019200008F4AFCFD9CFCF92DF92EF92FF920F930F
:101930001F93DF93CF93CDB7DEB76E970FB6F894B2
:10194000DEBF0FBECDBF7C018FE297E0B7010E94E2
:101950003E4C882309F4E9C0CE010196B70141E06D
:101960000E94CC618DB79EB708970FB6F8949EBFC2
:101970000FBE8DBFEDB7FEB7319657E2C52E57E0CB
:10198000D52EADB7BEB71296DC92CE9211978BEDE5
:1019900091E09383828383E191E09583848385E260
:1019A00091E0978386830E94DD36D7010D90002059
:1019B000E9F78D010E191F09055010400E0D1F1D6E
:1019C000EDB7FEB738960FB6F894FEBF0FBEEDBF69
:1019D000C8016FE171E044E050E00E94C906009741
:1019E00099F400D000D000D0EDB7FEB73196ADB776
:1019F000BEB71296DC92CE92119788ED91E0938358
:101A000082838DE491E01BC0C80164E271E044E090
:101A100050E00E94C9060097F1F400D000D000D039
:101A2000EDB7FEB73196ADB7BEB71296DC92CE9247
:101A3000119785ED91E0938382838CE891E0958303
:101A400084830E94DD36EDB7FEB736960FB6F89464
:101A5000FEBF0FBEEDBF00D000D087E297E0ADB76C
:101A6000BEB712969C938E93119782ED91E01496D7
:101A70009C938E9313970E94DD360F900F900F90DA
:101A80000F9080912D0790912E0720912B07309178
:101A90002C07821B930B60E140E00E94802F109284
:101AA0002A071092290782E993E090932C078093EC
:101AB0002B0790932E0780932D078E010B5F1F4FEE
:101AC00019C0C80162E973E04CE153E00E94C054C0
:101AD0009C01442737FD4095542F2C31B3E03B0740
:101AE000B0E04B07B0E05B07B0F0C90160E143E054
:101AF0000E94802F2F89388D498D5A8D8F85988926
:101B0000A989BA89281739074A075B07D1F620E067
:101B100030E040E050E0C90161E143E00E94802FE5
:101B2000CE0105960E949A5481E06E960FB6F89405
:101B3000DEBF0FBECDBFCF91DF911F910F91FF9000
:101B4000EF90DF90CF9008950F931F930E94AA2BE0
:101B50000E94FD0900D000D000D0EDB7FEB731964D
:101B600007E217E0ADB7BEB712961C930E9311971C
:101B70008DE793E09383828381EC92E09583848365
:101B80000E94DD3600D0EDB7FEB73196ADB7BEB7D7
:101B900012961C930E9311978FE593E093838283A3
:101BA00083ED90E09583848380917602868317820B
:101BB0000E94DD360F900F90EDB7FEB73196ADB7AE
:101BC000BEB712961C930E9311978CE293E0938309
:101BD000828384E494E0958384830E94DD368DB70C
:101BE0009EB706960FB6F8949EBF0FBE8DBF80E0DD
:101BF0001F910F9108954F925F926F927F928F92F3
:101C00009F92AF92BF92CF92DF92EF92FF920F938B
:101C10001F93DF93CF930F92CDB7DEB70E94AA2B0D
:101C20005B016C012DB73EB72C5130400FB6F894D4
:101C30003EBF0FBE2DBFEDB7FEB7319607E217E0EE
:101C4000ADB7BEB712961C930E9311978CEE93E02E
:101C500093838283A482B582C682D78280910C0A44
:101C6000808711868091060A817082871386809111
:101C7000060A86958170848715868091060A869566
:101C800086958170868717868091020A9091030A53
:101C9000A091040AB091050A808B918BA28BB38B23
:101CA00084E194E0958B848B84E894E0978B868B19
:101CB0008091FE099091FF09918F808F8091000A99
:101CC0009091010A938F828F0E94DD3690E0EDB7EC
:101CD000FEB77C960FB6F894FEBF0FBEEDBF78013D
:101CE00008EE13E023C000D000D000D0EDB7FEB75F
:101CF0003196ADB7BEB71196EC9211971296FC9241
:101D000013830283A92FB0E0A25FB54F8C91848327
:101D1000158299830E94DD3699819F5FEDB7FEB7EA
:101D200036960FB6F894FEBF0FBEEDBF80910C0A39
:101D3000F7E26F2EF7E07F2E9817A8F200D000D0C0
:101D4000ADB7BEB712967C926E9211978EED93E06E
:101D500014969C938E9313970E94DD3699240F90CE
:101D60000F900F900F90C301762C892EE2ED4E2E2E
:101D7000E3E05E2E64C0A92DB0E0FD01E551F74F10
:101D80006081662329F420E030E040E050E025C087
:101D9000CD01880F991F880F991FFC01E559F84F55
:101DA000E080F18002811381FC01E55DF74FAE1404
:101DB000BF04C006D10648F02081318142815381A1
:101DC0002A193B094C095D0908C0208131814281F3
:101DD00053812E193F09400B510BEDB7FEB73E97CB
:101DE0000FB6F894FEBF0FBEEDBF0DB71EB70F5F65
:101DF0001F4F71828282F80153824282648315826E
:101E00002683378340875187AA0FBB1FAA0FBB1FAA
:101E1000A559B84F8D919D910D90BC91A02D8287B1
:101E20009387A487B5870E94DD3693942DB73EB77C
:101E3000225F3F4F0FB6F8943EBF0FBE2DBF80917B
:101E40000D0A981608F497CF8DB79EB70E970FB668
:101E5000F8949EBF0FBE8DBFEDB7FEB7319687E2F7
:101E600097E0ADB7BEB712969C938E93119785EB12
:101E700093E09383828380911B09848315828091F0
:101E80001C098683178280911D0990911E099187F4
:101E9000808780911F0990912009A0912109B0911C
:101EA000220982879387A487B5870E94DD36EDB724
:101EB000FEB73E960FB6F894FEBF0FBEEDBF0F9073
:101EC000CF91DF911F910F91FF90EF90DF90CF9016
:101ED000BF90AF909F908F907F906F905F904F904A
:101EE00008950E9493090E94FB0D80E00895BF921F
:101EF000CF92DF92EF92FF920F931F936C01FC0140
:101F0000B080E1800E94AA2B20E831E541E050E05A
:101F10000E948A6A2B0D311D411D511DFF2400E0D6
:101F200010E0CA01B901A80197010E948A6AF6016E
:101F300060831F910F91FF90EF90DF90CF90BF9043
:101F400008958F929F92AF92BF92CF92DF92EF92BD
:101F5000FF920F931F934C01FC01A180E080FF24AE
:101F6000EA0CF11C0027F7FC0095102F0E94AA2B09
:101F7000BB24CC24DD2420E831E541E050E00E9480
:101F80008A6ACA01B901A60195010E948A6AE61A05
:101F9000F70A080B190BC801B701A60195010E94A9
:101FA0008A6AF40160831F910F91FF90EF90DF9098
:101FB000CF90BF90AF909F908F9008950E94AA2BD2
:101FC000AB01BC0180910D0AEBEEF8E0ABE2B8E0AA
:101FD000282F30E02E0F3F1F0AC08081882329F070
:101FE0004D935D936D937C93139731961496E217FE
:101FF000F30799F70895CF93DF939C011092AE06F3
:10200000FC01A081B181C0E0D0E00FC09C919D3265
:1020100031F09B3221F0892F80538A3068F4FE0121
:10202000E255F94F908321961196F90180819181B3
:102030000A96A817B90750F3C255D94F18821196BE
:10204000F901B183A0838EEA96E00E944D06CB0190
:10205000DF91CF9108956F927F928F929F92AF926E
:10206000BF92CF92DF92EF92FF920F931F93DF9375
:10207000CF9300D00F92CDB7DEB75C016A01DE01CD
:102080001196EEEDF2E083E001900D928150E1F7C0
:10209000698310E0A2E06A2E712C6C0E7D1E4E0149
:1020A0000894811C911C1CC0812F90E0B3014AE070
:1020B00050E00E941E07C5016EEA76E048E79401F1
:1020C00000E0EE24FF240E944035882341F08EEA90
:1020D00096E00E942F06F601E10FF11D80831F5F3D
:1020E00080910C0A181700F30F900F900F90CF916A
:1020F000DF911F910F91FF90EF90DF90CF90BF90F5
:10210000AF909F908F907F906F900895CF92DF92C5
:10211000EF92FF920F93DF93CF93CDB7DEB7C857FF
:10212000D0400FB6F894DEBF0FBECDBF6C016EEA93
:1021300076E048E72DE732E001E0EE24FF240E943C
:102140004035882311F480E128C0C6016E0108944F
:10215000C11CD11CB60148E729E732E001E0EE24BA
:10216000FF240E9440358823B9F08EEA96E0B6013C
:1021700040E150E00E94C906009771F48EEA96E0B3
:102180000E94C1351092CE0684EF93E06EEA76E0AD
:102190000E94BE3981E001C083E0C858DF4F0FB60E
:1021A000F894DEBF0FBECDBFCF91DF910F91FF90AE
:1021B000EF90DF90CF900895EF92FF920F936EEA29
:1021C00076E048E72FE832E001E0EE24FF240E94A9
:1021D00040358823C1F08EEA96E00E94C135109206
:1021E000EE06EEEAF6E0DF018081803209F08D93A1
:1021F0008081882311F03196F7CF84E494E06EEA71
:1022000076E00E94BE398FEF0F91FF90EF90089516
:10221000EF92FF920F931F93CF93DF93EC016EEA3F
:1022200076E048E72DE932E001E0EE24FF240E9449
:102230004035882311F00E94DE0FCE016EEA76E071
:1022400048E729E932E001E0EE24FF240E9440350E
:102250008823C9F08EEA96E00E942F061816190608
:1022600094F40E94FD0980912D0790912E072091F2
:102270002B0730912C07821B930B61E140E00E94F9
:10228000802F0E94DB38CE016EEA76E048E726E92F
:1022900032E001E0EE24FF240E944035882399F0CB
:1022A0008091AE06813339F48091060A80FD0BC01F
:1022B0000E94E03A08C0803331F48091060A80FF22
:1022C00002C00E94EB3ACE016EEA76E048E723E9CD
:1022D00032E001E0EE24FF240E944035882361F1C2
:1022E0008EEA96E00E942F06EC0118161906F4F407
:1022F0000E94AA2B7B018C01BE01882777FD809567
:10230000982F20E13EE040E050E00E94386AE60E5F
:10231000F71E081F191FE092020AF092030A0093A9
:10232000040A1093050A0E940D4006C0009711F0A0
:1023300081E103C00E94FD3F81E0DF91CF911F91B9
:102340000F91FF90EF9008952F923F924F925F92DE
:102350006F927F928F929F92AF92BF92CF92DF92B5
:10236000EF92FF920F931F93DF93CF93CDB7DEB71A
:102370002A970FB6F894DEBF0FBECDBF7B018C014C
:102380004B015C010894811C911CA11CB11C809123
:1023900046020E94263B6C012091230930912409BA
:1023A0004091250950912609E216F3060407150706
:1023B00018F08501740109C07C010027F7FC009525
:1023C000102FE20EF31E041F151F40900D0A80917E
:1023D000080A282E33246091060A6695669566954C
:1023E0006170552441E0642E712CC601AA2797FD27
:1023F000A095BA2F89839A83AB83BC837AC0E52DDD
:10240000F0E02614370409F470C0CF01880F991F3B
:10241000880F991F2BE2C22E28E0D22EC80ED91E9B
:10242000D6012D913D914D915C91211531054105CC
:10243000510509F45AC0DC01A559B84FBE83AD83DC
:102440008D919D910D90BC91A02D0097A105B10596
:1024500009F04BC0DF0183E0B695A7958A95E1F7B7
:10246000752D7770FD01E25FF54F808190E0072EBA
:1024700002C0959587950A94E2F780FD36C0AE5C60
:10248000B54F8C9190E002C0959587957A95E2F7CB
:1024900080FF1AC0ED81FE81E082F1820283138306
:1024A000DA01C9018E0D9F1DA01FB11FF6018083A7
:1024B0009183A283B383E980FA800B811C81E80EAB
:1024C000F91E0A1F1B1F10C0AD81BE818D929D9207
:1024D000AD92BC921397280D391D4A1D5B1DF60164
:1024E000208331834283538361E053940894611CB9
:1024F000711C541408F483CF6170660F660F660F69
:102500008091060A877F862B8093060A2A960FB64B
:10251000F894DEBF0FBECDBFCF91DF911F910F9119
:10252000FF90EF90DF90CF90BF90AF909F908F90F3
:102530007F906F905F904F903F902F900895AF9253
:10254000BF92CF92DF92EF92FF921F93CF93DF93D0
:10255000C0EED1E010E077E2E72E77E0F72E69EBEE
:10256000A62E62E0B62E57EBC52E52E0D52E8881FE
:10257000282F30E040E050E0143129F42C53304053
:102580004040504016C01E3159F4CA01B9012AE03A
:1025900030E040E050E00E94386A9B01AC0109C085
:1025A000113139F40E94263B9C01442737FD4095A8
:1025B000542F6C817D81FB0184918F35B9F18DB7EA
:1025C0009EB70A970FB6F8949EBF0FBE8DBFEDB7AA
:1025D000FEB73196ADB7BEB71296FC92EE92119748
:1025E000B382A282758364832683378340875187B1
:1025F0000E94DD36EDB7FEB73A960FB6F894FEBFEF
:102600000FBEEDBF153291F000D000D0ADB7BEB710
:102610001296FC92EE9211971496DC92CE9213973A
:102620000E94DD360F900F900F900F901F5F26963F
:10263000163209F09CCF0E94C93FEDB7FEB738971C
:102640000FB6F894FEBF0FBEEDBF319627E237E01C
:10265000ADB7BEB712963C932E93119721EA32E0A4
:10266000338322838483158285E090E09783868379
:102670000E94DD36EDB7FEB738960FB6F894FEBF70
:102680000FBEEDBFDF91CF911F91FF90EF90DF90D4
:10269000CF90BF90AF9008950E9493090E949F121F
:1026A00080E008958F929F92AF92BF92CF92DF9277
:1026B000EF92FF920F931F93DF93CF9300D000D040
:1026C000CDB7DEB76C0183E789831A821B821C8237
:1026D00010E0E2E08E2E912C8C0E9D1E5E0108947F
:1026E000A11CB11C1DC0812F90E0B4014AE050E054
:1026F0000E941E07C6016EEA76E048E7950100E0F9
:10270000EE24FF240E944035882349F08EEA96E0AB
:102710000E94C135812F6EEA76E00E949C391F5FCE
:1027200080910D0A1817F8F2C6016DE644E15AE0EF
:102730000E942B1084EA97E064E17AE00E94154041
:10274000C60169E64AE15AE00E942B108AEA97E046
:102750006AE17AE00E941540C60161E640E25AE073
:102760000E942B1080EB97E060E27AE00E94154017
:10277000C60164E646E25AE00E942B1086EB97E021
:1027800066E27AE00E9415400E94463AC60161E77F
:1027900042E35AE00E942B108CEB97E062E37AE070
:1027A0000E94154081E00F900F900F900F90CF91F5
:1027B000DF911F910F91FF90EF90DF90CF90BF902E
:1027C000AF909F908F900895AF92BF92CF92DF927B
:1027D000EF92FF920F931F93CF93DF9300D000D01F
:1027E00007E217E0ADB7BEB712961C930E93119790
:1027F00082E396E014969C938E9313970E94DD36A5
:10280000FF240F900F900F900F90E02E012FAEEA53
:10281000AA2EA6E0BA2EFDE2CF2EF6E0DF2ECBE206
:10282000D6E03EC08F2D6EEA76E00E947E3900D061
:1028300000D000D0EDB7FEB73196ADB7BEB7119658
:10284000EC92119712960C93D382C282B582A48225
:102850000E94DD362F2D30E080910D0A90E0019727
:10286000EDB7FEB736960FB6F894FEBF0FBEEDBFBC
:1028700028173907A1F000D000D0ADB7BEB7119628
:10288000EC92119712960C9312971496DC93CE93B8
:1028900013970E94DD360F900F900F900F90F394D6
:1028A00080910D0AF81608F4BDCF85E296E064E148
:1028B0007AE00E940C0989E196E06AE17AE00E94E0
:1028C0000C098FE096E060E27AE00E940C0987E054
:1028D00096E066E27AE00E940C0981E096E06CE204
:1028E0007AE00E940C0989EF95E062E37AE00E94A9
:1028F0000C0900D000D000D0EDB7FEB7319687E2CA
:1029000097E0ADB7BEB712969C938E9311978AEE5F
:1029100095E09383828380E190E0958384830E9495
:10292000DD36EDB7FEB736960FB6F894FEBF0FBE94
:10293000EDBFDF91CF911F910F91FF90EF90DF904E
:10294000CF90BF90AF9008950E9493090E94E41326
:1029500080E00895EF92FF920F939C0180917602A0
:102960008823B1F4C9016EEA76E048E72BE436E04B
:1029700001E0EE24FF240E944035882351F08EEAC6
:1029800096E00E94C1358EEA96E00E94E3398111FB
:1029900081E00F91FF90EF900895DF92EF92FF9208
:1029A0000F931F93CF93DF93EC010E940C30109292
:1029B0002A071092290782E993E090932C078093CD
:1029C0002B0790932E0780932D07BE016B5F7F4FDF
:1029D000FD8080E2F81621F0EC2EDD2EFE0104C011
:1029E000CB010E94A40D10C18581882359F080324B
:1029F00049F08A3039F08F3329F031968F32A1F7C0
:102A000052E1AEC050E0ACC0C52FD0E0FE01EE0FE9
:102A1000FF1FEE0FFF1FE157FE4F0190F081E02DE9
:102A2000849190E08017910709F0FDC03196849160
:102A300090E04C91242F332727FD30958217930780
:102A400009F0F1C093E7F91671F4453709F041C078
:102A5000CC0FDD1FCC0FDD1FCF56DE4FE881F98193
:102A6000CB01039647C0AAE6FA1699F54F3689F5C9
:102A70008B010D5F1F4FC8010E94AA14882389F59E
:102A80000E9493098DB79EB708970FB6F8949EBF22
:102A90000FBE8DBFEDB7FEB7319687E297E0ADB7B9
:102AA000BEB712969C938E93119786E292E0938321
:102AB00082838091E4019091E501958384838091E4
:102AC000E001868317820E94DD368DB79EB7089697
:102AD00096C08B010D5F1F4FC8010E94AA14882366
:102AE00039F1CC0FDD1FCC0FDD1FCF56DE4FE88153
:102AF000F981C8010995182F882309F485C08F3FF3
:102B0000C1F40E94FD0900D000D000D0EDB7FEB79F
:102B1000319687E297E0ADB7BEB712969C938E933D
:102B2000119783E292E09383828380EE91E060C00C
:102B300012E00E94CB0900D000D000D0EDB7FEB764
:102B4000319687E297E0ADB7BEB712969C938E930D
:102B5000119785E192E093838283148315824AC0A2
:102B60000F2D112707FD1095DB011196523109F049
:102B70004BCF8091060A85FF47C0CEEAD6E08E2D66
:102B80009D2D9C01D90101C08993EA2FEE1915965C
:102B90008C911597803229F0119696E0CE3CD9079A
:102BA00099F7F0E0E255F94F10828FE297E069E281
:102BB00071E040E00E945D4C8EEA96E00E94930C2A
:102BC000882399F50E94CB0900D000D000D0EDB742
:102BD000FEB7319687E297E0ADB7BEB712969C93E9
:102BE0008E93119787E092E09383828380E290E056
:102BF000958384830E94DD368DB79EB706960FB607
:102C0000F8949EBF0FBE8DBF80912D0790912E0727
:102C100020912B0730912C07821B930B61E140E040
:102C20000E94802F02C05F5FA1CFDF91CF911F91E3
:102C30000F91FF90EF90DF9008958F929F92AF9247
:102C4000BF92CF92DF92EF92FF920F931F93CF9399
:102C5000DF93EC017A018B01CB01BA010E94972A24
:102C60004C01C801B7010E94912A5C01888180FF54
:102C7000ACC0C801B7010E94852AC82EC801B7019F
:102C80000E948B2AD82E88818295837090E08230B2
:102C90009105B1F083309105F1F0892BB1F52981CF
:102CA00030E08C2D90E0059667E070E00E94776A36
:102CB00002C0359527958A95E2F720FD26C085C08C
:102CC0002D2D30E0898190E08F71907028173907A1
:102CD00009F07BC01AC0C801B70120E831E541E026
:102CE00050E00E948A6ACA01B9012A8130E040E0BE
:102CF00050E00E948A6A298130E040E050E062178B
:102D000073078407950709F060C0888186958695CA
:102D10008370B9F0823019F4D0FE13C056C08130F0
:102D200081F48FE1D81609F450C08DE1D81609F06E
:102D30005BC0C801B7010E947F2A029709F054C006
:102D400044C08CE390E0889E9001899E300D989E4F
:102D5000300D11242A0D3B1D888186FD29C00D816F
:102D60001E81EF81F8858B819C812817390768F1D6
:102D70000115110529F460E02817390739F51FC03E
:102D8000309719F1281B390BC901BF010E94636AF2
:102D9000AB016E9FC0016F9F900D7E9F900D11241F
:102DA0008217930791F460E0041715077CF007C0C1
:102DB000FE0140E0838194812817390711F461E016
:102DC00005C04F5F32964430A9F760E0862FDF914F
:102DD000CF911F910F91FF90EF90DF90CF90BF9018
:102DE000AF909F908F900895D0FCABCFEECF982FEF
:102DF0009B0180916A07981768F467E4969FB00179
:102E00001124665F7F4FC90147E450E021E937E0B4
:102E10000E94E60608952F923F924F925F926F9222
:102E20007F928F929F92AF92BF92CF92DF92EF925A
:102E3000FF920F931F93DF93CF93CDB7DEB7C754A5
:102E4000D0400FB6F894DEBF0FBECDBF2DB73EB752
:102E50002E5030400FB6F8943EBF0FBE2DBFEDB7D9
:102E6000FEB7319607E217E0ADB7BEB712961C93D6
:102E70000E9311978BE994E09383828380916A0784
:102E80008483158280910C0A868317828EE090E0FD
:102E90009187808784E090E0938782878CE090E040
:102EA000958784870E94DD36EE24EDB7FEB73E9607
:102EB0000FB6F894FEBF0FBEEDBFF02E012F5BE8FA
:102EC000C52E54E0D52E4CE0642E712C6C0E7D1E68
:102ED0008F2C912E31E7232E34E0332E24E7422E1F
:102EE00024E0522E92E9A92E93E0B92E57C18E2DDF
:102EF000BE016F5F7F4F0E94F716898182958370B4
:102F0000833039F48B81823020F0CE0102960E940A
:102F1000A10F2DB73EB72A5030400FB6F8943EBFF0
:102F20000FBE2DBFEDB7FEB73196ADB7BEB7119648
:102F3000FC92119712960C932FE834E0338322838E
:102F40008981848315828A81868317828B81808719
:102F500011860E94DD360F900F900F900F90EDB705
:102F6000FEB73196ADB7BEB71196FC921197129687
:102F70000C93D382C2828C819D81958384830E942D
:102F8000DD36EDB7FEB73196ADB7BEB71196FC9200
:102F9000119712960C93D382C2828E819F81958362
:102FA00084830E94DD36EDB7FEB73196ADB7BEB76C
:102FB0001196FC92119712960C93D382C282888547
:102FC0009985958384830E94DD36EDB7FEB73196EF
:102FD000ADB7BEB71196FC92119712960C9325E8E7
:102FE00034E0338322838A859B85958384830E9482
:102FF000DD3610E04DB75EB74A5F5F4F26C0E60D85
:10300000F71D80810E94463BADB7BEB718970FB63B
:10301000F894BEBF0FBEADBFEDB7FEB731961196A7
:10302000FC92119712960C9321E834E033832283AB
:10303000A0E0B0E084839583A683B7830E94DD3649
:103040001F5F4DB75EB7485F5F4F0FB6F8945EBF26
:103050000FBE4DBFE12FF0E080910D0A90E0019787
:10306000E817F90764F2E60DF71D80810E94463BE0
:10307000ADB7BEB718970FB6F894BEBF0FBEADBFC1
:10308000EDB7FEB7319611968C92119712969C92DD
:103090002BE734E033832283A0E0B0E08483958380
:1030A000A683B7830E94DD364DB75EB7485F5F4F9A
:1030B0000FB6F8945EBF0FBE4DBF8EEA96E0BE011C
:1030C000645C7F4F4CE050E00E94D7061092BA0635
:1030D00000D000D000D0EDB7FEB73196ADB7BEB787
:1030E00011968C92119712969C9228E734E03383C4
:1030F00022834EEA56E0558344830E94DD362E2D0E
:1031000030E080916A0790E00197ADB7BEB71696A0
:103110000FB6F894BEBF0FBEADBF2817390749F0F0
:1031200000D000D0EDB7FEB7F18202835482438213
:103130000EC000D000D0ADB7BEB71196FC9211976B
:1031400012960C93129714963C922E9213970E940B
:10315000DD360F900F900F900F908E2D63E00E9440
:10316000576A9230D1F480912D0790912E072091CB
:103170002B0730912C07821B930B60E143E00E94E8
:10318000802F10922A0710922907B0922C07A09244
:103190002B07B0922E07A0922D07E39480916A0727
:1031A000E81608F4A4CE00D000D087E297E0EDB78F
:1031B000FEB7928381838EE694E0948383830E949A
:1031C000DD360F900F900F900F90C95BDF4F0FB659
:1031D000F894DEBF0FBECDBFCF91DF911F910F914D
:1031E000FF90EF90DF90CF90BF90AF909F908F9027
:1031F0007F906F905F904F903F902F9008950E9426
:1032000093090E940B1780E00895DF92EF92FF92DE
:103210000F931F93DF93CF93CDB7DEB7C754D04042
:103220000FB6F894DEBF0FBECDBF20916A0782179C
:1032300008F046C0222309F443C090E0019627E439
:1032400030E0829F8001839F100D929F100D11240A
:10325000065F1F4F67E4D62E7E010894E11CF11C27
:1032600014C0C701B80147E450E021E937E00E94EB
:10327000E606C80187549040B70147E450E029E9C9
:1032800037E00E940207095B1F4F20916A072D9DBE
:10329000C00111240A960817190718F3215020932A
:1032A0006A07F999FECF1FBA89E090E092BD81BD0F
:1032B00020BD0FB6F894FA9AF99A0FBE81E001C0CA
:1032C00080E0C95BDF4F0FB6F894DEBF0FBECDBF05
:1032D000CF91DF911F910F91FF90EF90DF900895B4
:1032E000EF92FF920F936EEA76E048E72AE634E029
:1032F00001E0EE24FF240E944035882311F480E190
:1033000025C08EEA96E00E942F069C018FEF2F3F8A
:10331000380781F410926A07F999FECF1FBA89E045
:1033200090E092BD81BD10BC0FB6F894FA9AF99A5C
:103330000FBE0BC080916A0790E02817390714F080
:1033400081E104C0822F0E94051981E00F91FF9056
:10335000EF900895982F80916A07981710F080E0F9
:10336000089587E4989FC00111240A9647E450E02D
:1033700029E937E00E94020781E00895BC0190919D
:103380006A079E3010F080E0089587E4989FC0019E
:1033900011240A9647E450E029E937E00E94020729
:1033A00020916A072F5F20936A07F999FECF1FBA11
:1033B00089E090E092BD81BD20BD0FB6F894FA9AE5
:1033C000F99A0FBE81E00895AF92BF92CF92DF923B
:1033D000EF92FF920F931F93DF93CF93CDB7DEB79A
:1033E000C954D0400FB6F894DEBF0FBECDBF6C01FC
:1033F0000E94C135C6016EEA76E048E722E634E075
:1034000001E0EE24FF240E944035882309F4D8C04F
:103410008EEA96E00E942F065C012FEF8F3F920705
:103420000CF4D0C080916A0790E0A816B9060CF0A1
:10343000C9C0DA82C98286010C591F4F0EC0C7016C
:103440006BE271E043E050E00E94C906009781F012
:103450000894E11CF11CFA82E982E980FA80F70104
:103460008081882309F4ACC0E016F10640F3A8C0BF
:1034700083E090E0E80EF91EFA82E9828E010F5F88
:103480001F4FC8010E94FB0F8B83C8010E94FB0FD6
:103490008C83C8010E94FB0F8D8389819A810196DC
:1034A0009A838983C8010E94FB0F9F838E83C80182
:1034B0000E94FB0F99878887C8010E94FB0F9B879A
:1034C0008A87C8010E94FB0F9D878C8789819A811A
:1034D00002969A838983DD2478018E01025F1F4F53
:1034E0000AC0C7010E94FB0F0E94F53AF801ED0DDA
:1034F000F11D8083D39480910D0AD81690F38981B1
:103500009A8102969A8389836EEA76E048E72DE5F0
:1035100034E001E0EE24FF240E9440358E01025C7D
:103520001F4F882361F08EEA96E00E94C135C801E2
:103530006EEA76E04CE050E00E94D7061EC0C8015B
:1035400060E770E00E9488069FEFA9169FEFB9061A
:1035500021F480916A0790E001C0C5010196BE0187
:103560006A5B7F4F4AE050E00E941E0706C0FC01E4
:10357000ED0DF11D1082D39402C0CE010E96EFE244
:10358000ED15A8F78B8182958370833039F48D8196
:10359000823020F0CE0104960E94770FBE016D5F4D
:1035A0007F4FFFEFAF16FFEFBF0621F4CB010E9464
:1035B000BE1903C08A2D0E94AA19882329F402C0CB
:1035C00080E103C081E101C081E0C75BDF4F0FB63E
:1035D000F894DEBF0FBECDBFCF91DF911F910F9149
:1035E000FF90EF90DF90CF90BF90AF900895EF9253
:1035F000FF920F931F938C018FE297E069E271E0D5
:1036000040E00E945D4C7CE1E72E77E0F72EC70199
:10361000B8010E94C2060EEA16E0C80160E871E037
:103620000E94C206C801B7010E94AC06C80166E04C
:1036300077E00E947D061F910F91FF90EF90089513
:103640002F923F924F925F926F927F928F929F92B2
:10365000AF92BF92CF92DF92EF92FF920F931F93A0
:10366000DF93CF93CDB7DEB7A2970FB6F894DEBF46
:103670000FBECDBF4C018091060A85FD02C080E2DD
:103680005EC1C4016EEA76E048E72DE432E001E075
:10369000EE24FF240E9440358823B9F08EEA96E09C
:1036A0000E942F067C0121E08E36920708F044C16B
:1036B0000E94AA2B20E831E541E050E00E948A6A8E
:1036C00059016901CE18DF083EC0C4016EEA76E0F8
:1036D00048E727E432E001E0EE24FF240E94403571
:1036E000882309F42BC18EEA96E00E944D065B0107
:1036F0006C01C4016EEA76E048E723E432E00E9400
:103700004035882309F41AC1C601B50120E831E526
:1037100041E050E00E94AC6A69018EEA96E00E94A6
:103720004D0620E831E541E050E00E94AC6A5901C5
:103730002C153D0508F400C1C9018C199D098E5650
:10374000914008F0F9C019821A821B821C82C401C0
:10375000BE016F5F7F4F44E02EE332E001E0EE24D4
:10376000FF240E944035482E0E94CB0900D000D093
:1037700007E217E0EDB7FEB7128301838CE392E016
:10378000948383830E94DD36992493940F900F9045
:103790000F900F90FEEA2F2EF6E03F2EE9E06E2EFE
:1037A000712C6C0E7D1E502E812E02E913E0ACC0F0
:1037B000C6016EEA76E04AE050E00E941E078EEAFB
:1037C00096E00E94F71A8FE297E06EEA76E00E9498
:1037D0003E4C882309F495C019861B8618861F82E3
:1037E00088E393E09E838D83C3016EEA76E041E037
:1037F0000E94965C01C09924C3016EEA76E047E717
:1038000050E020E030E00E94B3571816190624F06B
:10381000C3010E949A5475C0FC01E355F94F8081A1
:103820008A3009F41082442059F0CE01019662EBEF
:1038300076E042E050E00E94C9060097E9F60AC02F
:103840008FE291E062EB76E042E050E00E94C90630
:10385000009791F2992081F000D000D000D0EDB710
:10386000FEB73196ADB7BEB711965C92119712961E
:103870008C9289E392E00FC000D000D000D0EDB769
:10388000FEB73196ADB7BEB711965C9211971296FE
:103890008C9285E392E093838283358224820E9416
:1038A000DD36ADB7BEB716960FB6F894BEBF0FBEE5
:1038B000ADBF0894E11CF11CC70169E170E00E94F2
:1038C000776A892B09F097CF80912D0790912E0769
:1038D00020912B0730912C07821B930B60E143E072
:1038E0000E94802F10922A071092290710932C070C
:1038F00000932B0710932E0700932D07EE24FF242F
:103900007ACF0894C11CD11CAC14BD0408F050CF70
:1039100000D000D087E297E0EDB7FEB792838183B5
:1039200083E392E0948383830E94DD3680E00F90EE
:103930000F900F900F9003C081E101C080E1A2962B
:103940000FB6F894DEBF0FBECDBFCF91DF911F91B0
:103950000F91FF90EF90DF90CF90BF90AF909F902E
:103960008F907F906F905F904F903F902F90089531
:103970009F92AF92BF92CF92DF92EF92FF920F93FE
:103980001F93DF93CF93CDB7DEB76E970FB6F89442
:10399000DEBF0FBECDBF982E5A016B018091B802D9
:1039A000882309F412C18091060A85FF0EC1CB015C
:1039B000BA0120E831E541E050E00E948A6ACA017C
:1039C000B9014EEA56E02AE030E00E945C078EEA38
:1039D00096E00E94F71A8FE297E069E271E040E01A
:1039E0000E945D4C8FE297E060E871E040E00E9449
:1039F0005D4C882351F48FE297E060E871E041E08C
:103A00000E941F4C882309F4E0C01D821F821C8283
:103A10001B8288E393E09A8389838E010B5F1F4F9B
:103A2000BEEAEB2EB6E0FB2EC801B70142E40E94CD
:103A3000965C4F89588D698D7A8DC8010E943252EB
:103A4000C70164E077E00E9488069920D1F5F7016C
:103A500001900020E9F73197EE19FF09EE0DFF1DE7
:103A600080911C0990E0BF014AE050E00E941E07CF
:103A7000C70162E077E00E947D06F7010190002017
:103A8000E9F73197EE19FF09EE0DFF1D80911B0933
:103A900090E0BF014AE050E00E941E07C70160E0CD
:103AA00077E00E947D06F70101900020E9F7319749
:103AB000EE19FF09EE0DFF1D80911D0990911E0961
:103AC0005AC0C7016CEF76E00E947D06E92DF0E058
:103AD000EE0FFF1FE957FE4F60817181C7010E9401
:103AE000AC06C70169EF76E00E947D0622E09216DF
:103AF000B9F033E0931699F141E0941609F040C013
:103B0000F70101900020E9F73197EE5AF6408091D5
:103B1000380A9091390AA0913A0AB0913B0A0FC035
:103B2000F70101900020E9F73197EE5AF6408091B5
:103B30003C0A90913D0AA0913E0AB0913F0AA6012D
:103B40009501281B390B4A0B5B0BCA01B901E255E1
:103B5000F94FAF012AE030E00E945C0711C0F70185
:103B600001900020E9F73197EE5AF640E255F94FFF
:103B70008091540A90E0BF014AE050E00E941E0785
:103B80000EEA16E0C80167EF76E00E947D06F801B4
:103B900001900020E9F73197E01BF10BE00FF11FD6
:103BA000C601B501AF012AE030E00E945C07C80100
:103BB00063EF76E00E947D06CE010196B8010E9477
:103BC000A761CE0105960E949A546E960FB6F8949E
:103BD000DEBF0FBECDBFCF91DF911F910F91FF9040
:103BE000EF90DF90CF90BF90AF909F900895CF92CD
:103BF000DF92EF92FF921F936B017C018091270966
:103C000090912809A0912909B0912A09A70196014C
:103C1000281B390B4A0B5B0BDA01C901855893400D
:103C2000A040B04078F1C0922709D0922809E092D4
:103C30002909F0922A092091540A30E040E050E02E
:103C400010912B09612F70E080E090E00E94386AAB
:103C500020916A02620F711D811D911D1F5F1093DB
:103C60002B09212F30E040E050E00E948A6A209327
:103C7000540A103639F483E0B701A6010E94B81C3B
:103C800010922B091F91FF90EF90DF90CF90089535
:103C9000CF93DF93EC018091B802882361F180918A
:103CA000060A85FF28C0CE0162E371E043E050E0E0
:103CB0000E94C906009771F48FE297E060E871E016
:103CC00040E00E945D4C8823B1F08DE497E00E94B3
:103CD000145711C0CE010E94F71A8FE297E06EEAE6
:103CE00076E00E943E4C882331F08FE297E06EEA46
:103CF00076E00E941B4CDF91CF910895EF92FF92E6
:103D00000F936EEA76E048E72FE232E001E0EE241E
:103D1000FF240E944035882311F480E105C08EEA1B
:103D200096E00E94481E81E00F91FF90EF90089569
:103D30000E94393A0E944442ABEEB8E080E090E045
:103D4000FC01E559F84F1082118212821382FC01A6
:103D5000E55DF74F10821182128213821D92049644
:103D6000803C910569F71092230910922409109262
:103D700025091092260908952F923F924F925F9243
:103D80006F927F928F929F92AF92BF92CF92DF926B
:103D9000EF92FF920F931F93DF93CF93CDB7DEB7D0
:103DA00027970FB6F894DEBF0FBECDBF4C0100EED3
:103DB000C02E01E0D02E6624772455241F82AA2429
:103DC000BB2412E0212E312C2C0E3D1E1A2D153253
:103DD00009F489C0183109F486C0AA2009F483C007
:103DE0001E3009F480C0103109F47DC02A2D9B2DAE
:103DF000F60140808181813009F41082D101E9ED22
:103E0000F2E085E001900D928150E1F7822FBE0132
:103E10006D5F7F4F4AE050E00E941E07C4016EEACA
:103E200076E048E7910100E0EE24FF240E9440354F
:103E30008823D1F1F6018181813011F4808334C06F
:103E40008EEA96E00E944D069B01AC01143129F4E4
:103E5000245C3F4F4F4F5F4F17C01E3159F42AE08B
:103E600030E040E050E00E94AC6AC901DA019C01F8
:103E7000AD010AC0113141F4CB010E94113B282F42
:103E800030E040E050E002C057FD0CC0F6018181F7
:103E900090E0A0E0B0E082179307A407B50714F004
:103EA000208302C0F1E0FF83F60180818415D9F000
:103EB000812F8150823010F466246394812F8052C8
:103EC000843010F466246394812F83508B3010F477
:103ED000552453941A3119F45524539404C01F31B6
:103EE00011F4772473940894A11CB11C86E090E02F
:103EF000C80ED91E96E2A916B10409F067CFC40115
:103F00006EEA76E048E72BE832E001E0EE24FF2499
:103F10000E9440358823B1F08EEA96E00E94C135B8
:103F20001092DE068EEA96E064E174E00E94FD39AC
:103F3000882341F084E194E06EEA76E00E94BE3985
:103F4000772473941982C4016EEA76E048E725E885
:103F500032E001E07E010894E11CF11C0E94403532
:103F60008823B9F08EEA96E00E94C1351092CE0601
:103F70008EEA96E064E874E00E94FD398823A1F09F
:103F800084E894E06EEA76E00E94BE397724739468
:103F90000BC08981882341F01092AE0684E894E03A
:103FA0006EEA76E00E94BE398091EC01882339F5F3
:103FB000C4016EEA76E048E721E832E001E0EE2451
:103FC000FF240E9440358823D1F08EEA96E00E94BB
:103FD0004D06162F072FF82EE92E0E94981E612FEE
:103FE000702F8F2D9E2D0E947D2B8091060A84FFBD
:103FF00006C0612F702F8F2D9E2D0E947D2DEF8189
:10400000EE2311F081E121C00E94B33A662041F015
:104010001092440A1092450A1092460A1092470ADA
:10402000772041F01092480A1092490A10924A0AE9
:1040300010924B0A552041F010924C0A10924D0AF2
:1040400010924E0A10924F0A81E027960FB6F8940C
:10405000DEBF0FBECDBFCF91DF911F910F91FF90BB
:10406000EF90DF90CF90BF90AF909F908F907F9018
:104070006F905F904F903F902F900895DF92EF9256
:10408000FF920F931F93DF93CF9300D0CDB7DEB78E
:104090008C010E94C1351A83098324E6E22EF12C9B
:1040A000E00EF11E0DC0C80166E371E043E050E090
:1040B0000E94C906009779F00F5F1F4F1A8309838A
:1040C00009811A81F8018081882309F44DC00E15F9
:1040D0001F0548F349C00D5F1F4F1A8309830E94D3
:1040E000981E10E000E07E010894E11CF11C9EEF98
:1040F000D92E2EC0C7010E94FB0FBC01009739F1D9
:10410000412F50E0E12FE695E695E695F0E0EA5D77
:10411000F54F808190E0212F277002C095958795FB
:104120002A95E2F780FD13C0FA01EE0FFF1FEE0F94
:10413000FF1FE55DF74FCB01A0E0B0E080839183E6
:10414000A283B3834551574FFA01D08201E01F5F2C
:1041500080910D0A181770F2002331F00E94AA2BEB
:104160000E94A41181E001C080E10F900F90CF91D7
:10417000DF911F910F91FF90EF90DF900895AF9224
:10418000BF92CF92DF92EF92FF920F931F93DF9334
:10419000CF93CDB7DEB7C754D0400FB6F894DEBF8B
:1041A0000FBECDBFE82E0E94981E8E2D81508E3FEF
:1041B00028F4BE016F5F7F4F0E94F716DD24FF24B5
:1041C000EEEFCE2E7CE0A72EB12CAC0EBD1E3BC078
:1041D0000F2D10E08FEFE81619F442E050E00BC00D
:1041E000EE20E9F1F501E00FF11F80810E94463BCE
:1041F000AC01009739F1F80163E0F695E7956A950F
:10420000E1F7EA5DF54F808190E02F2D277002C025
:10421000959587952A95E2F780FD14C0F801EE0F79
:10422000FF1FEE0FFF1FE55DF74FCA01A0E0B0E0F2
:1042300080839183A283B3830551174FF801C08215
:10424000DD24D394F39480910D0AF81608F4C0CFBE
:10425000DD2041F00E94AA2B0E94A41103C04CE370
:1042600050E0C9CFC95BDF4F0FB6F894DEBF0FBE79
:10427000CDBFCF91DF911F910F91FF90EF90DF9015
:10428000CF90BF90AF900895CF92DF92EF92FF92C0
:104290000F931F93CF93DF93D82EC62E79018A01F7
:1042A000C82FD0E060E00E94153AFE01EE0FFF1F1C
:1042B000EE0FFF1FE559F84F4081518162817381F4
:1042C000411551056105710509F47DC04E155F0565
:1042D0006007710708F061C02C2D30E0CE01019617
:1042E00028173907E1F0D0921B09FE01E551F74F7D
:1042F000808180931C09C701841B950B90931E0934
:1043000080931D09E0921F09F09220090093210972
:104310001093220980E0B801A7010E94B81C8E0109
:1043200083E0169507958A95E1F7B7E0FB2EFD200F
:10433000F801E05EF54F808190E00F2C02C095956A
:1043400087950A94E2F780FF18C080919402882331
:1043500081F08EE061E00E94EA65609194022AE0BB
:10436000629FB0011124882777FD8095982F0E94C5
:10437000F3668EE060E00E94EA65045D154FF80187
:10438000808190E002C095958795FA94E2F780FFCE
:1043900004C08D2D60E00E940D42FE01EE0FFF1F54
:1043A000EE0FFF1FDF01A559B84F1D921D921D9200
:1043B0001C921397E55DF74F1082118212821382CF
:1043C000C551D74F1882DF91CF911F910F91FF9068
:1043D000EF90DF90CF9008958F929F92AF92BF920F
:1043E000CF92DF92EF92FF920F931F93CF93DF93C1
:1043F0006C016EEA76E048E727E532E001E0EE2462
:10440000FF240E944035882309F48AC08EEA96E092
:104410000E942F06EC0197FD81C080910D0A90E06B
:10442000C817D9070CF07AC0C6016EEA76E048E7F3
:1044300024E532E00E944035882309F471C08EEAF9
:1044400096E00E942F06182F0E94AA2B4B015C01B8
:10445000112309F45AC0C6016EEA76E048E722E566
:1044600032E00E944035882309F45AC08EEA96E073
:104470000E944D06CB01019780529D4F08F04EC01F
:104480008091080A90E09E012F5F3F4F82179307AB
:1044900009F448C0FE0143E0F595E7954A95E1F738
:1044A000F0E0E25FF54F808190E0AE014770042EAE
:1044B00002C0959587950A94E2F780FD33C0FE010E
:1044C000EE0FFF1FEE0FFF1FE55DF74F808191811B
:1044D000A281B3810097A105B10521F5FE01EE0F80
:1044E000FF1FEE0FFF1FE55DF74FCB01A0E0B0E02F
:1044F00080839183A283B383C551D74F83E688839A
:10450000C501B4010E94A41107C08C2F6091080A54
:10451000A50194010E94442181E005C081E103C00E
:1045200080E101C080E3DF91CF911F910F91FF9057
:10453000EF90DF90CF90BF90AF909F908F900895B5
:104540004F925F926F927F928F929F92AF92BF92A3
:10455000CF92DF92EF92FF920F931F93CF93DF934F
:104560005B016C019091060A44244394492291FD19
:104570000CC080915E02882311F4FF2408C0F92E3C
:10458000F694F69481E0F82211F0FF24F394EE24DF
:104590005BC08E2D90E0FC01E65EF54F3081FC01A2
:1045A000E25FF54F20815E2C550C550C550C00E058
:1045B00010E0622E7724832E9924252D200FC22F00
:1045C000D0E0FE01E551F74FE081E336B0F544203D
:1045D00059F0FF2091F1C401002E02C095958795F6
:1045E0000A94E2F780FD29C0C301002E02C0959510
:1045F00087950A94E2F780FF08C0822F6091080A2D
:10460000A60195010E94442118C0EE23B1F0FE01DD
:10461000EE0FFF1FEE0FFF1FDF01A559B84F1D92D0
:104620001D921D921C921397E55DF74F1082118227
:1046300012821382C551D74F18820F5F1F4F083067
:10464000110509F0BACFE39480910C0AE81608F43A
:10465000A0CFDF91CF911F910F91FF90EF90DF904E
:10466000CF90BF90AF909F908F907F906F905F9012
:104670004F900895AF92BF92CF92DF92EF92FF9248
:104680000F931F935B016C018091060A83FDB6C0F6
:1046900080914C0A90914D0AA0914E0AB0914F0A18
:1046A0000097A105B10511F40E946B442091070AFF
:1046B00022952F7061E070E002C0660F771F2A9587
:1046C000E2F7882777FD8095982F20914C0A30914A
:1046D0004D0A40914E0A50914F0A86017501E21A27
:1046E000F30A040B150B2EE130E040E050E00E948D
:1046F000386A6E157F058007910708F07FC08091AA
:104700002C09882359F489EE99E06FE041E00E947A
:10471000B54889EE99E064E00E947148A0924C0A85
:10472000B0924D0AC0924E0AD0924F0A84ED99E0A1
:104730000E945F310E94E5667B018C010E948F4AD6
:104740000E94AC3184ED99E00E942134882361F409
:104750000E94E5666E197F09800B910B683C71051C
:104760008105910558F336C08091070A8F7002C009
:104770008F7080668093070A8091070A82958F70F8
:1047800090E00397ACF48091500A9091510AA09167
:10479000520AB091530AA6019501281B390B4A0B06
:1047A0005B0BDA01C901815C984AA040B04030F14E
:1047B000A092500AB092510AC092520AD092530A63
:1047C0000E946B448823D1F08091070A8F708093F8
:1047D000070A14C08091070A282F22952F702F5F97
:1047E0002F70922F9295907F8F70892B8093070A5C
:1047F00030E0273031050CF0BBCFBECF1F910F91B9
:10480000FF90EF90DF90CF90BF90AF900895EF9220
:10481000FF920F931F939B01AC018091EC018823C1
:1048200009F447C08091070A82958F7009F041C052
:104830008091060A83FD3DC08091440A9091450A0B
:10484000A091460AB091470A0097A105B10569F009
:1048500079018A01E81AF90A0A0B1B0BD801C70172
:1048600081589145A140B04020F12093440A3093F3
:10487000450A4093460A5093470A80912C098823A1
:1048800029F48BE097E061E00E941F3D0E94020C3A
:104890007B018C01611571058105910551F00E9424
:1048A0007D2B8091060A84FF04C0C801B7010E94D5
:1048B0007D2D1F910F91FF90EF90089584B7877F12
:1048C00084BF0E94ED420E943A400E94DF076CE3E1
:1048D00070E080E090E00E94742B8091060A84FDD5
:1048E00003C080E090E002C08DE99DE20E941D2C93
:1048F00064EF71E080E090E00E94F36680E00E9447
:10490000A3428091600088618093600081E280937F
:104910006000809160008064809360008AE197E08D
:1049200061E00E941F3D8FE297E060E044E00E945A
:10493000AC4C882329F08091060A80628093060A95
:104940000E946B44882321F08091070A8F7004C075
:104950008091070A8F7080618093070A64EF71E08D
:1049600080E090E00E94F3660E9444420E94AA2BDD
:104970006093400A7093410A8093420A9093430ADD
:104980000895BF92CF92DF92EF92FF920F931F9301
:10499000DF93CF93CDB7DEB7C754D0400FB6F894AE
:1049A000DEBF0FBECDBF6B017C018091400A9091AC
:1049B000410AA091420AB091430A0097A105B105AE
:1049C000D9F00F96A11DB11D8C159D05AE05BF0533
:1049D00098F480918E026FEF70E0681B71098CE093
:1049E0000E944B651092400A1092410A1092420AAE
:1049F0001092430A10922C0982E00E94B53BB82E17
:104A0000082F10E086FFD7C0C092400AD092410A1A
:104A1000E092420AF092430A809188026FEF70E0C0
:104A2000681B71098CE00E944B6580912C098330D2
:104A300020F4813008F07BC004C0833009F0BBC093
:104A40006AC0C8018F70907082309105A1F18430E6
:104A5000910509F441C0019709F0ADC0B7FE0CC043
:104A60008EE10E943E66892B21F48FEF0E94BF20C9
:104A7000A2C00E94DE0F9FC089EE99E00E94E44828
:104A800088EC99E060E00E94F13C89EE99E060E0FA
:104A900041E00E94B54881E797E00E946E3C60913A
:104AA000DE017091DF0189EE99E04AE050E00E945A
:104AB000C26981E00EC0B7FE03C00E94DB387BC034
:104AC00089EE99E00E94E44882EC99E00E947E3CE5
:104AD00082E080932C096FC0B7FE0CC082E697E09D
:104AE00060E00E941F3D81E597E061E00E941F3D6C
:104AF00083E0EFCF2091070A822F8F7090E06091C2
:104B00000C0A019670E00E94776A8F70207F282B34
:104B10002093070A50C00F7010700430110509F07F
:104B20004AC0B7FE07C0809137090E94BF2010928B
:104B30002C0941C08091370990E060916A0770E0CC
:104B40006F5F7F4F01960E94776A8093370980E4F8
:104B500097E060E00E941F3D80913709882331F182
:104B60008150BE016F5F7F4F0E94F7168EE397E082
:104B700061E00E941F3D89EE99E060E041E00E9403
:104B8000B5486091370989EE99E070E04AE050E05D
:104B90000E94136A8BE397E00E946E3C89EE99E0D5
:104BA000BE01645C7F4F0E94266A05C08BE297E0DD
:104BB00061E00E941F3DC95BDF4F0FB6F894DEBF76
:104BC0000FBECDBFCF91DF911F910F91FF90EF905E
:104BD000DF90CF90BF9008952F923F924F925F92B7
:104BE0006F927F928F929F92AF92BF92CF92DF92FD
:104BF000EF92FF920F931F93DF93CF93CDB7DEB762
:104C0000C954D0400FB6F894DEBF0FBECDBF80911F
:104C10004C028093080A0E948F4A0E94AC31909304
:104C20002E0980932D09009721F0845A9C4F0E94F1
:104C3000CD14A895109269070E94AA2B5B016C0104
:104C40000E94C1248091330990913409A0913509C3
:104C5000B09136098A159B05AC05BD0509F40DC355
:104C6000A0923309B0923409C0923509D092360926
:104C700080912C09882311F40E94A3428091060A96
:104C800081FF10C08091020A9091030AA091040A4A
:104C9000B091050AA816B906CA06DB0690F00E9474
:104CA000FD3F0FC08091020A9091030AA091040A6F
:104CB000B091050AA816B906CA06DB0610F40E94D0
:104CC0000D400E94FE3B9091060A9695917080914E
:104CD000090A869581708917C9F0992349F0A09235
:104CE0003C0AB0923D0AC0923E0AD0923F0A05C0EB
:104CF00082E0B601A5010E94B81C9091060A92704C
:104D00008091090A8D7F892B8093090A9091060A68
:104D10009695969591708091090A869586958170F1
:104D20008917C9F0992349F0A092380AB092390A3C
:104D3000C0923A0AD0923B0A05C081E0B601A501B3
:104D40000E94B81C9091060A94708091090A8B7F8A
:104D5000892B8093090AC601B5012CE330E040E0BD
:104D600050E00E948A6A79018A0180912F0990910E
:104D70003009A0913109B0913209E816F9060A0705
:104D80001B0709F4AAC0E0922F09F09230090093A2
:104D9000310910933209662455241E010894211C00
:104DA000311C90C0862DB1010E94F716C101B601D9
:104DB000A5010E941D16882309F483C07724462C80
:104DC00043947AC0872C99248091080A90E094013A
:104DD0002F5F3F4F8217930709F46DC0D40113E092
:104DE000B695A7951A95E1F7272D2770FD01E25F8B
:104DF000F54F808190E0022E02C0959587950A9428
:104E0000E2F780FD58C0AA5DB54F8C9190E002C0DA
:104E1000959587952A95E2F780FD4DC0ECE0F0E08E
:104E2000EC0FFD1FE80DF91D2081222309F443C07A
:104E3000F401EE0FFF1FEE0FFF1FE55DF74F8081BE
:104E40009181A281B3810097A105B105A1F5822FBF
:104E50000E94463B7C0100E010E0898181FF13C085
:104E600020916A0230E040E050E0C801B7010E94A2
:104E7000386A24E630E040E050E00E948A6AC901C6
:104E8000DA017C018D01F401EE0FFF1FEE0FFF1F11
:104E9000E55DF74FE082F18202831383E114F104B0
:104EA0000105110541F02BEE38E0820E931EF4014E
:104EB000408255245394739480910D0A781608F417
:104EC00081CF639480916A07681608F46BCF5520F0
:104ED00021F0C601B5010E94A4118091060A83FF4A
:104EE0002CC17724AEC0872D90E0FC01E25FF54F26
:104EF0002081672C660C660C660CEE24FF24422F82
:104F000050E02A965FAF4EAF2A9770E2472E7AE0C4
:104F1000572E480E591E6CE2262E6AE0362E280EB9
:104F2000391E862C8E0C6091080A082D10E0262F61
:104F300030E0C80101962817390709F479C0F80153
:104F4000E551F74F80818823A9F0F801EE0FFF1F8C
:104F5000EE0FFF1FE55DF74F80819181A281B38144
:104F6000A816B906CA06DB0628F0882DA601950109
:104F70000E9444219E2C2A968EAD9FAD2A970E2C1E
:104F800002C0959587950A94E2F780FD51C098017B
:104F9000220F331F220F331FF901E559F84F80818B
:104FA0009181A281B381A816B906CA06DB0608F46E
:104FB0003FC0255D374FF90180819181A281B38186
:104FC000A816B906CA06DB0698F5882D61E00E948E
:104FD000153AF201808190E00E2C02C095958795DC
:104FE0000A94E2F780FF16C08EE061E00E94EA6555
:104FF00080919402882371F0FAE08F9FB001112410
:10500000882777FD8095982F0E94F3668EE060E0F8
:105010000E94EA65F101808190E002C09595879534
:105020009A94E2F780FF04C0882D61E00E940D424F
:105030000894E11CF11CF8E0EF16F10409F071CFBF
:10504000739480910C0A781608F44DCFC601B5010F
:105050000E94A0220E944442B0910D0A2BE2822EAF
:1050600028E0922E80E0EE24FF24870160E070E0CB
:105070002BC0F4012081318142815381A216B306F5
:10508000C406D506D8F4FB0193E0F595E7959A950B
:10509000E1F7F0E0EE5CF54F808190E0A77002C090
:1050A00095958795AA95E2F780FF07C0E216F3066B
:1050B0000407150710F479018A0181E06F5F7F4FC3
:1050C00024E030E0820E931EA62F6B1790F2E09240
:1050D0002309F092240900932509109326098823B7
:1050E00061F50E94393A0E944442ABEEB8E080E09C
:1050F00090E0FC01E559F84F108211821282138270
:10510000FC01E55DF74F10821182128213821D921D
:105110000496803C910569F71092230910922409A6
:1051200010922509109226098091060A877F8093A4
:10513000060A80914C028093080A5090080A552074
:1051400009F470C0809152029091580240900D0A6B
:10515000FF2401E010E0252C3324682E77248824D6
:105160009924492F50E060E070E04C53504060407B
:10517000704050C02F2D30E02016310609F447C092
:10518000D90183E0B695A7958A95E1F7F7E0EF2E70
:10519000EF20FD01E25FF54F808190E00E2C02C010
:1051A000959587950A94E2F780FF31C0AC5EB54FC4
:1051B0008C9190E002C095958795EA94E2F780FF84
:1051C00026C0220F331F220F331FF901E559F84F74
:1051D00080819181A281B381860D971DA81DB91D83
:1051E000A816B906CA06DB0690F0255D374FF9010F
:1051F00080819181A281B381840F951FA61FB71F63
:105200008A159B05AC05BD0510F061E007C0F3945D
:105210000F5F1F4FF41408F4ADCF60E0852D81506F
:105220000E94153AC601B5010E94A0220E94444284
:1052300080912C09882389F4C601B50123E030E070
:1052400040E050E00E948A6A9B01AC012F513D4F23
:1052500081E0F90160810E94353FC601B5010E94DD
:105260003A23C601B5010E94FE0AC601B5010E949B
:105270000724C601B5010E94F71DC75BDF4F0FB6BB
:10528000F894DEBF0FBECDBFCF91DF911F910F917C
:10529000FF90EF90DF90CF90BF90AF909F908F9056
:1052A0007F906F905F904F903F902F9008958F92D6
:1052B0009F92AF92BF92CF92DF92EF92FF920F93A5
:1052C0001F93CF93DF937B018C01EA012CE330E045
:1052D00040E050E00E948A6A6883C801B7012CE36D
:1052E00030E040E050E00E948A6A122F032FF42E33
:1052F000E52E622F732F842F952F2CE330E040E0B2
:1053000050E00E948A6A6983612F702F8F2D9E2D35
:105310002CE330E040E050E00E948A6A122F032F15
:10532000F42EE52E622F732F842F952F28E130E085
:1053300040E050E00E948A6A6A83612F702F8F2DAF
:105340009E2D28E130E040E050E00E948A6A790119
:105350008A01C801B7016C5F7F4F8F4F9F4F27E0D5
:1053600030E040E050E00E948A6A6F5F6B8320E08B
:10537000AA24BB24650101C02F5F822E9924F40169
:10538000EE54F84FCF0183709070892B99F4CF01C0
:1053900064E670E00E94776A892B39F4CF0160E9F6
:1053A00071E00E94776A892B29F48EE691E0A0E0F3
:1053B000B0E004C08DE691E0A0E0B0E0A80EB91E18
:1053C000CA1EDB1EC501A0E0B0E0E816F9060A0718
:1053D0001B0790F62E83F401EE54F84F83E0882EDD
:1053E000912C8E229F228114910499F4CF0164E6BE
:1053F00070E00E94776A892B39F4CF0160E971E08F
:105400000E94776A892B29F48EE691E0A0E0B0E053
:1054100004C08DE691E0A0E0B0E0A81AB90ACA0A7B
:10542000DB0A980187010A191B092C093D09CF01E4
:1054300064E670E00E94776A7C01CF0160E971E068
:105440000E94776AAC01E4EEF2E060E0613051F472
:105450008114910449F4E114F10441F4411551051A
:1054600029F002C0808103C08CE101C08DE190E091
:10547000A0E0B0E0081719072A073B0740F0081B17
:10548000190B2A0B3B0B6F5F31966C30F9F66F5F8F
:105490006D83802F8F5F8C83DF91CF911F910F9150
:1054A000FF90EF90DF90CF90BF90AF909F908F9044
:1054B0000895EF92FF920F931F937B018C018091CF
:1054C0004F0990915009A0915109B0915209E816E5
:1054D000F9060A071B0771F0C801B70144E459E057
:1054E0000E945729E0924F09F09250090093510908
:1054F000109352091F910F91FF90EF9008950E9411
:10550000592A8091490990E008950E94592A809172
:10551000470990E008950E94592A8091480990E037
:1055200008950E94592A8091450990E008950E94AB
:10553000592A8091460990E008954F925F926F92A8
:105540007F928F929F92AF92BF92CF92DF92EF9213
:10555000FF920F931F93CF93DF934C01DC011696BC
:105560001C91612F70E080E090E020E833E341EE91
:1055700051E00E94386A5B016C0122EB37E0E12FB9
:10558000F0E0EE54F84F1DC0C90183709070892B74
:10559000B1F4C90164E670E00E94776A892B39F49E
:1055A000C90160E971E00E94776A892B41F480E8C3
:1055B00091E5A1E0B0E0A80EB91ECA1EDB1E2F5F68
:1055C0003F4F2E173F0701F7D40115968C91482EB7
:1055D0005524C90164E670E00E94776A7C01C90124
:1055E00060E971E00E94776A8C01C1E0D0E093E04D
:1055F000692E712C6222732227C0C230D10591F42A
:105600006114710479F4E114F10419F40115110520
:1056100049F480E89BE3A6E2B0E0A80EB91ECA1EDA
:10562000DB1E11C0FE01ED51FD4F608170E080E096
:1056300090E020E831E541E050E00E94386AA60E93
:10564000B71EC81ED91E2196C415D505B4F2D401C3
:1056500012966C9170E080E090E020E13EE040E046
:1056600050E00E94386A7B018C01F401618170E096
:1056700080E090E02CE330E040E050E00E94386AA7
:10568000E60EF71E081F191FD4018C91E80EF11CBD
:10569000011D111D14966C9170E0615070408827B7
:1056A00077FD8095982F20E831E541E050E00E9499
:1056B000386AE60EF71E081F191FEA0CFB1C0C1DAA
:1056C0001D1DB701C801DF91CF911F910F91FF9070
:1056D000EF90DF90CF90BF90AF909F908F907F9092
:1056E0006F905F904F9008956093D8017093D901A7
:1056F0008093DA019093DB01089560933A097093E7
:105700003B0980933C0990933D092091D801309149
:10571000D9014091DA015091DB01260F371F481F54
:10572000591F20933E0930933F09409340095093FD
:10573000410982E090E090934309809342090E94DE
:10574000E56660934B0970934C0980934D099093E3
:105750004E090895EF92FF920F931F931CC02F5F85
:105760003F4F4F4F5F4F20933A0930933B0940938F
:105770003C0950933D0988EE93E0A0E0B0E0E80ECC
:10578000F91E0A1F1B1FE0924B09F0924C0900936F
:105790004D0910934E090E94E566E0904B09F09088
:1057A0004C0900914D0910914E096E197F09800B2B
:1057B000910B20913A0930913B0940913C0950915D
:1057C0003D09685E73408040904048F680913E09F4
:1057D00090913F09A0914009B091410928173907DC
:1057E0004A075B07E8F0E0913809F09139093097F2
:1057F000B9F00995611571058105910519F00E94AF
:105800007D2B0EC020E030E0809142099091430949
:10581000892B11F021E030E03093430920934209B5
:1058200060913A0970913B0980913C0990913D0942
:105830001F910F91FF90EF900895909339098093F5
:10584000380980913A0990913B09A0913C09B091A7
:105850003D0980933E0990933F09A0934009B0937E
:1058600041090E94AA2B0895482F6AE00E94576AB6
:10587000282F30E084E0220F331F8A95E1F7842F30
:105880000E94576A892F820F0895CF93DF93EC010E
:1058900080915309909154098836910559F580ED0E
:1058A0009CE068E670E00E94DC6180ED9CE060E0D6
:1058B0000E945E6288810E94342C682F70E06F77AE
:1058C000707080ED9CE00E945E6289810E94342CA1
:1058D000682F80ED9CE00E945E628A810E94342CD9
:1058E000682F80ED9CE00E945E628B810E94342CC8
:1058F000682F2DC08F36910509F04AC080ED9CE0DD
:105900006FE670E00E94DC6180ED9CE060E00E9448
:105910005E6288810E94342C682F606880ED9CE074
:105920000E945E6289810E94342C682F80ED9CE089
:105930000E945E628A810E94342C682F80ED9CE078
:105940000E945E628B810E94342C682F686080ED1B
:105950009CE00E945E628C810E94342C682F80ED56
:105960009CE00E945E628D810E94342C682F80ED45
:105970009CE00E945E628E818E510E94342C682FC2
:1059800080ED9CE00E945E6280ED9CE00E94A1623E
:10599000DF91CF91089588E690E090935409809329
:1059A000530980ED9CE068E670E00E94DC6180EDC8
:1059B0009CE060E00E945E6280ED9CE00E94A1623B
:1059C0008823D9F08FE690E090935409809353098F
:1059D00080ED9CE06FE670E00E94DC6180ED9CE071
:1059E00060E00E945E6280ED9CE00E94A1628823DC
:1059F00021F0109254091092530908951F93CF93E8
:105A0000DF93EC01609153097091540961157105A0
:105A100009F46FC080ED9CE00E94DC6180ED9CE0A9
:105A200060E00E945E6280ED9CE00E94A162609155
:105A300053097091540980ED9CE047E050E00E94CA
:105A4000B26280ED9CE00E94EF61282F2F772295B3
:105A50002F701AE0219F900111248F70820F88838C
:105A600080ED9CE00E94EF61282F22952F70219FEE
:105A7000900111248F70820F898380ED9CE00E9439
:105A8000EF61282F2F7322952F70219F90011124F1
:105A90008F70820F8A8380ED9CE00E94EF61877097
:105AA0008B8380ED9CE00E94EF61282F22952F7060
:105AB000219F900111248F70820F8C8380ED9CE0D8
:105AC0000E94EF61282F22952F70219F90011124B1
:105AD0008F70820F8D8380ED9CE00E94EF61282FF4
:105AE0002F70225E82958F70819FC0011124280F34
:105AF0002E83DF91CF911F9108950F931F93DF9312
:105B0000CF93CDB7DEB727970FB6F894DEBF0FBEA1
:105B1000CDBF8E010F5F1F4FA8010E945729C801FA
:105B20000E94452C27960FB6F894DEBF0FBECDBF5E
:105B3000CF91DF911F910F9108950F931F93DF93E2
:105B4000CF93CDB7DEB727970FB6F894DEBF0FBE61
:105B5000CDBF8E010F5F1F4FC8010E94FE2CC801F0
:105B60000E949D2A27960FB6F894DEBF0FBECDBFC8
:105B7000CF91DF911F910F91089580ED9CE00E94DD
:105B8000B6620895DF92EF92FF920F931F93CF9327
:105B9000DF93D82E862FBA01213041F4675F7F4F03
:105BA0009B0140E050E0695070400EC0223029F067
:105BB00020E030E040E050E007C0625070409B01C0
:105BC00040E050E06E5F7F4FE82EFF248CE593E0CD
:105BD000E80EF91E8B01E7010FC0F881E0E0898132
:105BE00090E08E2B9F2BA0E0B0E0280F391F4A1FBA
:105BF0005B1F2296025010400230110570F7CB0156
:105C00008E7FD701A80FB91F6817790779F08C919B
:105C100090E0A0E0B0E0BA2FA92F982F882702C00B
:105C200040E050E0280F391F4A1F5B1FCA01AA2716
:105C3000BB270097A105B10599F7C90180959095FB
:105C4000ED2DF0E0E45AFC4F90838183DF91CF91FA
:105C50001F910F91FF90EF90DF90089510927403C1
:105C60001092750380E48093700310927103809307
:105C7000720388E16EE044E150E020E00E94C22D12
:105C80000895282F662321F0809181038617E1F47F
:105C9000809182038823C1F4809183038833A1F427
:105CA00080917F038B3781F4E22FF92F8091AE032F
:105CB00083838091AF0382838091B003818380913D
:105CC000B103808381E0089580E0089580915509B3
:105CD00086958095817008958091CC0980959091EA
:105CE000C809892B8093D0098091CD098095909126
:105CF000C909892B8093D1098091CE098095909113
:105D0000CA09892B8093D2098091CF0980959091FF
:105D1000CB09892B8093D309089590936A098093C6
:105D20006909709374096093730950936C094093E7
:105D30006B0980E298E090936E0980936D09109250
:105D4000700910926F093093720920937109309194
:105D5000DE012091DF018CEF94E390935D09809345
:105D60005C098CE394E390935F0980935E09209330
:105D700058093093590981E0809356098091570959
:105D80008F5F8770809357098093680908950F93F8
:105D90001F93BC010CE513E0C8010E940436C80142
:105DA000069662EC79E00E9404361F910F910895E7
:105DB000EF92FF920F931F937B010E94C72E0AE779
:105DC00013E0C801B7010E940C36C801049768ECC3
:105DD00079E00E940C361F910F91FF90EF9008958B
:105DE000EF92FF920F931F93CF93DF937C01EB0110
:105DF0008A0180E699E00E94D82E8881807F803ECB
:105E000049F088819981AA81BB818F5F9F4FAF4FF5
:105E1000BF4F31F48CE593E060EF72E00E940436EE
:105E200088E080936803109269038AE693E06BE749
:105E300077E049E050E00E94740610926C0381E123
:105E4000809373031093800300938103F0927E0389
:105E5000E0927F03109282031092840310928503D4
:105E6000DF91CF911F910F91FF90EF900895EF92E6
:105E7000FF920F931F9302E613E0C8010E94C72E02
:105E800074E1E72EF12CE00EF11EC8014896B7012F
:105E90000E940C36C70168EC79E00E940C360E9423
:105EA0002E2E1F910F91FF90EF900895BC0110923C
:105EB000E7091092E60981E08093550984ED99E0A5
:105EC0000E940C3608950F931F938C01889690932F
:105ED0006C0380936D030E942E2E10928E031092FD
:105EE0008F03045E1F4F82E36AE1A80122E00E9453
:105EF000C22DC8014A960E94184B1F910F91089518
:105F0000FF920F931F93CF93DF93EC01F62E042F94
:105F100010E08091750990917609A0917709B09170
:105F200078092B2F33274427552720938203A093EA
:105F300083039093840380938503F0928B03CE01B7
:105F40000E94632F1F5F011720F79E0140E050E081
:105F50008091750990917609A0917709B09178099F
:105F6000820F931FA41FB51F809375099093760924
:105F7000A0937709B0937809DF91CF911F910F918A
:105F8000FF900895CF93DF939C01862F80618093CB
:105F90008B03643029F02115310511F421E030E044
:105FA0009091800380917E038093800390937E0381
:105FB0009091810380917F038093810390937F036D
:105FC000C5E8D3E08881A901480F511D2C814C837D
:105FD0002883252F3327219753E0C138D50791F720
:105FE0001D861E8680E5898710926C0388E2809367
:105FF0006D030E94372F84E08B871C8682E36AE161
:106000004CE150E022E00E94C22D86E390E00E9425
:10601000184BDF91CF91089580916609909167099F
:1060200060E00E94C22F8091820390E0A0E0B0E087
:10603000BA2FA92F982F882720918303820F911DB3
:10604000A11DB11DBA2FA92F982F88272091840355
:10605000820F911DA11DB11DBA2FA92F982F88273E
:1060600020918503820F911DA11DB11D809375099B
:1060700090937609A0937709B09378090895E82F53
:106080004091800350E0292F30E04217530709F078
:1060900092C0809181038E1709F08DC080918B038F
:1060A000E82F81FF4EC010926C038CE280936D0349
:1060B0000E94372F82E180938B039091800380911F
:1060C0007E038093800390937E039091810380915F
:1060D0007F038093810390937F03E5E8F3E021E061
:1060E00030E08081A901480F511D44831082252F83
:1060F0003327319753E0E138F50799F7158616866F
:10610000118212828091DD01838314828D5F8093DE
:10611000DD0182E0818B84E0828B95E0938B148A91
:1061200080E68187938788E7848782E36AE140E29B
:1061300050E022E00E94C22D8AE390E00E94184BBA
:106140003AC084FF38C090916C0380E020916D03C9
:1061500030E0282B392B80918A03482F50E0A4E0AF
:1061600055954795AA95E1F7CA01880F991F880FA1
:10617000991F281B390B2451304037FF02C020E003
:1061800030E03093670920936609232B69F09A0168
:10619000220F331F220F331F2E5D3F4F6850704078
:1061A0006217730740F009C0E0FF05C080E090E08F
:1061B00060E00E94C22F20E030E0C90108950F93F3
:1061C0001F93DF93CF930F92CDB7DEB78C01045EA0
:1061D0001F4F10936C030C511040802F845E8093EE
:1061E0006D0389830E942E2E085F1F4F1093820338
:1061F0008981845180938303085F1F4F88E26AE19D
:10620000A80121E00E94C22DC8014A960E94184BA5
:106210000F90CF91DF911F910F910895FF920F93EF
:106220001F939C01F62E80E699E0B9010E94D82EBA
:1062300008E613E088E08093680310926903C801C0
:1062400002966BE777E049E050E00E9474068CE428
:1062500080936D0381E1809373030E942E2E109230
:1062600080038BE7809381038AE080937E03F09222
:106270007F031092820388E3809383031092840348
:1062800010928503025E1F4F80E3F80111928A95F8
:10629000E9F7C80162E378E04AE050E00E94740642
:1062A00088E26AE140E450E021E00E94C22D8AE5E4
:1062B00090E00E94184B1F910F91FF900895EF926C
:1062C000FF920F931F93BC0180E699E00E94D82EA5
:1062D00008E613E088E0F82EF09268031092690354
:1062E000C80102966BE777E049E050E00E9474062F
:1062F00084E580936D03EE24E394E09273030E949F
:106300002E2EF0927E0310927F0310928003109243
:10631000810385E0809382038091CB09809383037E
:1063200010928403E0928503C8014E9662E470E007
:1063300048E350E00E94A50684E262E240E450E0B7
:1063400020E00E94C22D82E690E00E94184B1F912F
:106350000F91FF90EF900895DF92EF92FF920F93CD
:106360001F93CF93DF93EC018091E409882319F008
:10637000CE010E940046209709F0BFC080915509C8
:106380008570F1F18091E6099091E709892BC1F5BB
:106390000E94504A8823A1F180EF92E00E94C72E0C
:1063A00088E080936803E6E0FE2EF09269038AE6B7
:1063B00093E063E777E048E050E00E9474060CE762
:1063C00013E0D8011D92FA94E9F7C8010A9762EC2C
:1063D00079E00E940436C801069664ED79E00E94D7
:1063E0000C36C801049768EC79E00E940C36809165
:1063F00055098860809355098AE290E00E94184B05
:106400008091E6099091E70901969093E7098093BE
:10641000E60980915609813009F003C2809155093F
:1064200081FFFFC102E0009356098091DC018F5F7C
:106430008093DC018F71109157091295110F107E16
:10644000182BE0905809D090590980E699E060EE49
:1064500079E00E94D82E78E0F72EF092680310922F
:1064600069038AE693E06BE777E049E050E00E9439
:1064700074068CE280936D0386E0809373030E9420
:106480002E2EE0928003D09281038BE080937E03D6
:1064900010937F03E2E8F3E0DF011D92FA94E9F73D
:1064A0008091DD01809384038D5F8093DD0180E620
:1064B00080938A0300938B0383E080938C03109274
:1064C0008D0310928E0310928F03109290031092FE
:1064D00091030093920384E08093930300939403C9
:1064E00086E28093950382E36AE140E250E022E095
:1064F0000E94C22D8AE390E0AFC0C932D10508F4F2
:1065000090C110916803183009F096C18091690319
:10651000863009F091C182E893E068EC79E044E0CC
:1065200050E00E948F06009709F086C180917103A8
:10653000813029F582E693E00E94C72E1092700305
:1065400082E0809371038CE793E062E773E00E943E
:10655000043682E793E062EC79E00E94043682E838
:1065600093E068E773E00E940C3688E793E068ECFC
:1065700079E00E940C368AE290E00E94184B8091EC
:10658000550983FF4EC110917103123009F049C1C2
:1065900088E793E064ED79E044E050E00E948F06E4
:1065A000009709F03EC180E699E062E773E00E943F
:1065B00004361093550935C1183009F032C1809165
:1065C0006903882309F02DC180916A03853409F09D
:1065D00028C18AE793E068EC79E044E050E00E944B
:1065E0008F060097A9F08AE793E060ED79E044E038
:1065F00050E00E948F06009759F08AE793E060EF21
:1066000072E044E050E00E948F06009709F009C153
:1066100080917303813019F580917E038830F9F4FD
:10662000E0915A09F0915B09309719F086E793E001
:1066300009950E94372F10927E0380918003883F36
:1066400028F0809181038F5F809381038091800384
:10665000885F80938003CE010E94184BE2C00E94A5
:106660001836882351F080917303813131F4CE01C3
:106670000E941D36882309F0D4C0C633D10528F402
:1066800080917303863009F0CCC0809180038B30F9
:1066900009F0BEC086E793E060EE79E044E050E0A8
:1066A0000E948F06009709F0BCC080918B03382FA1
:1066B00082FF13C0E0915C09F0915D09309759F0B9
:1066C0008091810382958695877063E040E050E079
:1066D00020E030E0099585E090C090916C0380E067
:1066E00020916D03022F10E0082B192B80918A0353
:1066F000482F50E064E0559547956A95E1F7CA0147
:10670000880F991F880F991F081B190B04511040FF
:1067100017FF02C000E010E080915609823079F541
:1067200031FF21C034FF1FC080E090E060E00E9494
:10673000C22F88E180938B03E0915E09F0915F099D
:10674000309719F420E030E007C080917F038295F4
:106750008695877009959C0183E080935609C9014D
:106760000E94632F5EC081E08093560934FF03C00E
:1067700080E090E002C0C801019664E046C083302A
:1067800081F50115110579F1E0915C09F0915D0940
:10679000309749F1440F551F440F551FCE010897FC
:1067A0004E5D5F4F8417950708F4AC01C801840F54
:1067B000951FC817D90710F0980103C09E01241B2C
:1067C000350B8091810382958695877060E00995ED
:1067D0008091E509882319F0C80168E016C0C80156
:1067E00008C08530F1F030FF0BC08330D1F0C80114
:1067F000019669E00E94C22F86E08093560911C07D
:106800000115110571F0C80160E00E94C22F09C096
:106810008091DE019091DF01BE010E943F309C011A
:1068200002C020E030E0C901DF91CF911F910F91AC
:10683000FF90EF90DF900895CA32D10508F0BCCEEA
:10684000F0CFBC01809173038130A1F480917E036D
:10685000882381F480918603823461F486E793E093
:1068600044E050E00E948F069C0180E0232B19F445
:1068700081E0089580E00895CF92DF92EF92FF9239
:106880000F931F93DF93CF93CDB7DEB728970FB643
:10689000F894DEBF0FBECDBF22E933E03E832D83E7
:1068A00038872F8390916809891709F08FC01C825F
:1068B0001B8285ED92E09A83898340916F09509104
:1068C000700941155105A9F58DB79EB70C970FB604
:1068D000F8949EBF0FBE8DBFEDB7FEB73196CE01C7
:1068E0000196ADB7BEB712969C938E9311978CEF1D
:1068F00097E0938382838091690990916A099583D7
:106900008483809173099091740997838683809121
:106910006B0990916C099187808780916D099091A6
:106920006E09938782870E94DD368DB79EB70C96DD
:1069300048C020916D0930916E09E0906909F0908E
:106940006A0900916B0910916C092115310519F044
:1069500061E471E004C064E471E024E837E0DA0146
:106960000D900020E9F76D010894C108D108C41A00
:10697000D50A8DB79EB740970FB6F8949EBF0FBE4D
:106980008DBFEDB7FEB73196CE010196ADB7BEB75C
:1069900012969C938E93119785E897E09383828358
:1069A000F582E482178306833187208773876287A5
:1069B000D586C486578746870E94DD368DB79EB739
:1069C00040960FB6F8949EBF0FBE8DBF2F813885BD
:1069D0008D819E81281B390BC90128960FB6F8942A
:1069E000DEBF0FBECDBFCF91DF911F910F91FF9002
:1069F000EF90DF90CF9008950F931F93CF93DF9385
:106A0000890190916809891759F0E0917109F09115
:106A1000720984E060E070E040E050E009952AC02F
:106A2000662341F52D30310528F1C0917109D091CF
:106A300072092097F9F04B595C4F85E491E0BA0157
:106A400043E050E00E94C9069C0180E0232B09F03E
:106A500081E060918A0370E0B4E075956795BA951E
:106A6000E1F7660F771F660F771F6E5D7F4FA801F6
:106A7000FE01099580E0DF91CF911F910F9108955C
:106A8000EF92FF920F93CF93DF93DC01EB01722F14
:106A9000532F002331F4822F932F9C01F90160E0E2
:106AA0003EC0822F932FFC0160E019C084913327F0
:106AB00027FD309590E02817390769F431968491C5
:106AC000882361F411968C918D3329F4872F952FAB
:106AD000FC0161E003C0872F952FFC0111962C91DA
:106AE000222339F1203229F12A3019F16623F1F2FB
:106AF00024C08081981771F431968081882371F4C5
:106B000011968C918D3331F4872F952F9C01F901CB
:106B100061E004C0872F952F9C01F90111969C918B
:106B2000992339F0903229F09A3019F0662309F34D
:106B300004C0613011F030E018C07A2F50E04150AD
:106B4000504002C0299311963A2F371B2C912223D3
:106B500059F0203249F02A3039F0263229F0832FBB
:106B600090E08417950774F31882E114F10411F092
:106B7000F7016083832FDF91CF910F91FF90EF900A
:106B80000895CF93DF93FC01EC0137C08B3211F4F1
:106B900080E231C0853279F5DF0111969181392F7C
:106BA00030533A3070F0892F8156863010F43752C6
:106BB00008C0892F8154863010F030E002C0392F90
:106BC0003753FD01319611962C91922F90539A30A4
:106BD00070F0822F8156863010F4975208C0822FB1
:106BE0008154863010F090E002C0922F9753832F8B
:106BF0008295807F892B899331968081882331F615
:106C00001882DF91CF910895DC01FB0186E00190AD
:106C10000D928150E1F708959C01FB0180819181E3
:106C2000A281B381F90180839183A283B383089504
:106C30008091A109811181E00895CF92DF92EF92B6
:106C4000FF920F931F93CF93DF93C9E7D9E0CC2432
:106C5000DD2430E029C02A814B818091800390E0BF
:106C6000042F10E080179107D9F4909181039217B7
:106C7000B9F48C818823A1F02091830330E028505F
:106C80003040F0908203EE242E0D3F1DE881F98103
:106C9000892F942F66E773E046E853E0099531E0C9
:106CA0000894C11CD11C25968091A10990E0C816BA
:106CB000D9068CF2832FDF91CF911F910F91FF9016
:106CC000EF90DF90CF900895EF92FF920F931F9374
:106CD000CF93DF93FC01EB018A0179011092E40963
:106CE000009729F088EC99E0BF010E940C362097AC
:106CF00019F0CE010E94562F0115110529F08CEDD7
:106D000099E0B8010E940C36E114F10429F08CECF2
:106D100099E0B7010E940C360E946C2E1092E70990
:106D20001092E60981E0DF91CF911F910F91FF90C2
:106D3000EF900895AF92BF92CF92DF92FF920F93A0
:106D40001F93CF93DF938C01EB01F42E1092E40993
:106D500038E341E050E060E070E018C0832F90E03D
:106D6000FC01B3E0F595E795BA95E1F7EE55F64FDE
:106D7000877090705A016B0104C0AA0CBB1CCC1C1C
:106D8000DD1C8A95D2F720812A292083315031F7E2
:106D900082EC99E0BE010E940436C80162EC79E001
:106DA0004F2D0E94724BDF91CF911F910F91FF9059
:106DB000DF90CF90BF90AF900895CF92DF92EF9287
:106DC000FF920F931F93DF93CF93CDB7DEB7EB8482
:106DD000FC84CD84DE84DE011F9601C0D801F6015B
:106DE0008491882309F4BCC00894C11CD11C84324E
:106DF00009F099C0F6010894C11CD11C8491863415
:106E000009F45FC0873434F4843469F0853409F0C0
:106E10008AC06EC08C34C9F1833509F445C088340A
:106E200009F081C00DC08D010E5F1F4FF701668113
:106E300077818D919C914AE050E00E941E077EC0B0
:106E40002C91822F992787FD909514E09595879531
:106E50001A95E1F78F702F702A300CF0295F8A3075
:106E60000CF0895F8D010E5F1F4FF701A681B7817E
:106E7000805DFD018193205D11962C933196D701A1
:106E80001796FC93EE931697A9CF8D010C5F1F4FB9
:106E90006D917D918D919C91F701468157812AE0FA
:106EA00030E00E945C074AC08D010E5F1F4F6D915C
:106EB0007C91D70116968D919C9117970E94C206DE
:106EC0003DC08D010E5F1F4F2D913C910AC0D7012F
:106ED0001696ED91FC91179781931796FC93EE937C
:106EE0001697F9012F5F3F4F8491882381F776CF62
:106EF0008D010E5F1F4F2D913C910AC0D701169650
:106F0000ED91FC91179781931796FC93EE9316974A
:106F1000F999FECF32BD21BDF89A80B52F5F3F4F62
:106F2000882361F75BCFF70126813781F9018193CF
:106F30009F01F701378326838D0150CFD701169625
:106F40008D919C911797FC0101900020E9F73197F2
:106F5000E81BF90B8E0F9F1FF701978386833ECFA7
:106F6000CF91DF911F910F91FF90EF90DF90CF9025
:106F70000895FF920F931F93CF93DF938C01F62E0A
:106F80000E94E566EB010CC00E948F4A0E94AC3162
:106F90000E94E5666C1B7D0B6053754708F0EFC0DF
:106FA0000E94504A882381F30E94E566EB010CC0E1
:106FB0000E948F4A0E94AC310E94E5666C1B7D0BDB
:106FC0006053754708F0DBC00E94662E882381F766
:106FD0001092E0091092E1091092E2091092E3097F
:106FE0008091E8098F5F8093E8098091DC0988230C
:106FF00061F488E098E0A8E0B8E08093DC09909321
:10700000DD09A093DE09B093DF098091E80990E0E3
:10701000906E6CED79E045E350E00E94F02EE6E8DA
:10702000F3E08CE0DF011D928A95E9F7DF011C9601
:1070300090E0FF2019F0F801808102C0F8018491EE
:107040000F5F1F4F8E3241F0882331F09F5FFD01AB
:10705000E90FF11D8083EDCFFD019193DF01A90FB1
:10706000B11D882329F7FD01119211961C92DF01B1
:10707000119641E04183FD01319611961C924183A6
:1070800086ED2CE533E0821B32968E0F80938603CB
:107090009091E809909387034093880340938B0372
:1070A00090E00E94DF300E94E5668B0161C00E9483
:1070B000E566601B710B6053754708F060C00E9465
:1070C0008F4AEC01009709F453C00E94AC31892B20
:1070D00009F04EC0C634D10508F44AC080917F0340
:1070E000853309F045C080918003803E09F040C09F
:1070F000909181038091E8099817D1F580918703D9
:107100008917B1F58091890390E08F709070892B79
:10711000B1F580918603E82FF0E0EA57FC4F9E011D
:10712000245A3C4F8081807C39F0329609C080819E
:10713000882311F4319604C03196E217F307B8F3AF
:10714000CF010E962817390798F08181813051F4CC
:107150008185843039F43A9680EE99E0BF010E942F
:107160000C3606C0818590E00A96E80FF91FDACF49
:107170008091E009882309F49ACF81E001C080E082
:10718000DF91CF911F910F91FF9008959C01F99984
:10719000FECF32BD21BDF89A80B508959C01F999C2
:1071A000FECF1FBA32BD21BD60BD0FB6F894FA9A6A
:1071B000F99A0FBE0895E091550AF091560A099583
:1071C0000895EF92FF920F931F93782F282F392F56
:1071D000F90120E030E040E050E03CC0F999FECFFA
:1071E000F2BDE1BDF89A90B579018A0184E0EE0C18
:1071F000FF1C001F111F8A95D1F7892F80538A30F9
:1072000030F4892F992787FD9095C09719C0892F51
:107210008154863030F4892F992787FD9095C79740
:107220000FC0892F8156863028F020E030E040E002
:1072300050E015C0892F992787FD9095875590407C
:107240009C01442737FD4095542F2E0D3F1D401FB4
:10725000511F31968E2F871B861708F4BFCFB901B7
:10726000CA011F910F91FF90EF900895EF92FF9246
:107270000F931F93CF93DF938B017A01C82FD0E038
:1072800094E0CC0FDD1F9A95E1F7CC55DB4FCE0192
:1072900066E00E94E138611571058105910521F1D3
:1072A0000115110529F0F8016083718382839383AE
:1072B000CE01069666E00E94E138611571058105F0
:1072C000910591F0E114F10429F0F70160837183D5
:1072D00082839383CE010C9664E00E94E1386115AD
:1072E00071058105910511F460E070E0CB01DF913B
:1072F000CF911F910F91FF90EF900895FB0190E0C7
:1073000024E0880F991F2A95E1F7108A9C012C55DB
:107310003B4FAC014C545B4FF999FECF32BD21BDC0
:10732000F89A80B58083882331F02F5F3F4F3196E4
:107330002417350789F70895FB0190E034E0880FA2
:10734000991F3A95E1F7108A9C012C553B4F8C54BC
:107350009B4F4081F999FECF1FBA32BD21BD40BD80
:107360000FB6F894FA9AF99A0FBE442331F0319689
:107370002F5F3F4F2817390761F70895AC01FB01D4
:107380000FC0F999FECF1FBADA01A80FB11DB2BD27
:10739000A1BD20BD0FB6F894FA9AF99A0FBE3196A6
:1073A0008E2F861B2081222361F7F999FECF1FBA09
:1073B000480F511D52BD41BD10BC0FB6F894FA9A4A
:1073C000F99A0FBE0895FC0184EF93E0F999FECF7E
:1073D00092BD81BDF89A30B52081332339F0222344
:1073E00051F00196321739F43196F0CF80E0222324
:1073F00019F481E0089580E00895FC01CB01F9992A
:10740000FECF92BD81BDF89A30B52081332349F07B
:10741000222339F00196321711F081E00895319658
:10742000EECF80E0321381E00895282F27708695F3
:107430008695869590E0662369F0FC01E25FF54F42
:1074400081E090E002C0880F991F2A95E2F7208121
:10745000282B0DC0FC01E25FF54F81E090E002C0F7
:10746000880F991F2A95E2F7809520812823208391
:10747000089510920E0A10920F0A1092100A10929C
:10748000110A1092120A1092130A0895AF92BF9235
:10749000DF92EF92FF920F931F93CF93DF930CE253
:1074A0001AE0EE24FF2441E0A42EB12CF801108252
:1074B000DE2CDD0CDD0CDD0CC0E0D0E08D2D8C2B46
:1074C00060E070E040E050E00E943639892B59F0CE
:1074D00095010C2E02C0220F331F0A94E2F7F80127
:1074E0008081822B80832196C830D10539F708949A
:1074F000E11CF11C0F5F1F4FF6E0EF16F104B1F62F
:10750000DF91CF911F910F91FF90EF90DF90BF908F
:10751000AF900895E0EEF1E022EC37E0F999FECF6C
:1075200032BD21BDF89A80B580832F5F3F4F3696DC
:1075300087E0283E380791F780913A028F5F809369
:107540000C0A90E053E0880F991F5A95E1F7809359
:107550000D0A9091700291708091060A8E7F892B9E
:107560008093060A0895EEEBF2E087EE97E0208123
:10757000F999FECF1FBA92BD81BD20BD0FB6F89418
:10758000FA9AF99A0FBE3697019721E0EA3DF20781
:1075900071F780913A028F5F80930C0A90E063E06C
:1075A000880F991F6A95E1F780930D0A90917002F8
:1075B00091708091060A8E7F892B8093060A089528
:1075C0008091060A81608093060A81E080937002B0
:1075D0000E94B33A08958091060A8E7F8093060A2E
:1075E000109270020E94B33A08958C33910510F402
:1075F000682F15C02AE28033920730F46CE370E004
:107600000E94636A655C0BC02DEF8032920710F018
:107610006EEF05C060E17EE00E94636A6451862FD0
:107620000895CF93DF93EC01D7FF04C088279927F3
:107630008C1B9D0B0E94F53A982FD7FD02C08058F5
:1076400002C080E8891BDF91CF910895482F90E018
:107650008058904097FF03C0909581959F4F282FA9
:1076600030E08C3360F08CE390E0B901689F9001CA
:10767000699F300D789F300D1124245D3D4047FDFA
:1076800003C0309521953F4FC9010895282F30E060
:107690008C33D8F08F3E68F48CE390E0A901489FCA
:1076A0009001499F300D589F300D1124245D3D40BD
:1076B0000CC080E19EE0A901489F9001499F300DD8
:1076C000589F300D1124205C364FC9010895109247
:1076D000EC091092EB0980E293E09093EA09809321
:1076E000E9090895EF92FF920F931F93CF93DF93D1
:1076F000E82E162F042FF22E662321F0623081F43B
:10770000222371F08E2D0E943E66892B11F000E03D
:1077100024C0FF2011F480E001C080E8082B1DC0C8
:10772000C0E0D0E08E2D0E943E66892B81F411309E
:1077300031F0123061F483E0C83ED80744F461E0D0
:1077400070E080E090E00E94F3662196EBCFFF208E
:1077500019F4C85ED3400CF00068802FDF91CF9100
:107760001F910F91FF90EF9008950F931F93082F93
:107770001091570A107861E070E080E090E00E947C
:10778000F3668FE10E943E66892B21F48FE1602F22
:1077900041E013C08EE10E943E66892B21F48EE108
:1077A000602F42E00AC08DE10E943E66892B11F0F5
:1077B00040E007C08DE1602F44E0212F0E94723B22
:1077C000482F8091570A90E08F709070242F30E0FE
:1077D000892B39F42F703070232B71F0842F806443
:1077E00006C02F703070232B39F4842F80624093B1
:1077F000570A1F910F910895842FF9CF8BE00E94B3
:107800003E6640E02091640230E08217930709F061
:1078100041E0440F440F8091060A8B7F842B8093B4
:10782000060A08951F93182F843690F064E60E948C
:10783000576A682F89EE99E070E04AE050E00E94B4
:10784000136A89EE99E069E471E00E94266A02C039
:107850008A30A0F0812F6AE00E94576A0E94576A1E
:10786000692F89EE99E070E04AE050E00E94136AC7
:1078700089EE99E069E471E00E94266A812F6AE04E
:107880000E94576A692F89EE99E070E04AE050E063
:107890000E94136A1F910895EF92FF920F931F9316
:1078A0008C0179EEE72E79E0F72E6AE070E00E9415
:1078B000776AC7014AE050E00E94136AC8016AE093
:1078C00070E00E94776ABC01C7014AE050E00E9464
:1078D000136A1F910F91FF90EF900895CF93DF935C
:1078E000EC0104C089EE99E00E943369FE01219603
:1078F00064916623B9F7DF91CF910895FF920F93BA
:107900001F93CF93DF938C0189EE99E060E040E014
:107910000E94B5488FEF9AE00E946E3CE801FF2478
:10792000688170E0A4E075956795AA95E1F789EE06
:1079300099E040E150E00E94136A699170E06F7035
:10794000707089EE99E040E150E00E94136A8DEF7B
:107950009AE00E946E3CF39484E0F81609F789EEF1
:1079600099E060E041E00E94B548F801648170E070
:10797000F4E075956795FA95E1F789EE99E040E1B5
:1079800050E00E94136AF801648170E06F707070BB
:1079900089EE99E040E150E00E94136A8BEF9AE093
:1079A0000E946E3CF801658170E0E4E07595679592
:1079B000EA95E1F789EE99E040E150E00E94136A10
:1079C000F801658170E06F70707089EE99E040E1B8
:1079D00050E00E94136ADF91CF911F910F91FF90A9
:1079E00008950F931F93CF93DF938C01462F89EE59
:1079F00099E060E00E94B548C0E0D0E0F801EC0FEB
:107A0000FD1F608189EE99E070E04AE050E00E943D
:107A1000136A84E09BE00E946E3C2196C330D1053E
:107A200069F7F801638189EE99E070E04AE050E07F
:107A30000E94136ADF91CF911F910F9108950F93C8
:107A40001F93CF93DF938C01462F89EE99E060E07E
:107A50000E94B548E80104C089EE99E00E943369AC
:107A60009E01201B822FFE01219664916623A1F7BF
:107A7000992787FD9095C0E1D0E0C81BD90B05C0C0
:107A80008FE09BE00E946E3C2197D7FFF9CFDF91FA
:107A9000CF911F910F9108950F931F93CF93DF9371
:107AA0008C01FC01EE0FFF1FE80FF91FEE0FFF1F07
:107AB000EE51FE4F8081918160E00E941F3D81EE7A
:107AC0009AE061E00E941F3D89EE99E060E041E0AC
:107AD0000E94B5480131110509F4A7C00231110512
:107AE0009CF401301105E1F10230110524F4011577
:107AF000110549F1D9C00C30110509F487C00E30C9
:107B0000110509F0D1C019C00B31110509F4B0C03D
:107B10000C3111054CF40331110509F462C0043134
:107B2000110509F0C1C064C00C31110509F4B0C0E1
:107B30000E31110509F0B8C071C089EE99E06BE40F
:107B400071E00E94266AF801EE0FFF1FE00FF11F9F
:107B5000EE0FFF1FE052FE4F80810E94123CC2C018
:107B60008091E601C82FD0E0E097D7FD05C08FEDEA
:107B70009AE00E946E3C07C08DED9AE00E946E3C38
:107B8000D095C195DF4FCE0164E070E00E94776A26
:107B900089EE99E04AE050E00E94136A8BED9AE08A
:107BA0000E946E3CCE0164E070E00E94776A9C0106
:107BB000BC0194E0660F771F9A95E1F7621B730B87
:107BC00029F488ED9AE00E946E3C06C089EE99E0A7
:107BD0004AE050E00E94136A83ED9AE00E946E3CF6
:107BE00087C081ED9AE00E946E3C6091520248C0CD
:107BF000809158028C3320F08FEC9AE00E946E3C0A
:107C00006091580270E06C5370402FC070912E024A
:107C100060E080912802680F711D27C06091940276
:107C20008AE0689FB001112420C020914602822F73
:107C300090E08058904097FF03C0909581959F4FAA
:107C4000682F70E08C3360F08CE390E0AB01489FCC
:107C5000B001499F700D589F700D1124645D7D40E7
:107C600027FD03C0709561957F4F89EE99E00BC0A9
:107C7000609182028DE070E00E944B65609182020B
:107C800089EE99E070E04AE050E00E94136A30C04B
:107C9000809188026FEF70E0681B71098CE00E9490
:107CA0004B6560918802ECCFF801EE0FFF1FE00FEB
:107CB000F11FEE0FFF1FE052FE4F81816081813086
:107CC00051F4662319F488EC9AE002C08BEC9AE038
:107CD0000E946E3C07C089EE99E070E04AE050E0F7
:107CE0000E94136A0731110519F486EC9AE012C05C
:107CF000C8014397029718F481EC9AE00BC0013158
:107D0000110519F48CEB9AE005C00E31110521F430
:107D100088EB9AE00E946E3CDF91CF911F910F910A
:107D200008950F931F93CF93DF93EC010AEA82E04B
:107D30000E94B53B482F50E09A012F7030702230DE
:107D40003105F9F02430310599F12130310509F080
:107D500079C0209709F479C0CE30D10509F475C0F7
:107D6000FE01EE0FFF1FEC0FFD1FEE0FFF1FE05295
:107D7000FE4F90818181891709F467C09F5F9083CE
:107D800064C0209709F45EC0CE30D10509F45AC012
:107D9000FE01EE0FFF1FEC0FFD1FEE0FFF1FE05265
:107DA000FE4F9081992309F44DC0915090834AC0B1
:107DB00086FF48C087FF0AC08091BE02882311F069
:107DC0000093BE020E94B33A11E040C0C330D10517
:107DD00039F48091F2018823E9F0CCE0D0E021C0B1
:107DE000CC30D10519F4CEE0D0E01BC0C531D105AF
:107DF00039F480915E02882369F4C7E1D0E011C0B4
:107E0000C231D10539F480914C02882319F4C5E1BF
:107E1000D0E007C0CE01019666E270E00E94776A6A
:107E2000EC01FE01EE0FFF1FEC0FFD1FEE0FFF1F19
:107E3000E052FE4F0480F581E02DE491EF3529F406
:107E4000219603C0882309F472CF10E0CE010E946E
:107E50004C3D112309F46BCF89EE99E00E94A348B1
:107E6000DF91CF911F910F9108950F931F93CF939F
:107E7000DF93482F062F89EE99E060E00E94B54815
:107E80008091070A8F7019F487EF9AE010C085EF90
:107E90009AE00E946E3C6091070A6F7089EE99E04B
:107EA00070E04AE050E00E94136A83EF9AE00E947B
:107EB0006E3C8091060A80FD06C087EE9AE061E084
:107EC0000E941F3D26C0E091070AEF70F0E0E25FDC
:107ED000F54F1081C1E0D0E08091070A8F7051F416
:107EE00080914C0290E0C817D90721F410FD06C01C
:107EF0006DE405C010FD02C06FE501C0602F89EE82
:107F000099E00E9433692196C930D10511F0169588
:107F1000E3CF82EE9AE00E946E3C89EE99E06DE03C
:107F200041E00E94B5488091060A81FD06C082FFAB
:107F300009C080915E02882329F089EE99E063E010
:107F40000E94714889EE99E06EE041E00E94B548D8
:107F50008091060A85FF05C089EE99E062E00E94E3
:107F6000714889EE99E06FE041E00E94B54860E019
:107F70008091070A82958F7090E003970CF061E082
:107F800089EE99E00E947148DF91CF911F910F9186
:107F9000089584E00E9429659C0183E02E3B380708
:107FA00010F080E0089583E02734380710F081E076
:107FB000089582E02B3E380710F082E0089582E0B9
:107FC000223A380710F083E0089582E0253638071A
:107FD00010F084E008952353324010F085E00895B6
:107FE0008FEF08958CEE93E06EEF79E048E050E07B
:107FF0002EEC38E30E94020708958091060A8D7FD7
:108000008093060A1092020A1092030A1092040A40
:108010001092050A0E94F23F08958091060A82603C
:108020008093060A0E94F23F089546E050E02EEC4D
:1080300038E30E94020708958EEF99E06CEE73E03A
:1080400048E050E026EC38E30E94E606A9E0BAE0FA
:10805000E6E0FAE083E001900D928150E1F70895A7
:108060009C01CB01B90146E050E026EC38E30E94C8
:10807000E606089564EF71E080E090E00E94F36608
:10808000F999FECF82EC97E092BD81BDF89A80B558
:10809000833D59F4F999FECF87EE97E092BD81BDFB
:1080A000F89A80B58A3A09F0A9C081E59BE060E0C2
:1080B0000E941F3D82E49BE061E00E941F3D80E042
:1080C00090E0F999FECF1FBA92BD81BD10BC0FB6EA
:1080D000F894FA9AF99A0FBE019628E08030920738
:1080E00081F70E94F23F84EF93E06DE471E00E941B
:1080F000BE3984E194E066E571E00E94BE3984E413
:1081000094E060E671E00E94BE3984E894E06FE795
:1081100071E00E94BE3924EA34E0E1E0F0E043E59A
:10812000F999FECF1FBA32BD21BD40BD0FB6F894FC
:10813000FA9AF99A0FBEF999FECF1FBA2F5F3F4FF7
:1081400032BD21BD21503040CF016AE070E00E9475
:10815000776A605D60BD0FB6F894FA9AF99A0FBE1F
:10816000F999FECF1FBA2E5F3F4F32BD21BDCF011F
:108170006AE070E00E94776A805D80BD0FB6F89477
:10818000FA9AF99A0FBE225F3F4F87E0243A3807E8
:1081900011F03196C5CF8FEFF999FECF1FBA32BDDE
:1081A00021BD80BD0FB6F894FA9AF99A0FBE2F5FE1
:1081B0003F4F97E02A3A390779F78CEB97E02FEF9A
:1081C000F999FECF1FBA92BD81BD20BD0FB6F894BC
:1081D000FA9AF99A0FBE019637E0823C930781F72D
:1081E0000E94B33A64EF71E080E090E00E94F36691
:1081F000E091550AF091560A099524C00E948A3AE6
:1082000084EA97E064E17AE00E9430408AEA97E0ED
:108210006AE17AE00E94304080EB97E060E27AE029
:108220000E94304086EB97E066E27AE00E943040A0
:108230008CEB97E062E37AE00E9430400E94463A7D
:108240000E941C4080E00E94B53B90E08F709070CF
:108250008130910519F0049779F503C085E290E02B
:1082600020C082E39BE060E00E941F3D60ED77E06C
:1082700080E090E00E94F36681E29BE060E00E9473
:108280001F3D81E19BE061E00E941F3D80E00E9474
:10829000B53B86FFFBCF89EE99E00E94E44880E081
:1082A00090E00E94913E8091BE02882329F0E091E7
:1082B000550AF091560A09958CE061E00E94AB6581
:1082C0008DE061E00E94AB65609182028DE070E01C
:1082D0000E944B65809188026FEF70E0681B710906
:1082E0008CE00E944B650895EF92FF920F931F93CD
:1082F000DC01CB0179018A01139A0E944C67139823
:10830000C7010E944C671F910F91FF90EF90089555
:108310002F923F924F925F926F927F928F929F9295
:10832000AF92BF92CF92DF92EF92FF920F931F9383
:10833000DF93CF9300D00F92CDB7DEB74B015C0136
:1083400079018A01DA01C901880F991FAA1FBB1F91
:108350008E0D9F1DA01FB11F582E692E7A2ECB2E79
:10836000D801C70125E0880F991FAA1FBB1F2A95B6
:10837000D1F78E199F09A00BB10B8983292E3A2EB4
:108380004B2EDD242FC0D501C4010A8004C0B69550
:10839000A795979587950A94D2F780FF07C0652D1A
:1083A000762D872D9C2DA801970106C0C801B70125
:1083B000252D362D472D5C2D0E9474418A819B818D
:1083C00001979B838A838F5F9F4FE9F6C801B701AE
:1083D0002981322D432D542D0E947441D394F8E10C
:1083E000DF1629F087E190E09B838A83CCCF0F9042
:1083F0000F900F90CF91DF911F910F91FF90EF9011
:10840000DF90CF90BF90AF909F908F907F906F90B4
:108410005F904F903F902F9008951F93DF93CF93DD
:10842000CDB7DEB728970FB6F894DEBF0FBECDBF2D
:10843000162FBE016F5F7F4FAE014B5F5F4F0E94F3
:108440003639AC01112329F069817A818B819C81B5
:1084500004C06D817E818F8198859A01369527951C
:108460005695479556954795240F351F40E050E0A7
:108470000E94884128960FB6F894DEBF0FBECDBF8C
:10848000CF91DF911F910895EF92FF920F931F9369
:10849000CF93DF9383E060E00E94EA6503E11AE096
:1084A0008091060A80FD02C060E002C0F801608190
:1084B000C7E0D0E0E62EFF2486E160E00E94EA6596
:1084C000B7010C2E02C0759567950A94E2F76170AA
:1084D00085E10E94EA6586E161E00E94EA652197F4
:1084E000FFEFCF3FDF0741F7015010408AE00D302A
:1084F0001807B1F683E061E00E94EA65DF91CF9151
:108500001F910F91FF90EF900895DF93CF93CDB718
:10851000DEB727970FB6F894DEBF0FBECDBFCE01F2
:1085200001960E94FE2C8C8190E0059667E070E039
:108530000E94776A27960FB6F894DEBF0FBECDBFB4
:10854000CF91DF910895DF92EF92FF920F931F93E7
:10855000D82E0E94AA2B7B018C0189EE99E060E065
:108560004D2D0E94B548C801B7010E94972A0E946C
:108570004C3C8DE09BE00E946E3CC801B7010E941C
:10858000912A0E944C3C8AE09BE00E946E3C0E9433
:108590008542E82FF0E0EE0FFF1FE655F54F85917D
:1085A00094910E946E3C88E09BE00E946E3CC80162
:1085B000B7010E947F2A0E944C3C86E09BE00E940B
:1085C0006E3CC801B7010E948B2A0E944C3C1F914F
:1085D0000F91FF90EF90DF9008958F92AF92CF921E
:1085E000EF920F931F93DF93CF93CDB7DEB7A09792
:1085F0000FB6F894DEBF0FBECDBF81E061E00E94F0
:10860000AB6581E061E00E94EA6583E061E00E9481
:10861000AB6583E061E00E94EA6586E161E00E946B
:10862000AB6585E161E00E94AB6510920E0A109285
:108630000F0A1092100A1092110A1092120A109248
:10864000130A0E94444281E060E00E94EA6580E0F3
:1086500061E00E94AB6580E061E00E94EA6581E034
:10866000809381008CE061E00E94AB658DE061E069
:108670000E94AB65609182028DE070E00E944B65C4
:10868000809188026FEF70E0681B71098CE00E9496
:108690004B6500D000D0EDB7FEB73196ADB7BEB791
:1086A00011961C9211821282138289EE99E061E088
:1086B00043E12FEF02E154E1E52E35E1C32E16E14F
:1086C000A12EB7E18B2E0E945B490F900F900F9067
:1086D0000F9089EE99E060E142E020E00E94EC48D2
:1086E0008BE060E00E94AB658BE061E00E94EA6590
:1086F00080ED9CE00E94B6628091060A81608093C2
:10870000060AA9E0BAE0E6E0FAE083E001900D9203
:108710008150E1F788E691E09093FF098093FE098C
:1087200088E394E09093010A8093000A81E08093AB
:108730000C0A88E080930D0ADE011196EEE0F3E06A
:1087400001900D928150E1F7DE011996E6E0F3E029
:1087500088E001900D928150E1F7DE015196EEEF35
:10876000F2E088E001900D928150E1F7DE01599628
:10877000E6EFF2E088E001900D928150E1F789EE9A
:1087800099E061E08E010F5F1F4FA8010E947B48B6
:108790001A821B8281E08C8389EE99E060E0A80157
:1087A0000E947B4889EE99E062E0AE01475F5F4F2F
:1087B0000E947B4889EE99E063E0AE014F5E5F4F17
:1087C0000E947B4889EE99E064E0AE01475E5F4F0E
:1087D0000E947B488CE161E00E94AB658CE160E027
:1087E0000E94EA658EE061E00E94AB658EE060E089
:1087F0000E94EA658FE160E00E94AB658EE160E077
:108800000E94AB658DE160E00E94AB658FE161E0A5
:108810000E94EA658EE161E00E94EA658DE161E017
:108820000E94EA650E94CB2C882329F48091060AD5
:1088300080618093060AA0960FB6F894DEBF0FBE43
:10884000CDBFCF91DF911F910F91EF90CF90AF905F
:108850008F900895CF93DF9380ED9CE060E570E00A
:108860000E94DC6180ED9CE060E00E945E6280ED31
:108870009CE00E94A162882311F080E029C080ED75
:108880009CE060E570E00E94DC6180ED9CE06AEFB6
:108890000E945E6280ED9CE00E94A16280ED9CE0FF
:1088A00060E570E046E050E00E94B26280ED9CE03E
:1088B0000E94E661892BD1F3CEEAD6E080ED9CE000
:1088C0000E94EF61899386E0C43BD807B9F781E045
:1088D000DF91CF910895DF93CF93CDB7DEB728977F
:1088E0000FB6F894DEBF0FBECDBF82E69BE061E01D
:1088F0000E941F3D0E94AA2B60934C0A70934D0A60
:1089000080934E0A90934F0A6093500A7093510AD5
:108910008093520A9093530A0E942A44882389F430
:108920001092AE0689E68093AF068093B0068DE282
:108930008093B10681E38093B20680917C0280939C
:10894000B30682E593E06EEA76E044E00E949A3650
:10895000882311F490E03AC090912E0280E020919B
:108960002802820F911D9093DF018093DE01809198
:10897000F201882319F00E94804722C08091F801FB
:1089800089838091FE018A83809104028B83809188
:108990000A028C83809110028D83809116028E834F
:1089A00080911C028F83809122028887AE014B5FE9
:1089B0005F4FCE010196BA0120E030E00E9464369C
:1089C00090E0882309F491E081E09827892F289688
:1089D0000FB6F894DEBF0FBECDBFCF91DF910895E3
:1089E000DF93CF9300D000D000D0CDB7DEB7DE014B
:1089F0001196E6E1F3E086E001900D928150E1F7F7
:108A000086E191E0ECE5F3E0DF019C011D9221504D
:108A10003040E1F78091580A833019F468ED79E02D
:108A200003C0BE016F5F7F4F84E490E043E450E0F9
:108A30000E94F02E8091580A833039F08CE593E043
:108A4000BE016F5F7F4F0E94043681E080938603F2
:108A50008093870386E0809388038091650A9091D4
:108A6000660AA091670AB091680A80938A0390937E
:108A70008B03A0938C03B0938D038091580A8330AD
:108A800039F486E893E00C9668EC79E00E940C36A5
:108A900082EA93E062EC79E00E940436A2E7B4E057
:108AA000EAECF2E002C081918D9332E0E03DF30701
:108AB000D1F79091580A992311F083E001C081E029
:108AC000809378048DE38093790487E080937A041F
:108AD00081E080937B04ACE7B4E0E2ECF9E002C013
:108AE00081918D9389E0E83CF807D1F78CE0809381
:108AF000820485E080938304E4ECF2E0A4E8B4E02F
:108B000002C081918D9322E0E93CF207D1F729E878
:108B100034E030936D0A20936C0A913069F582E35A
:108B20008093890484E080938A04D9011296E8EC4A
:108B3000F9E002C081918D9339E0EC3CF307D1F765
:108B400086E380938F0484E08093900481E994E02D
:108B500090936D0A80936C0ADC01E8EDF9E002C0A5
:108B600081918D9389E0EC3DF807D1F785E994E098
:108B700090936D0A80936C0A20916B0A222311F066
:108B800094E001C093E0A0916C0AB0916D0AFD01E0
:108B900087E3819311969C93DF01119681E0818395
:108BA000FD01319683E011968C93DF01119686E0EA
:108BB0008183CD01019690936D0A80936C0A2223E4
:108BC00039F011962C93019690936D0A80936C0A5C
:108BD000E0916C0AF0916D0A8FEF8193F0936D0A2A
:108BE000E0936C0ACF01865893400E94DF302696AE
:108BF0000FB6F894DEBF0FBECDBFCF91DF910895C1
:108C0000EF92FF920F931F93CF93DF938C0180918C
:108C1000580A823009F4F8C0833030F4882351F1C7
:108C2000813009F066C14BC0833021F0843009F0F7
:108C300060C1EAC00E94E56620915D0A30915E0A3B
:108C400040915F0A5091600AE090590AF0905A0AE8
:108C500000915B0A10915C0A2E0D3F1D401F511FB1
:108C6000621773078407950708F443C10E94F04414
:108C700084E018C00E94E5666093650A7093660AF6
:108C80008093670A9093680A1092C8091092C909E4
:108C90001092CA091092CB090E94F04481E00E9410
:108CA0003F4A81E08093580A0E94E5666093610A1A
:108CB0007093620A8093630A9093640A1AC106341F
:108CC000110508F4D5C080917F03833409F0D0C02A
:108CD00020918A0330918B0340918C0350918D0336
:108CE0008091650A9091660AA091670AB091680A1E
:108CF000281739074A075B0709F0BAC0C6E7D4E06E
:108D0000FE01A801445A5C4FDF01119691819D013B
:108D10002F5F3F4F8081853329F411968C918230EB
:108D200009F4C5C0F901E90FF11DE417F50760F377
:108D30009FC0FE019191E980EF0121969333D9F014
:108D4000943340F4933089F0963091F0913009F0EB
:108D500046C008C09A3379F09F3F09F451C096335A
:108D6000F1F537C08CEC99E036C084ED99E033C062
:108D70008CED99E030C0618170E080E090E0982F48
:108D8000872F762F66272981620F711D811D911D06
:108D9000982F872F762F66272A81620F711D811DDC
:108DA000911D982F872F762F66272B81620F711DBB
:108DB000811D911D28EE33E040E050E00E94386AAA
:108DC00060935D0A70935E0A80935F0A9093600AD5
:108DD00089C088ED99E0BE010E940C3683C0E09105
:108DE000690AF0916A0A309709F47CC080916B0A95
:108DF000981709F077C0892FBE014E2D099572C0D2
:108E00000E94F04482E04ECF0634110588F1809133
:108E10007F03833469F520918A0330918B0340915D
:108E20008C0350918D038091650A9091660AA09100
:108E3000670AB091680A281739074A075B07C1F427
:108E4000E6E7F4E0A801445A5C4FDF0111969181F6
:108E50009D012F5F3F4F8081853321F411968C91C6
:108E6000853071F1F901E90FF11DE417F50768F399
:108E70000E94E5662091610A3091620A4091630A7E
:108E80005091640A205F384D4F4F5F4F26173707C8
:108E90004807590748F02DC084ED99E00E94562FED
:108EA00083E08093580A25C01092580A22C088ECAB
:108EB00099E066E973E00E940C36045A1C4F39CFE2
:108EC00081E00E942E4A0E94E5666093590A7093E1
:108ED0005A0A80935B0A90935C0A8091D409882394
:108EE000F9F2DACFCE0DD11DC017D10708F421CF8A
:108EF00087CFDF91CF911F910F91FF90EF90089551
:108F0000CF93DF9381E08093E4099091C709892F83
:108F100082958F70805D8093C7029F70905D909363
:108F2000C8021092580A0E94E566EB0104C00E9434
:108F30008F4A0E9400468091580A833061F00E9457
:108F4000E5666C1B7D0B6053754728F40E94504A00
:108F5000882389F3ECCF0E946C2E1092E7091092BF
:108F6000E60990E08091580A833009F491E0892F56
:108F7000DF91CF9108950F931F938C01FC0186819F
:108F800060E00E94EA6581E090E00E944C67F80191
:108F9000868161E00E94EA6581E090E00E944C6772
:108FA000F801868160E00E94EA6584E690E00E9414
:108FB0004C671F910F910895CF92DF92EF92FF922D
:108FC0000F931F93CF93DF93D82EC92E282F392FBD
:108FD000C9018C01C0E0D0E0E62EFF24F8018781B2
:108FE00061E00E94AB65B7010C2E02C075956795D4
:108FF0000A94E2F76170F80187810E94EA65219680
:109000000F5F1F4FC830D10549F78D2D9C2D0E9451
:10901000BB47DF91CF911F910F91FF90EF90DF90B1
:10902000CF900895CF92DF92EF92FF920F931F930C
:10903000CF93DF93D82EC92E282F392FC9018C0149
:10904000C0E0D0E0E62EFF24F801878161E00E94B5
:10905000AB65B7010C2E02C0759567950A94E2F7CF
:109060006170F80187810E94EA6521960F5F1F4FAA
:10907000C430D10549F78D2D9C2D0E94BB47DF914F
:10908000CF911F910F91FF90EF90DF90CF900895B7
:109090001F93CF93DF93EC01162F8C81642F0E94D6
:1090A000EA658D818F3F19F060E00E94EA658F8547
:1090B00084FF05C0CE01612F0E94DC470EC0612FE6
:1090C00070E084E0759567958A95E1F7CE010E947E
:1090D0001248CE01612F0E941248DF91CF911F915B
:1090E000089541E00E94484881E090E0089540E002
:1090F0000E9448480895EF92FF920F931F93CF93D9
:10910000DF938C017A016770660F660F660F6064EB
:109110000E947748C0E0D0E0D801ED91FC91D701E2
:10912000AC0FBD1F0190F081E02DC8016C91099535
:109130002196C830D10581F7DF91CF911F910F9112
:10914000FF90EF900895FC0160896E7F608B6860EE
:109150000E9477480895FC016089862F8460808B87
:109160006C60CF010E9477480895DF93CF93CDB70D
:10917000DEB728970FB6F894DEBF0FBECDBF9C01B7
:10918000FE013196A4E2B3E088E00D900192815097
:10919000E1F7F9018389481710F0482F4150E42F77
:1091A000F0E0EE0FFF1FEC0FFD1F8181680F60687C
:1091B000C9010E94774828960FB6F894DEBF0FBE0B
:1091C000CDBFCF91DF91089561E00E94774880ED97
:1091D00097E00E944C670895CF93DF93EC014230F3
:1091E00018F08F8588608F874B8B1C8A222329F08B
:1091F000413019F48F8584608F8780E593EC0E945D
:109200004C678C8160E00E94EA658E8160E00E947C
:10921000EA658D818F3F19F060E00E94EA656F85F5
:1092200064FD1DC0CE0163E00E94124884E991E113
:109230000E944C67CE0163E00E94124884E991E1EC
:109240000E944C67CE0163E00E94124886E990E0DC
:109250000E944C67CE0162E00E94124816C0606214
:10926000CE010E94774884E991E10E944C676F85A6
:109270006062CE010E94774886E990E00E944C67C8
:109280006F856062CE010E9477486F856062CE0173
:109290000E94774884E0888BCE010E94AB48CE01C3
:1092A0000E94E44882E0898BCE0166E00E94774804
:1092B000DF91CF9108956F927F928F92AF92CF926C
:1092C000EF920F931F93DF93CF93CDB7DEB73C019F
:1092D000162F842FF301448325830683E782C086FB
:1092E000A18682869D8593879E8594879F85958795
:1092F0009889968761E00E94AB65F30185818F3F75
:1093000019F061E00E94AB65F301868161E00E9483
:10931000AB65112319F0F301178603C080E1F30157
:109320008787C30160E141E020E00E94EC48CF91D3
:10933000DF911F910F91EF90CF90AF908F907F9022
:109340006F9008958091710A61E00E94EA657894B7
:109350000895FF920F931F93082F162FF42EF89461
:109360008091710A60E00E94EA651F71102B1EBD9A
:109370000DB407FEFDCFFEBC0DB407FEFDCF0E946D
:10938000A2491F910F91FF9008951F93182F282F26
:1093900030E0207630708091720A90E0281739070B
:1093A00099F080EA6FE143E00E94A949412F40769D
:1093B0004093720A50E085E0559547958A95E1F70C
:1093C00080E86FE10E94A9491F9108950F931F93B0
:1093D000182F062F0E94C54980E4612F402F0E945C
:1093E000A9491F910F9108950F931F93182F072FCD
:1093F0000E94E649812F8F5F602F0E94E6491F91EE
:109400000F9108950F931F93182F062FF8948091B2
:10941000710A60E00E94EA65802F8F71812B8EBDFA
:109420000DB407FEFDCF1EBC0DB407FEFDCF07FF38
:1094300004C01EBC0DB407FEFDCF1EB50E94A2499C
:10944000812F1F910F9108951F93182F0E94C549D6
:1094500080E0612F0E94024A1F910895882311F431
:109460001092700A8091700A882341F488E30E9468
:10947000244A682F6E7F88E30E94E64908951F936F
:10948000182F88E30E94244A682F616088E30E94B5
:10949000E649112319F481E08093700A1F91089521
:1094A00084ED61E10E94E64982ED61E00E94E649B7
:1094B0008AEE0E94244A80FDFBCF82ED60E00E948C
:1094C000E64989ED0E94244A90E096958795969505
:1094D0008795817008950F931F93CF93DF93EC01CD
:1094E0008B01F8948091710A60E00E94EA658AE33A
:1094F0008EBD0DB407FEFDCF09C01EBC0DB407FE26
:10950000FDCF8EB5F80181938F0121972097A9F7A0
:109510000E94A249DF91CF911F910F9108950F935F
:109520001F93DF93CF9300D000D000D0CDB7DEB72C
:1095300089E30E94244A882319F400E010E048C01F
:109540006091730A7091740A80E00E94F44986E089
:1095500090E0BE016F5F7F4F0E946B4A89819A81C4
:109560009093740A8093730A2B813C81E0916E0A78
:10957000F0916F0A8D8187FD03C000E010E00EC0FE
:10958000245030408F01015010402017310708F45B
:109590008901C8016CE573E00E946B4AF801E45A46
:1095A000FC4F10826091730A7091740A8CE06130F4
:1095B000780724F08CE06FEF7BE003C061507040CF
:1095C0008CE00E94F44980E86EE140E40E94A949E1
:1095D000C80126960FB6F894DEBF0FBECDBFCF915F
:1095E000DF911F910F9108950F931F93CF93DF93F6
:1095F0008C01EB01F8948091710A60E00E94EA65A9
:109600008AE78EBD0DB407FEFDCF08C088818EBDF0
:109610000DB407FEFDCF2196015010400115110534
:10962000A9F70E94A249DF91CF911F910F91089550
:10963000CF93DF93EC018CE10E94244A81FF0FC09D
:1096400080E86FE140E80E94A94980EA6FE140E8C4
:109650000E94A94980EA6CE142E00E94A94982E0A7
:1096600060E07CE00E94F449BE016050744F86E0E7
:109670000E94F4498AE760E040E00E94A949CE01D7
:109680006CE573E00E94F44A80E86FE148E00E94D4
:10969000A949DF91CF91089584E061E00E94AB6514
:1096A00084E061E00E94EA6585E061E00E94AB65CC
:1096B00087E061E00E94AB6586E060E00E94AB65F8
:1096C00085E061E00E94EA6585E060E00E94EA656D
:1096D00087E060E00E94EA6580E58CBD8DB5816021
:1096E0008DBD08951F93CF93DF93EB01142F9093BB
:1096F0006F0A80936E0A0CB406FC02C00E944C4BA9
:109700001093710A812F61E00E94AB650E94A2490B
:109710008FEF60E04FEF0E94A94962E070E080E0C7
:1097200090E00E94F36680E06DE10E94024A882387
:10973000D1F31092740A1092730A88E060E070E02E
:109740000E94F4498CE060E070E00E94F4498AE0F5
:109750006FEF7BE00E94F44984E060E07CE00E94CF
:10976000F44986E06FEF71E10E94F44980E00E94C5
:109770003F4A88E26FE370E30E94F44980E369EFB7
:1097800077EF0E94F44980EC6DE00E94E64981EC9D
:1097900060E00E94E64980E862EC42E30E94A94949
:1097A00086EC62E17CE00E94F44984EC62E10E9474
:1097B000E6498AEC6AEE75E00E94F44984EE68811D
:1097C0000E94E64985EE69810E94E64982EE6A813F
:1097D0000E94E64983EE6B810E94E64980EE6C812F
:1097E0000E94E64981EE6D810E94E64984ED60E1C8
:1097F0000E94E64986ED60E071E00E94F4498AEE3D
:109800000E94244A80FDFBCF8FE10E94C54980E879
:109810006BE140EC0E94A94980E86FE144E00E94BE
:10982000A94982E70E94244A863008F08F5FDF91C1
:10983000CF911F9108954E960E946E5C0895DF931C
:10984000CF93CDB7DEB76A970FB6F894DEBF0FBEE1
:10985000CDBFFB01242F19821B82BC01625E7F4FAA
:10986000CE010196AF010E94555D6A960FB6F8943D
:10987000DEBF0FBECDBFCF91DF9108954E960E94FF
:10988000A65C0895CF93DF93EC01662331F06E96CA
:10989000D093860CC093850C6E9788A1882321F005
:1098A000CE014E960E949A54CE014E962596BE0148
:1098B0000E94EA51DF91CF910895DF92EF92FF92DB
:1098C0000F931F93DF93CF93CDB7DEB76A970FB691
:1098D000F894DEBF0FBECDBF9C01FB01D42E1982D0
:1098E0001B8280818F3241F48181882329F4C90150
:1098F000642F0E94424C22C08901025E1F4F7E01EC
:109900000894E11CF11CC701B801AF0121E00E94DD
:10991000A65B882391F08B81823078F0D801F70123
:109920008AE101900D928150E1F7DD2021F0109342
:10993000860C0093850C81E001C080E06A960FB62A
:10994000F894DEBF0FBECDBFCF91DF911F910F9175
:10995000FF90EF90DF9008950F931F93CF93DF93C5
:10996000EC010E94E3608823C9F08E010B5F1F4F5A
:10997000C801BE0141E00E948F4D882339F4C8011F
:10998000BE0140E00E948F4D882341F0CE0161E08E
:109990000E94424C882319F081E001C080E0DF91F1
:1099A000CF911F910F9108958FEF9FEFAFEFBFEF12
:1099B00080937A0C90937B0CA0937C0CB0937D0CDD
:1099C00010927E0C08950F931F938C01CB01BA0166
:1099D0006250704080409040F801248130E040E0C7
:1099E00050E00E94386A9B01AC01F80182859385A2
:1099F000A485B585280F391F4A1F5B1FB901CA010D
:109A00001F910F91089580917E0C80FF3DC0409181
:109A10007A0C50917B0C60917C0C70917D0C809144
:109A20007F0C9091800C2AE73AE00E9438608823EE
:109A300069F180917E0C81FF22C08091750A82308D
:109A4000F0F04091760A5091770A6091780A70910F
:109A5000790A80917A0C90917B0CA0917C0CB0914A
:109A60007D0C480F591F6A1F7B1F80917F0C9091BE
:109A7000800C2AE73AE00E943860882339F0809110
:109A80007E0C8E7F80937E0C81E0089580E00895A7
:109A90000E94034D0895DF92EF92FF920F931F9360
:109AA0007B018C01D42E80917A0C90917B0CA0913B
:109AB0007C0CB0917D0C8E159F05A007B107E1F0DD
:109AC0000E94034D882311F1D2FC0CC080917F0CC1
:109AD0009091800CB801A7012AE73AE00E94AF609C
:109AE0008823A1F010927E0CE0927A0CF0927B0C0D
:109AF00000937C0C10937D0C83E0D82280917E0C27
:109B00008D2980937E0C2AE73AE002C020E030E005
:109B1000C9011F910F91FF90EF90DF9008956F9210
:109B20007F928F929F92AF92BF92CF92DF92EF92ED
:109B3000FF920F931F93CF93DF93EC01142F709339
:109B4000800C60937F0C1A8A82E090E0A0E0B0E085
:109B500088839983AA83BB8310927E0C8FEF9FEF3B
:109B6000AFEFBFEF80937A0C90937B0CA0937C0CAB
:109B7000B0937D0C442321F466247724430136C03E
:109B8000453008F0EFC060E070E080E090E040E039
:109B90000E944B4DDC01009709F4E4C0412F50E0D6
:109BA00041505040FA0174E0EE0FFF1F7A95E1F743
:109BB000E80FF91FE254FE4F808190E08F7790709C
:109BC000892B09F0CFC064E0440F551F6A95E1F777
:109BD000A40FB51FAA53BE4F6D907D908D909C90A1
:109BE000611471048104910409F4BCC0C401B3017F
:109BF00040E00E944B4D5C01009709F4B3C0FC01AA
:109C0000838594858050924009F0ACC0F50120898D
:109C1000222309F4A7C0468557854115510509F44B
:109C2000A1C02093750A85858C83198691E060E038
:109C300070E00AC0990F6F5F7F4F6830710509F4BB
:109C400091C089858F5F89878C81891799F7F50184
:109C5000668977896115710519F080E090E005C08B
:109C6000F50164A175A186A197A16093760A70930E
:109C7000770A8093780A9093790A6A01EE24FF2488
:109C8000C60CD71CE81CF91CCE86DF86E88AF98A48
:109C9000F501018912891C8B0B8B30E040E050E00C
:109CA0000E94386A6C0D7D1D8E1D9F1D6D8B7E8BF5
:109CB0008F8B988F35E0000F111F3A95E1F7015017
:109CC0001E4F012F11270695980140E050E0260F06
:109CD000371F481F591F2A873B874C875D87F5012F
:109CE00083899489009721F07C0100E010E005C091
:109CF000F501E0A0F1A002A113A1C401B301621B10
:109D0000730B840B950B6E0D7F1D801F911F0984B3
:109D100004C096958795779567950A94D2F76D83D9
:109D20007E838F839887653FFFE07F07F0E08F0792
:109D3000F0E09F0718F48CE08A8B14C0655F7F4FBA
:109D40008040904010F480E10AC0F50184A595A5FB
:109D5000A6A5B7A58D8B9E8BAF8BB88F80E28A8B23
:109D600081E001C080E0DF91CF911F910F91FF90C2
:109D7000EF90DF90CF90BF90AF909F908F907F90AB
:109D80006F90089542600E944B4D08958F929F926C
:109D9000AF92BF92CF92DF92EF92FF920F931F93F9
:109DA000CF93DF93EC016A017B01480159014230F6
:109DB00051056105710508F44BC08D819E81AF810D
:109DC000B8850196A11DB11D84179507A607B70791
:109DD00008F43EC08A89803129F4252F362F472F79
:109DE00055270BC08032A1F59A01AB0117E05695BB
:109DF0004795379527951A95D1F78E859F85A88920
:109E0000B989280F391F4A1F5B1FCA01B90141E0F8
:109E10000E94C24E9C010097D9F08A89803149F492
:109E2000F601F070EE0FFF1FE20FF31F91828082A8
:109E30000DC0F601EF77F070EE0FFF1FEE0FFF1F62
:109E4000E20FF31F80829182A282B38281E001C07F
:109E500080E0DF91CF911F910F91FF90EF90DF9005
:109E6000CF90BF90AF909F908F900895CF92DF9248
:109E7000EF92FF920F931F93CF93DF93EC017A0140
:109E80008B016901423051056105710508F453C029
:109E90008D819E81AF81B8850196A11DB11D84176A
:109EA0009507A607B70708F446C08A89803129F4C8
:109EB0005527412F302F2F2D0BC08032E1F59A010D
:109EC000AB0167E056954795379527956A95D1F789
:109ED0008E859F85A889B989280F391F4A1F5B1F66
:109EE000CA01B90140E00E94C24E9C01009719F1DD
:109EF0008A89803159F4F701F070EE0FFF1FE20FED
:109F0000F31F80819181A0E0B0E00EC0F701EF77F0
:109F1000F070EE0FFF1FEE0FFF1FE20FF31F8081A7
:109F20009181A281B381BF70F60180839183A28366
:109F3000B38381E001C080E0DF91CF911F910F9149
:109F4000FF90EF90DF90CF9008958F929F92AF9205
:109F5000BF92CF92DF92EF92FF920F931F93DF9306
:109F6000CF9300D000D0CDB7DEB75C016A017B0192
:109F70004E010894811C911CC501B701A6019401F2
:109F80000E94364F8823B1F1C501B701A60100E058
:109F900010E020E030E00E94C64E882359F1F50120
:109FA00080819181A281B381C816D906EA06FB0699
:109FB00020F4C082D182E282F382C980DA80EB8011
:109FC000FC80F5018289803151F4F8EFCF16FFEF64
:109FD000DF06F0E0EF06F0E0FF0670F209C088EF60
:109FE000C8168FEFD8068FEFE8068FE0F80620F24C
:109FF00081E001C080E00F900F900F900F90CF9103
:10A00000DF911F910F91FF90EF90DF90CF90BF9065
:10A01000AF909F908F9008952F923F924F925F92B2
:10A020006F927F928F929F92AF92BF92CF92DF9268
:10A03000EF92FF920F931F93DF93CF93CDB7DEB7CD
:10A0400066970FB6F894DEBF0FBECDBF1C014987DF
:10A050005A876B877C873E872D87DC0115962D916B
:10A060003D914D915C9118972F5F3F4F4F4F5F4F40
:10A070002D833E834F835887ED85FE8500811181B6
:10A0800022813381011511052105310549F048016F
:10A0900059010894811C911CA11CB11C10E006C040
:10A0A000DC018D909D90AD90BC9011E07501640134
:10A0B000442455243201F10185819681A781B08520
:10A0C000481659066A067B0608F09DC02D813E8120
:10A0D0004F8158852C153D054E055F0550F4F2E083
:10A0E0008F2E912CA12CB12CE2E0CE2ED12CE12C84
:10A0F000F12CC101B701A6019E012F5F3F4F0E94C5
:10A10000364F882309F47FC089819A81AB81BC8155
:10A110000097A105B10571F08C149D04AE04BF0435
:10A1200009F010E0460157010894811C911CA11C04
:10A13000B11C16C0D701C6010196A11DB11D8B8BA4
:10A140009C8BAD8BBE8B88199909AA09BB092985FF
:10A150003A854B855C8582179307A407B50759F0AC
:10A160000894411C511C611C711C0894C11CD11C19
:10A17000E11CF11CA0CF112349F08B899C89AD898A
:10A18000BE89F10180839183A283B383C101B701AA
:10A19000A6010FEF1FEF2FEF3FE00E94C64E88236E
:10A1A00099F431C02601370108944108510861082B
:10A1B0007108C101B301A201970186010E94C64E38
:10A1C000882309F1730162018C149D04AE04BF045D
:10A1D00048F3AD85BE854D915D916D917C914115A2
:10A1E00051056105710539F0C101950184010E9495
:10A1F000C64E882341F0ED85FE8580829182A28241
:10A20000B38281E001C080E066960FB6F894DEBFAD
:10A210000FBECDBFCF91DF911F910F91FF90EF90B7
:10A22000DF90CF90BF90AF909F908F907F906F9076
:10A230005F904F903F902F9008958091C10085FDD1
:10A24000FCCF8091C00085FFF8CF6093C60081E00D
:10A2500090E008951092840C1092830C80E393E0B8
:10A260009093820C8093810C08950F931F93CF934A
:10A27000DF93DC01EB018A0180E090E020E2FE0147
:10A28000E80FF91F208301968B309105C1F757E045
:10A2900040E024C0622F2E3219F080E79BE007C017
:10A2A0005A3051F15AE048E018C0321729F1FC0148
:10A2B000019634913323C9F75417F0F02132E0F0BE
:10A2C0002F37D0F4822F81568A3110F4622F6052DA
:10A2D000FE01E40FF11D60834F5F11962C91222344
:10A2E00011F02F32B9F6F801B183A08390E0888194
:10A2F000803219F091E001C090E0892FDF91CF9179
:10A300001F910F910895CF92DF92EF92FF920F93DA
:10A310001F93DF93CF9300D000D0CDB7DEB77C0181
:10A32000FC0186899789A08DB18D89839A83AB833F
:10A33000BC8300E010E06E010894C11CD11C49816F
:10A340005A816B817C81D70114968D919C911597D0
:10A3500096010E94364F882379F1D7011496ED912A
:10A36000FC9115978481080F111DB0E100301B0787
:10A3700018F529813A814B815C818289803131F4E1
:10A38000285F3F4F40405040D0F205C0285F3F4F0C
:10A390004F4F5F40A0F2C801A0E0B0E029E0880F75
:10A3A000991FAA1FBB1F2A95D1F7F701828B938BA8
:10A3B000A48BB58B81E001C080E00F900F900F90CF
:10A3C0000F90CF91DF911F910F91FF90EF90DF9051
:10A3D000CF900895CF93DF93EC01FB018A8188230E
:10A3E000D1F57D836C8382898031C9F582E08A83CF
:10A3F0001E8A1F8A188E198E83899489A0E0B0E086
:10A4000035E0880F991FAA1FBB1F3A95D1F78A8B99
:10A410009B8BAC8BBD8B0FC083E08A83858996892B
:10A42000A789B08D8E8B9F8BA88FB98FCE010E948C
:10A430008351882381F081E089831E821F821886E0
:10A4400019861A861B861C861D861E861F86188AFC
:10A45000198A1B8201C080E0DF91CF91089580327C
:10A46000D1F7DACF6F927F928F929F92AF92BF9285
:10A47000CF92DF92EF92FF920F931F93CF93DF93D0
:10A48000EC017A018B012A81222309F480C08A8998
:10A490009B89AC89BD8984179507A607B70708F47F
:10A4A00076C085C0E114F1040105110551F41E8246
:10A4B0001F82188619861A861B861C861D8681E0D7
:10A4C00067C02A853B854C855D85EC81FD81818552
:10A4D00090E00996215030404040504039014A01F7
:10A4E000082E04C096948794779467940A94D2F7C0
:10A4F0002F5F3F4F4F4F5F4F0894E108F10801096C
:10A5000011095701680104C0D694C794B794A79461
:10A510008A95D2F70894E11CF11C011D111DA614A7
:10A52000B704C804D90428F02115310541055105A7
:10A5300049F48E899F89A88DB98D8E839F83A887C2
:10A54000B98716C0A618B708C808D90811C04E8127
:10A550005F81688579858C819D8194010E94364F49
:10A560000894A108B108C108D108882331F40FC0AC
:10A5700046E0842E912C8C0E9D1EA114B104C104C2
:10A58000D10429F7EA86FB860C871D8798CF80E0E7
:10A59000DF91CF911F910F91FF90EF90DF90CF90BF
:10A5A000BF90AF909F908F907F906F9008952230D2
:10A5B00009F078CFE7CFCF93DF93EC01462F6E857C
:10A5C0007F85888999890E944B4DAC01009719F4C9
:10A5D00020E030E00AC08B81282F30E065E0220FB8
:10A5E000331F6A95E1F7240F351FC901DF91CF9121
:10A5F00008950F931F93CF93DF938C01FC01828109
:10A600008823F1F1818187FF38C0C80161E00E9491
:10A61000DB52EC010097A1F18881853E89F1F801B8
:10A620008281823040F482899389A489B5898C8F94
:10A630009D8FAE8FBF8FF801868997899B8F8A8FF8
:10A6400086899789A08DB18DCD01AA27BB279D8BC7
:10A650008C8BE091870CF091880C309751F0BE0103
:10A660006A5E7F4FCE0148960995888D998D9B8BA8
:10A670008A8BF80181818F7781830E94034D04C00A
:10A6800081E0F801808380E0DF91CF911F910F91ED
:10A6900008956F927F928F929F92AF92BF92CF92C6
:10A6A000DF92EF92FF920F931F93DF93CF9300D02F
:10A6B00000D0CDB7DEB77C015A016B01DC011296E8
:10A6C0008C911297813009F091C011968C9181FF85
:10A6D0008DC0A0C00097A105B10511F481E087C02D
:10A6E000F7016284738484849584C701B601A5014F
:10A6F0000E943252882309F479C0D70114968D91B3
:10A700009C911597A114B104C104D10489F4569603
:10A710004D915D916D917C9159970E94A54F882331
:10A7200009F464C0F701168A178A108E118E44C08E
:10A73000D70116964D915D916D917C9119979E016F
:10A740002F5F3F4F0E94364F882309F44FC0D70137
:10A750001496ED91FC91159749815A816B817C810A
:10A760008289803149F4483FBFEF5B07B0E06B0757
:10A77000B0E07B0748F020C0483F8FEF58078FEFCD
:10A7800068078FE07807C0F4CF010E94A54F8823A7
:10A7900069F1D70116964D915D916D917C91199754
:10A7A00014968D919C9115970FEF1FEF2FEF3FE0BF
:10A7B0000E94C64E8823D1F0F701A28AB38AC48AC8
:10A7C000D58A818180688183C7010E94F9528823DC
:10A7D00069F0B601A5016A147B048C049D0410F491
:10A7E000B401A301C7010E94325201C080E00F9062
:10A7F0000F900F900F90CF91DF911F910F91FF90CD
:10A80000EF90DF90CF90BF90AF909F908F907F9010
:10A810006F900895F70182899389A489B589841777
:10A820009507A607B70708F055CFE0CF1F93CF9342
:10A83000DF93EC01142F262F30E0F90185E0EE0FB5
:10A84000FF1F8A95E1F7E658F54F8385817121F066
:10A85000842F827109F064C080917A0C90917B0CF6
:10A86000A0917C0CB0917D0C8E879F87A88BB98BB3
:10A870006B83F901B5E0EE0FFF1FBA95E1F7E658DB
:10A88000F54F2489358940E050E0A901332722277C
:10A890002E8B3F8B488F598F828D938DA0E0B0E037
:10A8A000282B392B4A2B5B2B2E8B3F8B488F598FB4
:10A8B000838590E088719070009751F4848D958D18
:10A8C000A68DB78D8A8B9B8BAC8BBD8B81E008C02E
:10A8D000409731F5CE010E948351882309F184E02D
:10A8E0008A83812F8F7089831E821F821886198622
:10A8F0001A861B861C861D8614FF18C0CE0140E0F8
:10A9000050E060E070E00E944953882379F408C069
:10A910004A895B896C897D89CE010E94325202C0CE
:10A920001A8280E0DF91CF911F91089515FDF0CF3D
:10A9300081E0F8CF0F931F938C010E94F952F80128
:10A9400012821F910F910895CF93DF93EC0140E0A5
:10A9500050E060E070E00E944953882369F0CE0126
:10A9600061E00E94DB52FC01009731F085EE8083AC
:10A970001A820E94034D01C080E0DF91CF910895BB
:10A980002F923F924F925F927F928F929F92AF92BF
:10A99000BF92CF92DF92EF92FF920F931F93DF93BC
:10A9A000CF93CDB7DEB728970FB6F894DEBF0FBEB2
:10A9B000CDBF98878F835E834D83DC0112968C9187
:10A9C0001297882309F41EC111968C9180FF1AC139
:10A9D00034C1F501EE19FF09FE83ED837A836983A3
:10A9E0008F81988506969C838B834D805E8003C102
:10A9F000AF81B8851A962D913D914D915C911D972F
:10AA00008FEF282E81E0382E222233221496ED91EA
:10AA1000FC91159759016A0109E0D694C794B7943F
:10AA2000A7940A95D1F774807A947A2012968C9123
:10AA3000823049F4E588F6880789108DEA0CFB1C02
:10AA40000C1D1D1D35C02114310411F5772001F5B1
:10AA5000211531054105510559F4EF81F8858689A5
:10AA60009789A08DB18D86839783A087B18710C009
:10AA7000AF81B88516964D915D916D917C91199736
:10AA8000CF012B813C810E94364F882309F4BAC044
:10AA9000EF81F88546815781608571858481958134
:10AAA0000E94E34C7B018C01E70CF11C011D111D80
:10AAB0002114310499F4F0E04F16F2E05F0670F0D3
:10AAC00020917A0C30917B0C40917C0C50917D0C44
:10AAD000E216F3060407150709F0CFC0C801B70155
:10AAE00040E00E944B4D009709F48CC040E052E0DA
:10AAF0004219530942014415550508F44A019C01C5
:10AB0000220D331D89819A81B901A4010E949C06FE
:10AB100059C080917F0C9091800CB801A7012981C8
:10AB20003A810E94AF60882309F46CC0812C12E046
:10AB3000912E48C0D52CD694AF81B88512968C91B1
:10AB40001297823049F01496ED91FC91159784810B
:10AB500087198D1508F4D82EE216F3060407150799
:10AB600070F02D0D311D411D511DE216F306040735
:10AB7000150728F40E94034D882309F443C08091EF
:10AB80007F0C9091800CB801A7010E948C608823F3
:10AB9000C9F109811A81FF2408C0B8010E948A5FA7
:10ABA00000501E4F882371F1F39480917F0C909197
:10ABB000800CFD1490F30E947260882319F19D2C83
:10ABC000990C8824E981FA81E80DF91DFA83E9835B
:10ABD000940140E050E0EF81F88582859385A4855B
:10ABE000B585820F931FA41FB51F82879387A48703
:10ABF000B587481859084114510409F0F9CE4D8120
:10AC00005E8102C04FEF5FEFCA0128960FB6F8943D
:10AC1000DEBF0FBECDBFCF91DF911F910F91FF908F
:10AC2000EF90DF90CF90BF90AF909F908F907F90EC
:10AC30005F904F903F902F900895AF81B8855296C6
:10AC4000AD90BD90CD90DC9055971A96ED90FD900B
:10AC50000D911C911D97ED81FE819F0140E050E018
:10AC6000D601C5018E199F09A00BB10B2817390712
:10AC70004A075B0708F0ADCEB1CEF0E04F16F4E026
:10AC80005F0608F057CF45CFDF93CF930F92CDB734
:10AC9000DEB7BE016F5F7F4F41E050E00E94C054BD
:10ACA000019719F02FEF3FEF03C08981282F30E083
:10ACB000C9010F90CF91DF910895EF92FF920F930A
:10ACC0001F93CF93DF93EC018A81823038F1EA84BD
:10ACD000FB840C851D85CE010E94445697FD1EC045
:10ACE0008A859B85AC85BD854F96A11DB11D8A8740
:10ACF0009B87AC87BD8725E016950795F794E79469
:10AD00002A95D1F72E2D30E02F70307095E0220F6C
:10AD1000331F9A95E1F72658354F02C020E030E006
:10AD2000C901DF91CF911F910F91FF90EF9008958E
:10AD3000CF93DF93EC018A81843071F5CE0140E03E
:10AD400050E060E070E00E94325210C0CE010E94DC
:10AD50005D56FC01009701F180818823A1F0853EBA
:10AD600029F08E3219F0838583FF16C02A853B8532
:10AD70004C855D858A899B89AC89BD8928173907EF
:10AD80004A075B0718F381E08A838981826089839F
:10AD9000CE010E94A45401C080E0DF91CF910895BC
:10ADA000DF92EF92FF920F931F93CF93DF938C016B
:10ADB000EB017A01D22E8C819D81F80195838483E9
:10ADC0008281882329F56115710559F521C0A701F4
:10ADD00065E0440F551F6A95E1F760E070E0CE0131
:10ADE0000E9432528823A1F0CE010E945D56FC01E0
:10ADF000009771F08081882359F0853E49F08E32AA
:10AE000039F06E2D6F70C8014D2D0E94165401C08F
:10AE100080E0DF91CF911F910F91FF90EF90DF9035
:10AE2000089527FFD4CFF4CFAF92BF92CF92DF9295
:10AE3000EF92FF920F931F93DF93CF93CDB7DEB7BF
:10AE40006A970FB6F894DEBF0FBECDBF8C01198292
:10AE50001B8240E050E060E070E00E9432525E01F0
:10AE60000894A11CB11C52C0C8010E945D56FC018F
:10AE7000009709F466C08081882309F456C0853E96
:10AE800009F444C08E3209F441C0838583FD3EC07D
:10AE9000A7019601F5E05695479537952795FA95C0
:10AEA000D1F77901C501B801A90121E00E94D0566E
:10AEB000882309F446C08B81843021F4C5010E94A7
:10AEC000145706C08A8182608A83C5010E94A454F7
:10AED0008823B9F10894E11CF11CA70160E070E03F
:10AEE000E5E0440F551F661F771FEA95D1F7F8017B
:10AEF00082859385A485B58584179507A607B7072E
:10AF000029F0C8010E9432528823D9F0F801C28486
:10AF1000D384E484F58482899389A489B589C81689
:10AF2000D906EA06FB0608F49FCFF8018281825019
:10AF3000823028F0C8010E949856882319F081E0D9
:10AF400001C080E06A960FB6F894DEBF0FBECDBF99
:10AF5000CF91DF911F910F91FF90EF90DF90CF90F5
:10AF6000BF90AF9008952F923F924F925F926F9251
:10AF70007F928F929F92AF92BF92CF92DF92EF9289
:10AF8000FF920F931F93DF93CF930F92CDB7DEB74E
:10AF90002C015B013A01490100E010E0EE24EA9443
:10AFA000FE2C1E010894211C311C13C00A0D1B1D10
:10AFB000F80160838114910419F46A3049F41EC0C9
:10AFC000772767FD7095C4010E94B7060097B1F41A
:10AFD000860168010894C11CD11CC614D70444F52D
:10AFE000C201B10141E050E00E94C0547C018130B7
:10AFF0009105F1F469816D30C9F6EBCF8601A00EA1
:10B00000B11EF5011082C8010F90CF91DF911F9101
:10B010000F91FF90EF90DF90CF90BF90AF909F90F7
:10B020008F907F906F905F904F903F902F900895FA
:10B03000F7FEE5CF0FEF1FEFE6CFCF93DF93EC01E5
:10B040009C012A5F3F4F8C819D8141E050E060E090
:10B0500070E00E940C508823A1F08E899F89A88DF2
:10B06000B98D0097A105B10559F48E819F81A885FE
:10B07000B9858E8B9F8BA88FB98F898180688983D2
:10B0800081E0DF91CF9108953F924F925F926F924E
:10B090007F928F929F92AF92BF92CF92DF92EF9268
:10B0A000FF920F931F93DF93CF93CDB7DEB72A970D
:10B0B0000FB6F894DEBF0FBECDBF4C01162F072F81
:10B0C0005A874987DC0112968C911297813009F0DA
:10B0D000B0C111968C9181FFACC1C9C1F401428904
:10B0E00053896489758982859385A485B58584177C
:10B0F0009507A607B70731F0C4010E943252882392
:10B1000009F497C1812F902F9C0138872F832985BF
:10B110003A853E832D8351C1D4011496ED91FC9163
:10B120001597DA01C90119E0B695A7959795879506
:10B130001A95D1F7F480FA94F82289011170FF2052
:10B1400009F052C00115110509F04EC0D401169640
:10B150004D915D916D917C91199741155105610556
:10B16000710571F1CF019E012F5F3F4F0E94364F55
:10B17000882309F45EC129813A814B815C81D40125
:10B180001496ED91FC9115978289803149F4283FFE
:10B19000BFEF3B07B0E04B07B0E05B0748F019C0DA
:10B1A000283FEFEF3E07EFEF4E07EFE05E0788F432
:10B1B000D40116962D933D934D935C93199714C02B
:10B1C000F40186899789A08DB18D0097A105B105FD
:10B1D00031F4C4010E941D58882331F42AC1F401BE
:10B1E00086839783A087B187D40116964D915D9190
:10B1F0006D917C91199714968D919C9115970E9451
:10B20000E34C5B016C01AF0CB11CC11CD11C0115DE
:10B210001105C9F4ED81FE81E050F240D8F5D4016A
:10B220001A962D913D914D915C911D9752968D915D
:10B230009D910D90BC91A02D281739074A075B07F7
:10B2400010F045E001C041E0C601B5010E944B4D40
:10B25000009709F4EEC040E052E0401B510B4D80D6
:10B260005E804415550508F42A019C01200F311F0A
:10B27000C9016F817885A2010E949C06040D151DED
:10B280000050124009F07DC00E94484D882309F00B
:10B2900078C0CFC0ED81FE81E050F44000F5809190
:10B2A0007A0C90917B0CA0917C0CB0917D0C8A154E
:10B2B0009B05AC05BD0511F40E94D44C80917F0C18
:10B2C0009091800CB601A5012F8138850E943860CD
:10B2D000882309F4AEC0412CF2E05F2E52C0D401A5
:10B2E0001496ED91FC91159784818F193E803694C8
:10B2F000831508F4382E032D10E020E030E0809113
:10B300007F0C9091800CB601A5010E94F05F88230C
:10B3100009F48FC06F8078848601750122C0809106
:10B320007A0C90917B0CA0917C0CB0917D0CE8166E
:10B33000F9060A071B0711F40E94D44C80917F0C78
:10B340009091800CB3010E94645FE0E0F2E06E0E29
:10B350007F1E0894E11CF11C011D111D882309F4B6
:10B3600068C08E2D8A198315D0F280917F0C909140
:10B37000800C0E943E5F882309F45BC0532C550C5F
:10B380004424920140E050E0F40182859385A48535
:10B39000B585820F931FA41FB51F82879387A4874B
:10B3A000B5872F813885240D351D38872F838D81F2
:10B3B0009E81841995099E838D83D4011A962D91BF
:10B3C0003D914D915C911D97ED81FE81EF2B09F030
:10B3D000A3CE52968D919D910D90BC91A02D821778
:10B3E0009307A407B50740F4D40152962D933D93DB
:10B3F0004D935C9355970BC08091870C9091880C6E
:10B40000892B59F0E985FA85EF2B39F0D401119693
:10B410008C911197806811968C93F401818183FF40
:10B4200005C0C4010E94F952882319F049855A8544
:10B4300005C081E0D4018C934FEF5FEFCA012A96DB
:10B440000FB6F894DEBF0FBECDBFCF91DF911F9135
:10B450000F91FF90EF90DF90CF90BF90AF909F90B3
:10B460008F907F906F905F904F903F90089582FDF6
:10B4700035CE48CE9F92AF92BF92CF92DF92EF929D
:10B48000FF920F931F93CF93DF938C01FC0182896E
:10B490009389A489B589805E9F4FAF41B04008F081
:10B4A0005CC0C8010E941D58882309F456C0D80109
:10B4B00016964D915D916D917C91199714968D9191
:10B4C0009C9115970E94E34C5B016C0145E00E9442
:10B4D0004B4DEC01009709F442C080E092E0FE0180
:10B4E0009C01119221503040E1F79C2EED2EFF245B
:10B4F000F39411C0B601A5014F0D511D611D711DC1
:10B5000080917F0C9091800C292D3E2D0E943860F7
:10B51000882319F1F394D8011496ED91FC911597B5
:10B520002481F21638F330E040E050E089E0220F49
:10B53000331F441F551F8A95D1F752968D919D91C7
:10B540000D90BC91A02D820F931FA41FB51FF80171
:10B55000828B938BA48BB58B02C0C0E0D0E0CE0170
:10B56000DF91CF911F910F91FF90EF90DF90CF90DF
:10B57000BF90AF909F9008953F924F925F926F92CD
:10B580007F928F929F92AF92BF92CF92DF92EF9273
:10B59000FF920F931F93CF93DF934C01EB01442E47
:10B5A000352E522E8C819D81F40195838483CB01AD
:10B5B00040E050E060E070E00E94325277244FC0DB
:10B5C000CE010E94445697FDABC08A859B85AC8511
:10B5D000BD8581509E4FAF4FBF4F8A879B87AC87F9
:10B5E000BD87A0907A0CB0907B0CC0907C0CD09062
:10B5F0007D0C2AE7E22E2AE0F22E00E010E0602E19
:10B60000F7018081882311F0853E79F4772041F499
:10B61000F401A686B786C08AD18A638277247394A0
:10B62000F7018081882391F428C0B80195E0660F66
:10B63000771F9A95E1F76658754F842D932D4BE04F
:10B6400050E00E948F06009709F47DC00F5F1F4FE6
:10B6500080E290E0E80EF91E0031110581F62A859E
:10B660003B854C855D858A899B89AC89BD89281776
:10B6700039074A075B0708F4A3CF56FE51C051FEB5
:10B680004FC0772051F0F4016380C40161E00E9453
:10B69000DB52EC01009761F443C08A81823009F4E7
:10B6A0003FC0CE010E943A5A0097D1F1EC016624C6
:10B6B00080E2FE0111928A95E9F7DE01242D332DF7
:10B6C000C901FC018BE001900D928150E1F7E091FE
:10B6D000870CF091880C309739F0BE01625F7F4F84
:10B6E000CE014096099508C081E298E2998B888B3B
:10B6F00080E098E09F878E87888999899B8B8A8BC9
:10B70000998F888F8E859F859F8B8E8B0E94034D8E
:10B71000882331F0C401662D452D0E94165401C0C6
:10B7200080E0DF91CF911F910F91FF90EF90DF901C
:10B73000CF90BF90AF909F908F907F906F905F90D1
:10B740004F903F90089557FEE5CFEACF2F923F925A
:10B750004F925F926F927F928F929F92AF92BF9221
:10B76000CF92DF92EF92FF920F931F93DF93CF93CD
:10B77000CDB7DEB7C454D0400FB6F894DEBF0FBECD
:10B78000CDBF3C016B01DE01A05CBF4F11965C9305
:10B790004E9323962FAF23976115710509F483C04B
:10B7A0001E8618A6FC018281882309F07CC01C86B5
:10B7B0001EA2FA0180818F32F1F086015CE0E52E55
:10B7C000F12CEC0EFD1E40E4A42EB12CAC0EBD1EDF
:10B7D0004E010894811C911C2596FFAEEEAE259774
:10B7E00036E2232E312C2C0E3D1E270124C011964B
:10B7F000B183A08301C0FD01A081B1818C918F3202
:10B80000B1F3D60112968C91129782508230A8F231
:10B810008E010A5D1F4F14966D917C911597C8019A
:10B820000E94EA51882351F63EC0342D252D870110
:10B83000832F922F7C01F50180819181B401A501B4
:10B840000E943551882329F42EC03196D501ED93FD
:10B85000FC93D501ED91FC9180818F32B1F3882367
:10B86000C9F0C701B801A40121E00E94BC5A882395
:10B87000D1F00C151D0519F0C8010E949A542596A7
:10B88000EEADFFAD2597EE16FF0679F6C101322D1C
:10B89000292FCDCFC301B801A40123962FAD239743
:10B8A0000E94BC5A01C080E0CC5BDF4F0FB6F89419
:10B8B000DEBF0FBECDBFCF91DF911F910F91FF90E3
:10B8C000EF90DF90CF90BF90AF909F908F907F9040
:10B8D0006F905F904F903F902F9008950F931F931C
:10B8E000DF93CF93CDB7DEB76A970FB6F894DEBF7C
:10B8F0000FBECDBF9C01AB0119821B828E010F5F71
:10B900001F4FC801B90122E00E94A65B882319F0ED
:10B91000C8010E94A4546A960FB6F894DEBF0FBE09
:10B92000CDBFCF91DF911F910F910895FB01242F7F
:10B930006091850C7091860CAF010E94A65B089502
:10B94000FC01128210820E94965C0895DF93CF93CF
:10B95000CDB7DEB76A970FB6F894DEBF0FBECDBF86
:10B960009C01AB0119821B82CE010196B90121E035
:10B970000E94A65B6A960FB6F894DEBF0FBECDBFDD
:10B98000CF91DF910895EF92FF920F931F93DF9372
:10B99000CF93CDB7DEB7A0970FB6F894DEBF0FBE3A
:10B9A000CDBF8C017B01FB018281823008F46FC026
:10B9B000C80123EC0E94BC5A882309F468C081E0C6
:10B9C000F801818384E08283C8010E943A5A892B5E
:10B9D00009F45DC0C8010E94F952882309F457C0D8
:10B9E000C80161E00E94DB52FC01009709F44FC0DE
:10B9F00080E18387DE01119680E201900D928150F3
:10BA0000E1F78EE28983FE01329620E2CE010C96A8
:10BA10002193E817F907E1F7F80146895789608D06
:10BA2000718D848195810E94E34C41E00E944B4DD1
:10BA30009C01009761F1DC01FE01319680E20190EA
:10BA40000D928150E1F78EE28A83F7018281825064
:10BA5000823028F41C8E1B8E1E8A1D8A0CC0F701B2
:10BA600086899789A08DB18D9C8F8B8FCD01AA2758
:10BA7000BB279E8B8D8BD9019096FE01319680E27B
:10BA800001900D928150E1F70E94034D01C080E0CA
:10BA9000A0960FB6F894DEBF0FBECDBFCF91DF9159
:10BAA0001F910F91FF90EF9008952F923F924F9228
:10BAB0005F926F927F928F929F92AF92BF92CF923E
:10BAC000DF92EF92FF920F931F93DF93CF93CDB747
:10BAD000DEB7C454D0400FB6F894DEBF0FBECDBF62
:10BAE0003C016B01DE01A05CBF4F11965C934E934D
:10BAF00023962FAF23976115710509F487C01E8621
:10BB000018A6FC018281882309F080C09AC08601B2
:10BB1000FCE0EF2EF12CEC0EFD1EE0E4AE2EB12C7D
:10BB2000AC0EBD1E4E010894811C911C2596FFAEE3
:10BB3000EEAE259776E2272E312C2C0E3D1E2701E6
:10BB400024C01196B183A08301C0FD01A081B18101
:10BB50008C918F32B1F3D60112968C91129782504C
:10BB60008230A8F28E010A5D1F4F14966D917C9170
:10BB70001597C8010E94EA51882351F647C0342D19
:10BB8000252D8701832F922F7C01F50180819181E2
:10BB9000B401A5010E943551882329F437C031969C
:10BBA000D501ED93FC93D501ED91FC9180818F320D
:10BBB000B1F3882329F1C701B801A40121E00E9453
:10BBC000BC5A882361F42396BFAD2397BB23F1F0C1
:10BBD000C701B801A4010E94C35C8823B9F00C1509
:10BBE0001D0519F0C8010E949A542596EEADFFADCF
:10BBF0002597EE16FF0619F6C101322D292FC1CF68
:10BC0000C301B801A4010E94C35C01C080E0CC5B09
:10BC1000DF4F0FB6F894DEBF0FBECDBFCF91DF91DF
:10BC20001F910F91FF90EF90DF90CF90BF90AF905A
:10BC30009F908F907F906F905F904F903F902F904C
:10BC400008951C861EA2ED91FC91119780818F3280
:10BC500009F05DCF7ACF40E082E002C0880F4F5FED
:10BC6000861710F44630D1F7242F30E0C90195959E
:10BC7000879580658CBD40FF02C080E004C080E0F5
:10BC8000463009F081E08DBD089584E061E00E94B6
:10BC9000EA6584E061E00E94AB6586E060E00E94B6
:10BCA000AB6585E061E00E94AB6587E061E00E94E2
:10BCB000AB650895FF920F931F93CF93DF938B0192
:10BCC0000E94E566EB01FF24FA9409C00E94E56634
:10BCD0006C1B7D0B6017710710F080E008C0FEBC84
:10BCE0000DB407FEFDCF8EB58F3F81F781E0DF9168
:10BCF000CF911F910F91FF900895FC01808161E029
:10BD00000E94EA658FEF8EBD0DB407FEFDCF08954A
:10BD1000CF93DF93EC01DA016EBD0DB407FEFDCFCA
:10BD20008C918EBD1196EC91119782E090E00DB44C
:10BD300007FEFDCFEEBD22E08030920731F0FD011D
:10BD4000E80FF91FE0810196F2CF0DB407FEFDCF99
:10BD50008FEF8EBD0DB407FEFDCF8FEF8EBD0DB4FE
:10BD600007FEFDCF8FEF8EBD0DB407FEFDCF8EB564
:10BD70008B838F71853011F481E006C083E1898364
:10BD8000CE010E947D5E80E0DF91CF910895BF9249
:10BD9000CF92DF92EF92FF920F931F93CF93DF9397
:10BDA000EC016B017A010E94E5668B01BB24BA9419
:10BDB00009C00E94E566601B710B6D52714010F066
:10BDC00081E10BC0BEBC0DB407FEFDCF8EB58B83E9
:10BDD0008F3F79F38E3F39F08FE08983CE010E9447
:10BDE0007D5E80E030C0D7011197EF28D9F08FEF4A
:10BDF0008EBD20E030E09FEF0BC00DB407FEFDCFFD
:10BE00008EB59EBDF601E20FF31F80832F5F3F4F7B
:10BE10002A173B0790F30DB407FEFDCF8EB5AC0D8E
:10BE2000BD1D8C931B828FEF8EBD0DB407FEFDCF21
:10BE30008EB58FEF8EBD0DB407FEFDCF8EB5CE0152
:10BE40000E947D5E81E0DF91CF911F910F91FF9065
:10BE5000EF90DF90CF90BF9008950F931F938C01C8
:10BE600089E89CE0F80162810E942B5EF8018081E4
:10BE700060E00E94EA651F910F910895CF93DF93D0
:10BE8000EC010E942D5FCE0168E572E00E945A5ECF
:10BE9000882389F08DEF8EBD0DB407FEFDCFCE0156
:10BEA00068E572E00E945A5E882329F0CE010E9464
:10BEB0007D5E81E006C082E18983CE010E947D5EC5
:10BEC00080E0DF91CF9108950F931F93CF93DF937D
:10BED000EC018B010E942D5FCE0168E572E00E94AB
:10BEE0005A5E882361F0CE016CEFA8010E94885E43
:10BEF000882329F0CE010E947D5E81E006C085E1A5
:10BF00008983CE010E947D5E80E0DF91CF911F91F9
:10BF10000F910895EF92FF920F931F938C017B0175
:10BF20000E942D5FC801B70140E052E00E94C75E49
:10BF30001F910F91FF90EF900895FF920F931F9321
:10BF4000DF93CF9300D000D0CDB7DEB78C01F62EB3
:10BF500029833A834B835C830E942D5FC80168E587
:10BF600072E00E945A5E8F2D80648EBD0DB407FE74
:10BF7000FDCFFE0131969E012350304083818EBD5E
:10BF80000DB407FEFDCF3197E217F307B9F7FF2095
:10BF900011F087E801C085E98EBD0DB407FEFDCF25
:10BFA0008CE0F81631F48FEF8EBD0DB407FEFDCF97
:10BFB0008EB590E02FEF2EBD0DB407FEFDCF8EB5F0
:10BFC00087FF02C09150B9F7F80183830F900F905B
:10BFD0000F900F90CF91DF911F910F91FF900895D7
:10BFE000AF92BF92CF92DF92EF92FF920F931F9387
:10BFF000CF93DF93EC015A016B017801890167E36C
:10C0000020E030E040E050E00E949D5FCE0167E11B
:10C01000A80197010E949D5F882311F089E013C059
:10C020008C81833039F089E0AA0CBB1CCC1CDD1C50
:10C030008A95D1F7CE0169E1A60195010E949D5F25
:10C04000882339F087E08983CE010E947D5E80E0FD
:10C0500004C0CE010E947D5E81E0DF91CF911F91EF
:10C060000F91FF90EF90DF90CF90BF90AF90089529
:10C07000CF92DF92EF92FF920F931F93CF93DF93B4
:10C08000EC017A018B0169018C81833039F099E0F0
:10C09000EE0CFF1C001F111F9A95D1F7CE0168E12D
:10C0A000A80197010E949D5F882319F086E089838B
:10C0B0000CC0CE016EEFA6010E94885E882329F095
:10C0C000CE010E947D5E81E004C0CE010E947D5EB3
:10C0D00080E0DF91CF911F910F91FF90EF90DF9063
:10C0E000CF900895CF93DF93EC016CE020E030E037
:10C0F00040E050E00E949D5F882339F083E089830F
:10C10000CE010E947D5E80E004C0CE010E947D5E73
:10C1100081E0DF91CF910895CF93DF93EC019A01F5
:10C12000AB018C81833039F069E0220F331F441F4B
:10C13000551F6A95D1F7CE0162E10E949D5F882369
:10C1400039F085E08983CE010E947D5E80E004C0E5
:10C15000CE010E947D5E81E0DF91CF910895CF9264
:10C16000DF92EF92FF920F931F93CF93DF93EC0137
:10C170007A018B0169018C81833039F0B9E0EE0CD2
:10C18000FF1C001F111FBA95D1F7CE0161E1A80174
:10C1900097010E949D5F882339F084E08983CE0156
:10C1A0000E947D5E80E006C0CE01B60140E052E014
:10C1B0000E94C75EDF91CF911F910F91FF90EF908A
:10C1C000DF90CF900895BF92CF92DF92EF92FF92CF
:10C1D0000F931F93CF93DF93EC01B42E1C8219822F
:10C1E00068830E94E5666B01888161E00E94AB650F
:10C1F000888161E00E94EA6589E89CE00E94455ED2
:10C2000080E48A8389E89CE060E40E942B5E80E001
:10C210009FEF9EBD0DB407FEFDCF8F5F8A30C9F73B
:10C2200009C00E94E5666C197D09615D774010F0D8
:10C2300081E063C0CE0160E020E030E040E050E00B
:10C240000E949D5F813069F71FEFCE0168E02AEA06
:10C2500031E040E050E00E949D5F853011F481E0C4
:10C260000DC080E01EBD0DB407FEFDCF9EB58F5FF3
:10C270008430C1F79B839A3A31F482E08C838C81BD
:10C28000823051F40DC00E94E5666C197D09615D34
:10C290007740D8F282E031C0EE24FF2487010FC03E
:10C2A000E12CF12C012D80E4182F09C00E94E566D5
:10C2B0006C197D09615D774010F08AE01EC0CE01E7
:10C2C00067E320E030E040E050E00E949D5FCE0157
:10C2D00069E2A80197010E949D5F882339F78C814C
:10C2E000823031F5CE016AE320E030E040E050E0FA
:10C2F0000E949D5F882339F088E08983CE010E94E7
:10C300007D5E80E01AC08FEF8EBD0DB407FEFDCFBD
:10C310008EB5807C803C11F483E08C8380E09FEFBD
:10C320009EBD0DB407FEFDCF2EB58F5F8330C1F7E4
:10C33000CE010E947D5EBA8281E0DF91CF911F9194
:10C340000F91FF90EF90DF90CF90BF900895DB01A9
:10C350000D900020E9F71197A61BB70B0496AD01CD
:10C360000E9444580895DF93CF930F92CDB7DEB764
:10C3700069830496BE016F5F7F4F41E050E00E94E9
:10C38000445820E030E0019711F421E030E0C90189
:10C390000F90CF91DF9108950F931F938C01049616
:10C3A0000E94A05CF8011382128288E393E09183DB
:10C3B00080831F910F91089581E08093CF0C60934B
:10C3C000AC0C1092CD0C1092CE0C08952091AB0CB9
:10C3D00030E08091AA0C281B3109C90108954091D1
:10C3E000AA0C8091AB0C481718F02FEF3FEF0AC052
:10C3F000E42FF0E0E657F34F8081282F30E04F5FC5
:10C400004093AA0CC9010895E091AA0C8091AB0C4D
:10C41000E81718F0EFEFFFEF06C0F0E0E657F34F34
:10C420008081E82FF0E0CF01089508951092D30C99
:10C430001092D20C88EE93E0A0E0B0E08093D40C90
:10C440009093D50CA093D60CB093D70C80E493E0D6
:10C450009093D10C8093D00C0895CF92DF92EF92FD
:10C46000FF920F931F93CF93DF937C016B018A019F
:10C470008091CF0C8823A1F0C0E0D0E00DC0D7019F
:10C48000ED91FC91D601AC0FBD1F0190F081E02D24
:10C49000C7016C9109952196C017D10780F304C09C
:10C4A000CB01642F0E945F63C801DF91CF911F9180
:10C4B0000F91FF90EF90DF90CF900895DF93CF938F
:10C4C0000F92CDB7DEB7FC0169838091CF0C882332
:10C4D000C9F08091CE0C803238F081E090E09383F7
:10C4E000828320E030E015C08091CD0CE82FF0E091
:10C4F000E355F34F998190838F5F8093CD0C8093A8
:10C50000CE0C05C0CE01019661E00E945F6321E080
:10C5100030E0C9010F90CF91DF9108950F93062F5E
:10C520008091AC0C6DEA7CE04091CE0C21E00E9441
:10C530000A631092CD0C1092CE0C1092CF0C0F917A
:10C54000089561E00E948E620895413208F040E251
:10C55000862F6AE87CE00E94C1621092AA0C809348
:10C56000AB0C089521E00E94A56208951092AA0CD8
:10C570001092AB0C1092CD0C1092CE0C0E940B6559
:10C580000895382F413210F040E042C08091DC0C19
:10C590008823E1F791E09093DC0C2093DE0C8FEF81
:10C5A0008093490D1092040D41504093050D4F5F4B
:10C5B0009093DD0C8091DD0C330F832B8093DD0C89
:10C5C0008091DF0C813041F41092DF0C8091DD0C02
:10C5D0008093BB0085EC01C085EE8093BC00809108
:10C5E000DC0C8130E1F38091040D841710F440914C
:10C5F000040D20E030E00AC0FB01E20FF31FD90177
:10C60000AC51B34F8C9180832F5F3F4F2417A0F321
:10C61000842F08950F931F93582F122F413210F03B
:10C6200081E04AC08091DC0C8823E1F782E08093AE
:10C63000DC0C0093DE0C8FEF8093490D1092040DFB
:10C640004093050DA4EEBCE0FB0102C081918D93E7
:10C650008E2F861B8417D0F31092DD0C8091DD0C99
:10C66000550F852B8093DD0C8091DF0C813041F4D8
:10C670001092DF0C8091DD0C8093BB0085EC01C033
:10C6800085EE8093BC00112321F08091DC0C823078
:10C69000E1F38091490D8F3F11F480E00DC080914E
:10C6A000490D803211F482E007C08091490D80333A
:10C6B00011F084E001C083E01F910F910895482F8D
:10C6C000613210F081E008958091DC0C843011F02B
:10C6D00082E008956093270DA6E0BDE0842F9C01C1
:10C6E000F90102C081918D938E2F841B8617D0F3A0
:10C6F00080E008951F920F920FB60F9211242F938E
:10C700003F934F935F936F937F938F939F93AF93D9
:10C71000BF93EF93FF938091B90090E0887F907072
:10C720008036910509F4F2C081369105CCF5883246
:10C73000910509F47BC089329105B4F480319105EB
:10C7400009F46FC0813191053CF4009709F447C1A9
:10C75000089709F04FC165C08831910509F466C09A
:10C76000809709F047C182C08034910509F4A4C0C4
:10C770008134910544F48033910509F482C0C8974F
:10C7800009F038C189C08035910509F489C0883520
:10C79000910509F496C08834910509F02BC1AEC00B
:10C7A0008839910509F413C189399105ECF488376A
:10C7B000910509F4ABC0893791054CF48836910591
:10C7C00009F4A4C08037910509F014C19FC08838CE
:10C7D000910509F4FCC08039910509F49DC08038A9
:10C7E000910509F007C198C0803B910509F4C6C0C6
:10C7F000813B91054CF4803A910509F49FC0883A39
:10C80000910509F0F7C0BAC0803C910509F4E3C076
:10C81000883C910509F4DFC0883B910509F0EAC026
:10C82000C2C08091DD0C8093BB00CFC09091040DFD
:10C830008091050D981768F49091040DE92FF0E0B0
:10C84000EC51F34F80818093BB009F5F9093040D68
:10C85000BCC08091DE0C882309F44BC085ED809329
:10C86000BC008091BC0084FDFCCFC2C080E28093FC
:10C87000490D85ED8093BC008091BC0084FDFCCF08
:10C88000B7C080E38093490D85ED8093BC00809113
:10C89000BC0084FDFCCFACC088E38093490D9BC0F5
:10C8A0008091040D9091BB00E82FF0E0EC51F34F24
:10C8B00090838F5F8093040D9091040D8091050DFE
:10C8C00082C08091040D9091BB00E82FF0E0EC5104
:10C8D000F34F90838F5F8093040D8091DE0C88234B
:10C8E00041F085ED8093BC008091BC0084FDFCCFBD
:10C8F0007FC081E08093DF0C84EA6EC085ED809379
:10C90000BC008091BC0084FDFCCF72C083E08093AA
:10C91000DC0C1092480D59C08091480D803208F00F
:10C9200056C08091480D9091BB00E82FF0E0E85D83
:10C93000F24F90838F5F8093480D47C08091480DE0
:10C94000803230F4E091480DF0E0E85DF24F108263
:10C9500085ED8093BC008091BC0084FDFCCF1092DB
:10C96000DC0C6091480DE091E20CF091E30C88E260
:10C970009DE070E009951092480D2DC084E08093F1
:10C98000DC0C1092260D1092270DE091E00CF09136
:10C99000E10C09958091270D882329F481E080938B
:10C9A000270D1092060D9091260DE92FF0E0EA5F19
:10C9B000F24F80818093BB009F5F9093260D9091F2
:10C9C000260D8091270D981710F485EC01C085E89D
:10C9D0008093BC000FC085EC8093BC0009C010920E
:10C9E000490D85ED8093BC008091BC0084FDFCCF97
:10C9F0001092DC0CFF91EF91BF91AF919F918F91BD
:10CA00007F916F915F914F913F912F910F900FBE4A
:10CA10000F901F9018951092DC0C81E08093DE0C33
:10CA20001092DF0C81E161E00E94EA6580E161E043
:10CA30000E94EA65E9EBF0E080818E7F808380814F
:10CA40008D7F808380E28093B80085E48093BC0072
:10CA50000895982F8E3008F09E5097708091D002E4
:10CA60008295880F880F807C892B80937C00809131
:10CA70007A00806480937A0080917A0086FDFCCFF2
:10CA80002091780040917900942F80E030E0282BAD
:10CA9000392BC90108951F93CF93DF93182FEB0112
:10CAA00061E00E94AB65209709F44AC0CF3FD105F1
:10CAB00009F449C0E12FF0E0E252F44F8491833051
:10CAC000C1F0843028F4813051F08230B1F50CC0CF
:10CAD000863019F1873049F1843079F514C084B576
:10CAE000806884BDC7BD33C084B5806284BDC8BDC5
:10CAF0002EC080918000806880938000D093890050
:10CB0000C093880024C08091800080628093800060
:10CB1000D0938B00C0938A001AC08091B0008068C7
:10CB20008093B000C093B30012C08091B0008062C7
:10CB30008093B000C093B4000AC0C038D1051CF483
:10CB4000812F60E002C0812F61E00E94EA65DF91E1
:10CB5000CF911F910895CF93DF93482F50E0CA01E2
:10CB60008254944FFC0134914256544FFA018491FF
:10CB7000882369F190E0880F991FFC01E058F44F79
:10CB8000A591B491FC01E657F44FC591D491662369
:10CB900051F42FB7F8948C91932F909589238C930F
:10CBA000888189230BC0623061F42FB7F8948C918F
:10CBB000932F909589238C938881832B88832FBF13
:10CBC00006C09FB7F8948C91832B8C939FBFDF9105
:10CBD000CF910895482F50E0CA018252944FFC0132
:10CBE0002491CA018254944FFC0194914256544FAF
:10CBF000FA013491332309F440C0222351F1233048
:10CC000071F0243028F42130A1F0223011F514C045
:10CC10002630B1F02730C1F02430D9F404C080911F
:10CC200080008F7703C0809180008F7D809380008B
:10CC300010C084B58F7702C084B58F7D84BD09C0D4
:10CC40008091B0008F7703C08091B0008F7D80937A
:10CC5000B000E32FF0E0EE0FFF1FE657F44FA59171
:10CC6000B4912FB7F894662321F48C919095892381
:10CC700002C08C91892B8C932FBF0895682F70E090
:10CC8000CB018252944FFC012491CB018254944FEA
:10CC9000FC0144916256744FFB019491992319F45D
:10CCA00020E030E03CC0222351F1233071F02430E9
:10CCB00028F42130A1F0223011F514C02630B1F053
:10CCC0002730C1F02430D9F404C0809180008F77E0
:10CCD00003C0809180008F7D8093800010C084B558
:10CCE0008F7702C084B58F7D84BD09C08091B0006C
:10CCF0008F7703C08091B0008F7D8093B000892F23
:10CD000090E0880F991F8C56944FFC01A591B49127
:10CD10008C9120E030E0842311F021E030E0C90163
:10CD200008951F920F920FB60F9211242F933F93E5
:10CD30004F935F936F937F938F939F93AF93BF9323
:10CD400020914E0D30914F0D4091500D5091510D4D
:10CD50007091520DDA01C9010296A11DB11D672F14
:10CD60006A5F6D3730F06D57DA01C9010396A11D76
:10CD7000B11D6093520D80934E0D90934F0DA09373
:10CD8000500DB093510D80914A0D90914B0DA09193
:10CD90004C0DB0914D0D0196A11DB11D80934A0D12
:10CDA00090934B0DA0934C0DB0934D0DBF91AF914F
:10CDB0009F918F917F916F915F914F913F912F91B3
:10CDC0000F900FBE0F901F9018958FB7F894209179
:10CDD0004E0D30914F0D4091500D5091510D8FBF20
:10CDE000B901CA0108959B01AC017FB7F894809105
:10CDF0004A0D90914B0DA0914C0DB0914D0D66B523
:10CE0000A89B05C06F3F19F00196A11DB11D7FBF02
:10CE1000BA2FA92F982F8827860F911DA11DB11D0C
:10CE200063E0880F991FAA1FBB1F6A95D1F7BC0149
:10CE30002DC0FFB7F89480914A0D90914B0DA091B1
:10CE40004C0DB0914D0DE6B5A89B05C0EF3F19F014
:10CE50000196A11DB11DFFBFBA2FA92F982F8827BA
:10CE60008E0F911DA11DB11DE3E0880F991FAA1F10
:10CE7000BB1FEA95D1F7861B970B885E9340C8F2DB
:10CE8000215030404040504068517C4F21153105C1
:10CE90004105510571F60895019739F0019729F080
:10CEA000880F991F01970197F1F70895789484B539
:10CEB000826084BD84B5816084BD85B5826085BD96
:10CEC00085B5816085BDEEE6F0E08081816080837C
:10CED000E1E8F0E01082808182608083808181605F
:10CEE0008083E0E8F0E0808181608083E1EBF0E026
:10CEF000808184608083E0EBF0E0808181608083CA
:10CF0000EAE7F0E0808184608083808182608083B2
:10CF10008081816080838081806880831092C100DD
:10CF2000089508951F920F920FB60F9211242F9318
:10CF30003F934F938F939F93EF93FF934091C6003E
:10CF40002091930D3091940D2F5F3F4F2F733070D0
:10CF50008091950D9091960D2817390759F0E09121
:10CF6000930DF091940DED5AF24F40833093940D50
:10CF70002093930DFF91EF919F918F914F913F914E
:10CF80002F910F900FBE0F901F901895E091E70D15
:10CF9000F091E80DE05CFF4F81919191208131810A
:10CFA000821B930B8F739070892B11F00E949167F5
:10CFB00008951F920F920FB60F9211242F933F9353
:10CFC0008F939F93EF93FF932091D70D3091D80DBE
:10CFD0008091D90D9091DA0D2817390731F480919D
:10CFE000C1008F7D8093C10014C0E091D90DF091F4
:10CFF000DA0DE956F24F20818091D90D9091DA0D2A
:10D0000001968F7390709093DA0D8093D90D2093D1
:10D01000C600FF91EF919F918F913F912F910F90BB
:10D020000FBE0F901F901895DC011C96ED91FC919E
:10D030001D97E05CFF4F2191319180819181281BE8
:10D04000390B2F733070C9010895DC011C96ED91E6
:10D05000FC911D97E05CFF4F20813181E054F0404E
:10D06000DF01AE5BBF4F8D919C9111972817390757
:10D0700019F42FEF3FEF07C08D919C91E80FF91F36
:10D080008081282F30E0C9010895DC011C96ED91C4
:10D09000FC911D97E05CFF4F20813181E054F0400E
:10D0A000DF01AE5BBF4F8D919C9111972817390717
:10D0B00019F42FEF3FEF10C08D919C911197E80F5D
:10D0C000F91F20818D919C91119701968F7390701B
:10D0D00011969C938E9330E0C9010895FC018685DA
:10D0E0009785DC01A05CBF4FFC01EE5BFF4F2D91EB
:10D0F0003C9111978081918128173907C1F70895D4
:10D10000CF93DF93EC01EE85FF85E05CFF4F20813C
:10D110003181E054F0402F5F3F4F2F733070DF01BB
:10D12000AE5BBF4F8D919C91119728173907D1F3B2
:10D13000E05CFF4F80819181E054F040E80FF91FDF
:10D140006083EE85FF85E05CFF4F31832083EE89AD
:10D15000FF89208181E090E00D8C02C0880F991F2B
:10D160000A94E2F7282B208381E090E0DF91CF91B1
:10D1700008951092DE0D1092DD0D88EE93E0A0E090
:10D18000B0E08093DF0D9093E00DA093E10DB0939C
:10D19000E20D80E593E09093DC0D8093DB0D83E559
:10D1A0009DE09093E80D8093E70D87E99DE09093D3
:10D1B000EA0D8093E90D85EC90E09093EC0D80935F
:10D1C000EB0D84EC90E09093EE0D8093ED0D80ECF0
:10D1D00090E09093F00D8093EF0D81EC90E09093B0
:10D1E000F20D8093F10D86EC90E09093F40D809316
:10D1F000F30D84E08093F50D83E08093F60D87E0D6
:10D200008093F70D85E08093F80D81E08093F90D10
:10D210000895CF92DF92EF92FF920F931F93CF93D7
:10D22000DF937C016B018A01C0E0D0E00FC0D60122
:10D230006D916D01D701ED91FC910190F081E02D90
:10D24000C7010995C80FD91F0150104001151105DC
:10D2500071F7CE01DF91CF911F910F91FF90EF9069
:10D26000DF90CF900895DC01ED91FC910190F08169
:10D27000E02D09950895CF93DF93DB010D900020F9
:10D28000E9F71197A61BB70BEC01E881F981028041
:10D29000F381E02DAD010995DF91CF9108954F9273
:10D2A0005F927F928F929F92AF92BF92CF92DF92C6
:10D2B000EF92FF920F931F93DF93CF93CDB7DEB71B
:10D2C000A1970FB6F894DEBF0FBECDBF2C01742E10
:10D2D000CB01223008F42AE019A231E2C32ED12C6E
:10D2E000CC0EDD1E822E9924AA24BB24672D752F17
:10D2F000A50194010E948A6A79018A01C801B701D7
:10D30000A50194010E94386A472D461B0894C10864
:10D31000D1084A3014F4405D01C0495CF6014083F5
:10D32000E114F1040105110521F07E2C5F2DC801E7
:10D33000DDCFC201B6010E943B69A1960FB6F894F9
:10D34000DEBF0FBECDBFCF91DF911F910F91FF9038
:10D35000EF90DF90CF90BF90AF909F908F907F9095
:10D360005F904F900895DC012115310541F4ED9156
:10D37000FC910190F081E02D642F099508950E94A1
:10D380004F690895EF92FF920F931F939A017B01CB
:10D3900000E010E0B801A7010E94B3691F910F914E
:10D3A000FF90EF900895CF92DF92EF92FF920F934C
:10D3B0001F93CF93DF93EC016A017B0121153105A7
:10D3C00041F4E881F9810190F081E02D642F099505
:10D3D0001FC02A303105D1F477FF17C0E881F981E9
:10D3E0000190F081E02D6DE209958C0144275527CD
:10D3F000BA014C195D096E097F09CE012AE00E942D
:10D400004F699801280F391F04C02AE00E944F6914
:10D410009C01C901DF91CF911F910F91FF90EF9077
:10D42000DF90CF900895EF92FF920F931F937B01AF
:10D430009A010027F7FC0095102FB801A7010E9460
:10D44000D3691F910F91FF90EF9008950E943B695F
:10D450000895CF93DF930E9456670E945E24C6EC26
:10D46000D7E60E94EC252097E1F30E94C667F9CF2A
:10D47000629FD001739FF001829FE00DF11D649FB8
:10D48000E00DF11D929FF00D839FF00D749FF00D44
:10D49000659FF00D9927729FB00DE11DF91F639FE5
:10D4A000B00DE11DF91FBD01CF0111240895991B95
:10D4B00079E004C0991F961708F0961B881F7A958B
:10D4C000C9F780950895AA1BBB1B51E107C0AA1F8D
:10D4D000BB1FA617B70710F0A61BB70B881F991F15
:10D4E0005A95A9F780959095BC01CD01089597FBB9
:10D4F000092E07260AD077FD04D0E5DF06D00020EC
:10D500001AF4709561957F4F0895F6F7909581957F
:10D510009F4F0895A1E21A2EAA1BBB1BFD010DC04F
:10D52000AA1FBB1FEE1FFF1FA217B307E407F507D3
:10D5300020F0A21BB30BE40BF50B661F771F881FAF
:10D54000991F1A9469F760957095809590959B0145
:10D55000AC01BD01CF01089597FB092E05260ED021
:10D5600057FD04D0D7DF0AD0001C38F45095409501
:10D57000309521953F4F4F4F5F4F0895F6F79095A7
:10D580008095709561957F4F8F4F9F4F0895EE0F57
:10D59000FF1F0590F491E02D09942F923F924F9236
:10D5A0005F926F927F928F929F92AF92BF92CF9233
:10D5B000DF92EF92FF920F931F93CF93DF93CDB73C
:10D5C000DEB7CA1BDB0B0FB6F894DEBF0FBECDBFB4
:10D5D00009942A88398848885F846E847D848C8485
:10D5E0009B84AA84B984C884DF80EE80FD800C818E
:10D5F0001B81AA81B981CE0FD11D0FB6F894DEBF71
:0CD600000FBECDBFED010895F894FFCFE0
:10D60C00687474703A2F2F75692E6F70656E737015
:10D61C0072696E6B6C65722E636F6D2F6A73002E60
:10D62C0063677A002E6A677A002F00763D5B00777D
:10D63C006C00616C6C00743D5B0000727300726472
:10D64C00000D0A0000323030002E0076006F70653D
:10D65C006E646F6F7200426F73746F6E2C4D41006D
:10D66C00687474703A2F2F75692E6F70656E7370B5
:10D67C0072696E6B6C65722E636F6D2F6A7300002E
:10D68C002F6C6F67732F003A013B013E012F01870E
:10D69C000008118A00710F8D0070199000E4199325
:10D6AC00003E209600450B9900FF189C00BC1E9F65
:10D6BC00004C13A2008610A500C509A800EC21ABF4
:10D6CC00005213AE00A414B100201BB4007E1EB790
:10D6DC00002F0ABA00DC107B100E0000010A50006B
:10D6EC00D300DB083C081C6CE60840080101ED087F
:10D6FC0043080101F208470800FFFC084C0800FF32
:10D70C000809500800FF1409540800FF20095808A4
:10D71C0000FF2C095C0800FF3909600800FF46096E
:10D72C00640800FF5309680850FF60096C0800FF8B
:10D73C006B09700814006C097408000577097808E7
:10D74C00010183097C0880F784097E0800088F0991
:10D75C008208003C9D0986083C78AC098B080001C6
:10D76C00BB0990080101C809940864FAD709980804
:10D77C000101E5099B080001F4099F0800FF020A5A
:10D78C00A4086EFF0B0AAA0864FF190AAE080FFF63
:10D79C00280AB20800C8350AB6080005420ABA08B9
:10D7AC00CCFF4F0ABE0809FF580AC30836FF610AAE
:10D7BC00C80877FF6A0ACD080101730AD208000174
:10D7CC00830AD5084F532D303000638253633501E3
:10D7DC000100000000A60709696F000000000000AE
:10D7EC00002E6F4F1F1C1F1E1F1E1F1F1E1F1E1FD4
:10D7FC00FFFFFFFFFFFF00000703050810000000FC
:10D80C0006091F00151500001F111F11131E00140F
:10D81C00081501050515FFFFFFFFFFFF00000000C5
:10D82C007148096900004000140054000000000019
:10D83C001D51096900000000B36109690000000076
:10D84C005E622D62E661EF61046215620000000009
:0CD85C00806809691468456825686E68DA
:00000001FF
